:020000040000FA
:1020000002AABB02DA058F27AFA775A70F8FA77F9C
:10201000327E0012D222E52724FF92B47FE87E03AD
:1020200002D22202D2E4D286D2872202D62C7D01AD
:102030007F8012A855901B9DE0FEA3E02400FFE4E2
:102040003EFEC36480948050066307FF6306FF7CF6
:10205000007D021227FDE51B2FFFE51A3EFE7C00E6
:0A2060007D021227FD8E1A8F1B224D
:10206B0002D5EA7D1AAF16AE15129C1112D7347D2C
:10207B0018AF16AE15129C1112D46F900968740329
:10208B00F09009677409F02202C77E8F27AFA775FE
:10209B00A70F8FA77F327E0012D222E52724FF9253
:1020AB00B57FC87E0002D22202D6D9E590540C230C
:1020BB00C0E074D7C0E0C082C08302D700E5905463
:1020CB000C23C0E074D7C0E0C082C08302D708E500
:1020DB0090540C23C0E074D7C0E0C082C08302D7F9
:1020EB0010E590540C23C0E074D7C0E0C082C083CD
:0A20FB0002D718EFC40390D700735A
:1021060002244EE86480F8E933E83360110460F095
:10211600ED33EC337009E8FCE9FDEAFEEBFF22043F
:1021260060DED3EB9FEA9EE99DE8C2E78CF0C2F73A
:1021360095F0400CE8CCF8E9CDF9EACEFAEBCFFB06
:1021460012241985D0F05804700320D5B3E8047022
:10215600075002B2D502245892D5EC0460F7E4CCBD
:10216600C0E0C398F8603B94186008400DD0E0FBCF
:10217600022430E4FBFAC9FC8028E830E406E4C90E
:10218600FBE4CAFCE830E305E4C9CACBFCE8540723
:102196006010F8C3E913F9EA13FAEB13FBEC13FC2E
:1021A600D8F130F52FC3E49CFCEF9BFFEE9AFEEDD1
:1021B60099FDD0E0FBEF4E4D4C701222DB0302245A
:1021C60055EC2CFCEF33FFEE33FEED33FDED30E73F
:1021D600EB022430EF2BFFEE3AFEED39FDD0E0FBAB
:1021E60050130BBB0003022458ED13FDEE13FEEF54
:1021F60013FFEC13FC022430EC4D6011E849701714
:10220600ED33EC3304600DE4FCFFFEFD22E933E818
:10221600330470F802244E12241958046009E4CCE1
:1022260024815006285009022458284003022455C8
:10223600C0E0EB4A7044B98006D0E0FB022444EFCC
:102246004E701CBD8008EBFFEAFEE9FD80EBE98DD0
:10225600F0A4FEE5F00222E7E9CDF9EAFEEBFFEF96
:1022660089F0A4FCE5F0CE89F0A42EFFE435F0CD8C
:1022760089F0A42DFEE435F08067EF4E7005BD8031
:10228600D780C3EF8BF0A4ACF0EE8BF0A42CFCE46B
:1022960035F0F8EF8AF0A42CE5F038FCE433CB8D6A
:1022A600F0A42CFCE5F03BF8EE8AF0A42CFCE5F05B
:1022B60038F8E433CF89F0A42CFCE5F038CF3400AD
:1022C600CE89F0A42FFFE5F03EFEE433C98DF0A4DD
:1022D6002EFEE5F039CD8AF0A42FFFE5F03EFEE4B0
:1022E6003DFD33D0E0FB50070BBB000F022458EC3A
:1022F6002CFCEF33FFEE33FEED33FD0224300224D7
:1023060058EC5D046005E85904700302244E12245B
:1023160019580460F6EC4860F2EC7004FDFEFF22EA
:10232600C860DB2481C85009C398600250060224A5
:10233600559850CAF582E9294B4A7005AB820224AA
:102346004475F0007C1A7880C3EF9BEE9AED9940B5
:102356000DC3EF9BFFEE9AFEED99FDE842F0DC23FC
:10236600ACF0D0E0FFD0E0FED0E0FDAB8220E7107D
:102376001BEB60BAEC2CFCEF33FFEE33FEED33FDC6
:10238600022430E803F830E705C0F075F000EF2FBF
:10239600FFEE33FEED33FD40B830E7C280AA75F09C
:1023A60020800E75F010800575F0087D007E007F98
:1023B600003392D530D5031229E1EC334010EF33C8
:1023C600FFEE33FEED33FDEC33FCD5F0ED22E5F008
:1023D600247EA2D513CC92E7CDCEFF22EDD2E7CD57
:1023E60033EC3392D524814006E4FFFEFDFC22FC4B
:1023F600E4CFCECDCC24E0501174FF80EDC3CC13D6
:10240600CCCD13CDCE13CECF13CF0470F030D5DEA6
:102416000229E1E9D2E7C933E833F892D5EDD2E7EC
:10242600CD33EC33FC5002B2D522EC30E7100FBFAF
:10243600000C0EBE00080DBD00040BEB6014A2D507
:10244600EB13FCED92E7FD2274FFFCFDFEFF22E498
:1024560080F8A2D574FF13FC7D80E480EFF920E7B5
:102466002824F950037907E4F42402FB18DBFDE67F
:1024760024FB5014E9600DE4F618E604F6B40A08E5
:10248600E4F6D9F57401F60A22C2D522ED33EC330F
:1024960092D5FA602AB4FF33EDC2E77BFF60067A75
:1024A6002479B7E4227A2479C020D5047A2479BB2A
:1024B600224E614E002B494E46002D494E4600E401
:1024C6007A08F608DAFC7B00740722E8C0E0ECC064
:1024D600E0EDC0E0EEC0E0EFC0E0EA75F010A4CA9F
:1024E600ABF075F04DA42BFBE435F0FCEA2410FAB2
:1024F600EB34C5FBEC34D9FCEDC2E7FF75F056A40E
:10250600F42411C5F0F434C58FF0A42AE5F03BE4B9
:102516003CF620E7141225C5D0E0FFD0E0FED0E05F
:10252600FDD0E0FC1223078014F4041225C5D0E088
:10253600FFD0E0FED0E0FDD0E0FC1221FED0E0F8B6
:10254600E6FAEDD2E7CD33EC332482FBE4C3CF3396
:10255600CFCE33CECD33CD33DBF37B0775F00A8494
:102566006004F6081B0AE5F0F6088FF0740AA4FF6B
:10257600ACF08EF0740AA42CFEACF050010C8DF079
:10258600740AA42CFDE435F0F608DBDE7407223F5E
:102596008000004120000042C80000447A00004646
:1025A6001C400047C35000497424004B1896804CC9
:1025B600BEBC205A0E1BCA6753C21C749DC5AEFB17
:1025C60060065407601C23231225F3EB5438600978
:1025D6001225DF1225EE1221FEECF8EDF9EEFAEFE8
:1025E600CB22EB1225EE80F1543803241C9025955E
:1025F600FE93FC0EEE93FD0EEE930ECE93FF22E7B6
:1026060009F608DFFA8046E709F208DFFA803E8815
:10261600828C83E709F0A3DFFA8032E309F608DF4C
:10262600FA8078E309F208DFFA807088828C83E307
:1026360009F0A3DFFA806489828A83E0A3F608DFC3
:10264600FA805889828A83E0A3F208DFFA804C80F8
:10265600D280FA80C680D4806980F2803380108070
:10266600A680EA809A80A880DA80E280CA803389D0
:10267600828A83ECFAE493A3C8C582C8CCC583CC0E
:10268600F0A3C8C582C8CCC583CCDFE9DEE7800DE0
:1026960089828A83E493A3F608DFF9ECFAA9F0EDC0
:1026A600FB2289828A83ECFAE0A3C8C582C8CCC51E
:1026B60083CCF0A3C8C582C8CCC583CCDFEADEE8EC
:1026C60080DB89828A83E493A3F208DFF980CC88D1
:1026D600F0EF60010E4E60C388F0ED2402B40400F2
:1026E60050B9F582EB2402B4040050AF232345828F
:1026F6002390265573BB010689828A83E022500205
:10270600E722BBFE02E32289828A83E49322BB018D
:102716000CE58229F582E5833AF583E0225006E945
:102726002582F8E622BBFE06E92582F8E222E5824A
:1027360029F582E5833AF583E49322BB010FF8E598
:102746008229F582E5833AF583E028F0225009C50F
:102756008229F8E58226F622BBFE09C58229F8E21F
:102766002582F222F8EA2583F583E9932822BB0124
:102776000689828A83F0225002F722BBFE01F322E9
:10278600F8BB010DE58229F582E5833AF583E8F089
:10279600225006E92582C8F622BBFE05E92582C835
:1027A600F222BC000BBE0029EF8DF084FFADF022B3
:1027B600E4CCF875F008EF2FFFEE33FEEC33FCEEB9
:1027C6009DEC984005FCEE9DFE0FD5F0E9E4CEFDAC
:1027D60022EDF8F5F0EE8420D21CFEADF075F0087F
:1027E600EF2FFFED33FD4007985006D5F0F222C3D8
:1027F60098FD0FD5F0EA22C2D5EC30E709B2D5E450
:10280600C39DFDE49CFCEE30E715B2D5E4C39FFF03
:10281600E49EFE1227A8C3E49DFDE49CFC800312FF
:1028260027A830D507C3E49FFFE49EFE22C5F0F833
:10283600A3E028F0C5F0F8E582158270021583E062
:1028460038F022A3F8E0C5F025F0F0E58215827095
:10285600021583E0C838F0E822BB0110E58229F5AD
:1028660082E5833AF583E0F5F0A3E0225009E925F5
:1028760082F886F008E622BBFE0AE92582F8E2F530
:10288600F008E222E5832AF583E993F5F0A3E993BC
:1028960022F8BB0111E58229F582E5833AF583E842
:1028A600F0E5F0A3F0225009E92582C8F608A6F063
:1028B60022BBFE09E92582C8F2E5F008F222E88F7C
:1028C600F0A4CC8BF0A42CFCE98EF0A42CFC8AF0AE
:1028D600EDA42CFCEA8EF0A4CDA8F08BF0A42DCCB0
:1028E6003825F0FDE98FF0A42CCD35F0FCEB8EF009
:1028F600A4FEA9F0EB8FF0A4CFC5F02ECD39FEE4EF
:102906003CFCEAA42DCE35F0FDE43CFC2275F00833
:10291600758200EF2FFFEE33FECD33CDCC33CCC521
:102926008233C5829BED9AEC99E58298400CF5823C
:10293600EE9BFEED9AFDEC99FC0FD5F0D6E4CEFBAE
:10294600E4CDFAE4CCF9A88222B800C1B90059BA9C
:10295600002DEC8BF084CFCECDFCE5F0CBF97818CA
:10296600EF2FFFEE33FEED33FDEC33FCEB33FB10C4
:10297600D703994004EB99FB0FD8E5E4F9FA2278DE
:1029860018EF2FFFEE33FEED33FDEC33FCC933C9F0
:1029960010D7059BE99A4007EC9BFCE99AF90FD8FA
:1029A600E0E4C9FAE4CCFB2275F010EF2FFFEE331A
:1029B600FEED33FDCC33CCC833C810D7079BEC9A59
:1029C600E899400AED9BFDEC9AFCE899F80FD5F0E2
:1029D600DAE4CDFBE4CCFAE4C8F922C3E49FFFE4D1
:1029E6009EFEE49DFDE49CFC22EB9FF5F0EA9E42F0
:1029F600F0E99D42F0EC6480C864809845F022EBD3
:102A06009FF5F0EA9E42F0E99D42F0E89C45F022EF
:102A1600E8600FECC313FCED13FDEE13FEEF13FF9E
:102A2600D8F122E8600FEFC333FFEE33FEED33FD3E
:102A3600EC33FCD8F1227401FF3395E0FEFDFC086F
:102A46000808E6CF2FF618E6CE3EF618E6CD3DF698
:102A560018E6CC3CF622ECF0A3EDF0A3EEF0A3EFE3
:102A6600F022A8828583F0D083D082122A7F122A90
:102A76007F122A7F122A7FE473E493A3C583C5F0ED
:102A8600C583C8C582C8F0A3C583C5F0C583C8C5BC
:102A960082C822A42582F582E5F03583F58322FAE1
:102AA600E6FB0808E6F925F0F618E6CA3AF622D05B
:102AB60083D082F8E4937012740193700DA3A393EC
:102AC600F8740193F5828883E4737402936860EF67
:102AD600A3A3A380DFD083D082E493701274019302
:102AE600700DA3A393F8740193F5828883E473743D
:102AF60002936C70127403936D700C7404936E7071
:102B0600067405936F60DDA3A3A3A3A3A380CAE302
:102B1600F5F009E208B5F06D606B80F3E3F5F009B6
:102B2600E608B5F060605E80F387F009E608B5F068
:102B360054605280F487F009E208B5F04860468098
:102B4600F488828C8387F009E0A3B5F0386036807C
:102B5600F488828C8387F009E493A3B5F027602577
:102B660080F388828C83E3F5F009E0A3B5F0166064
:102B76001480F388828C83E3F5F009E493A3B5F01F
:102B860004600280F2022C40808580E7808E80D22D
:102B9600803C8015806C807E809B80B5808B80A178
:102BA600804F8070803A022C4C89828A83ECFAE44A
:102BB60093F5F0A3C8C582C8CCC583CCE493A3C85B
:102BC600C582C8CCC583CCB5F070606E80E18982C1
:102BD6008A83E493F5F0A3E208B5F05E605C80F2C8
:102BE60089828A83E0F5F0A3E608B5F04D604B8054
:102BF600F389828A83E0F5F0A3E208B5F03C603AF7
:102C060080F389828A83E493F5F0A3E608B5F02A77
:102C1600602880F2805389828A83ECFAE493F5F087
:102C2600A3C8C582C8CCC583CCE0A3C8C582C8CC1E
:102C3600C583CCB5F004600280E27FFFB5F0020FD9
:102C46002240027F012289828A83ECFAE0F5F0A312
:102C5600C8C582C8CCC583CCE0A3C8C582C8CCC5CC
:102C660083CCB5F0D560D380E389828A83ECFAE021
:102C7600F5F0A3C8C582C8CCC583CCE493A3C8C568
:102C860082C8CCC583CCB5F0B160AF80E288F0EDE8
:102C96002402B4040050A3F582EB2402B4040050CD
:102CA600992323458223902B8E73E3F5F009E208DE
:102CB600B5F06BDFF58067E3F5F009E608B5F05E81
:102CC600DFF5805A87F009E608B5F052DFF6804E48
:102CD60087F009E208B5F046DFF6804288828C83E9
:102CE60087F009E0A3B5F036DFF6803288828C8360
:102CF60087F009E493A3B5F025DFF5802188828C5F
:102D060083E3F5F009E0A3B5F014DFF580108882BF
:102D16008C83E3F5F009E493A3B5F002DFF4022D0A
:102D2600DF808780E9809080D4803E8015806E8029
:102D36007E809D80B7808D80A380518074803C0208
:102D46002DEB89828A83ECFAE493F5F0A3C8C58259
:102D5600C8CCC583CCE493A3C8C582C8CCC583CCF4
:102D6600B5F076DFE3DEE1807089828A83E493F54D
:102D7600F0A3E208B5F062DFF4805E89828A83E020
:102D8600F5F0A3E608B5F051DFF5804D89828A8318
:102D9600E0F5F0A3E208B5F040DFF5803C89828AD1
:102DA60083E493F5F0A3E608B5F02EDFF4802A80DD
:102DB60002805789828A83ECFAE493F5F0A3C8C5AA
:102DC60082C8CCC583CCE0A3C8C582C8CCC583CC99
:102DD600B5F006DFE4DEE280007FFFB5F0020F22E9
:102DE60040027F012289828A83ECFAE0F5F0A3C8CB
:102DF600C582C8CCC583CCE0A3C8C582C8CCC58370
:102E0600CCB5F0D5DFE5DEE380CF89828A83ECFAA4
:102E1600E0F5F0A3C8C582C8CCC583CCE493A3C8AB
:102E2600C582C8CCC583CCB5F0AFDFE4DEE280A9AD
:102E360088F0EF60010E4E60ABED2402B404005042
:102E460098F582EB2402B40400508E232345822396
:102E5600902D2773EF4E6012EF60010EEDBB010B54
:102E660089828A83F0A3DFFCDEFA2289F05007F715
:102E760009DFFCA9F022BBFEFCF309DFFCA9F02266
:102E8600EF8DF0A4A8F0CF8CF0A428CE8DF0A42E60
:102E9600FE2278A37C097D017BFF7AE27988122CD9
:102EA60093EF3395E04F700302C18D78A37C097DC3
:102EB600017BFF7AE2798F122C93EF3395E04F7006
:102EC6000302500578A37C097D017BFF7AE2799C99
:102ED600122C93EF3395E04F700302C8D178A37C90
:102EE600097D017BFF7AE279A1122C93EF3395E0FD
:102EF6004F700302930F78A37C097D017BFF7AE272
:102F060079A6122C93EF3395E04F700302AE1B782F
:102F1600A37C097D017BFF7AE279AB122C93EF3318
:102F260095E04F700302BCD578A37C097D017BFF39
:102F36007AE279B3122C93EF3395E04F700302DAFD
:102F46001978A37C097D017BFF7AE279B7122C936D
:102F5600EF3395E04F700302D78D78A37C097D018E
:102F66007BFF7AE279BB122C93EF3395E04F700327
:102F760002654378A37C097D017BFF7AE279C5125D
:102F86002C93EF3395E04F700302674778A37C09D3
:102F96007D017BFF7AE279CD122C93EF3395E04FDA
:102FA60070030270CD78A37C097D017BFF7AE279FC
:102FB600D2122C93EF3395E04F700302632B78A364
:102FC6007C097D017BFF7AE279D9122C93EF339548
:102FD600E04F700302760578A37C097D017BFF7ABA
:102FE600E279DC122C93EF3395E04F70030235C083
:102FF60078A37C097D017BFF7AE279E2122C93EFBC
:103006003395E04F700302A71778A37C097D017BF7
:10301600FF7AE279E8122C93EF3395E04F700302C2
:10302600A7B678A37C097D017BFF7AE279EE122CA4
:1030360093EF3395E04F700302BD4778A37C097D7B
:10304600017BFF7AE279F4122C93EF3395E04F700F
:1030560003026EF378A37C097D017BFF7AE279FE99
:10306600122C93EF3395E04F700302DA3D78A37C80
:10307600097D017BFF7AE37909122C93EF3395E002
:103086004F700302963C78A37C097D017BFF7AE3AF
:103096007913122C93EF3395E04F700302CD6978C4
:1030A600A37C097D017BFF7AE3791F122C93EF3312
:1030B60095E04F70030247D078A37C097D017BFF22
:1030C6007AE37925122C93EF3395E04F700302D9FA
:1030D600E378A37C097D017BFF7AE3792C122C939C
:1030E600EF3395E04F700302D9EC78A37C097D019C
:1030F6007BFF7AE37932122C93EF3395E04F70031E
:1031060002D7F478A37C097D017BFF7AE379361236
:103116002C93EF3395E04F700302D6F278A37C0927
:103126007D017BFF7AE3793B122C93EF3395E04FD9
:1031360070030283C778A37C097D017BFF7AE3795C
:1031460044122C93EF3395E04F7002801678A37CDF
:10315600097D017BFF7AE3794A122C93EF3395E0E0
:103166004F700302D3F178A37C097D017BFF7AE3DC
:103176007950122C93EF3395E04F7002801678A3A6
:103186007C097D017BFF7AE37955122C93EF339509
:10319600E04F700302593178A37C097D017BFF7AE9
:1031A600E3795E122C93EF3395E04F700280167828
:1031B600A37C097D017BFF7AE37969122C93EF33B7
:1031C60095E04F700302D4C078A37C097D017BFF94
:1031D6007AE37974122C93EF3395E04F700302A5CE
:1031E600D778A37C097D017BFF7AE3797F122C9344
:1031F600EF3395E04F700302A67778A37C097D0133
:103206007BFF7AE3798B122C93EF3395E04F7003B3
:10321600028A0F78A37C097D017BFF7AE3799F12EE
:103226002C93EF3395E04F7003029E1E78A37C0922
:103236007D017BFF7AE379B2122C93EF3395E04F51
:10324600700302AD0178A37C097D017BFF7AE379E7
:10325600BE122C93EF3395E04F700302C92578A375
:103266007C097D017BFF7AE379CB122C93EF3395B2
:10327600E04F700302D97F78A37C097D017BFF7A3A
:10328600E379D5122C93EF3395E04F700302CDFA14
:1032960078A37C097D017BFF7AE379E4122C93EF16
:1032A6003395E04F700302D97278A37C097D017BC8
:1032B600FF7AE379EE122C93EF3395E04F70030219
:1032C600B93278A37C097D017BFF7AE379FF122C62
:1032D60093EF3395E04F7003029CC178A37C097D80
:1032E600017BFF7AE4790F122C93EF3395E04F7050
:1032F6000302D8AE78A37C097D017BFF7AE47927A7
:10330600122C93EF3395E04F700302D8BF78A37C5D
:10331600097D017BFF7AE4793D122C93EF3395E02A
:103326004F7003027ACB78A37C097D017BFF7AE498
:103336007949122C93EF3395E04F700302C6CF788C
:10334600A37C097D017BFF7AE4795B122C93EF3332
:1033560095E04F700302C9CB78A37C097D017BFF02
:103366007AE47967122C93EF3395E04F7003029E4F
:10337600CB78A37C097D017BFF7AE47974122C93C8
:10338600EF3395E04F7003028EB178A37C097D017F
:103396007BFF7AE47985122C93EF3395E04F700327
:1033A60002AC7078A37C097D017BFF7AE4799512E3
:1033B6002C93EF3395E04F700302AD8E78A37C0912
:1033C6007D017BFF7AE479A2122C93EF3395E04FCF
:1033D600700302B45578A37C097D017BFF7AE479FA
:1033E600A8122C93EF3395E04F700302B4D378A361
:1033F6007C097D017BFF7AE479B5122C93EF339536
:10340600E04F700302D55E78A37C097D017BFF7ACD
:10341600E479C4122C93EF3395E04F700302D80879
:1034260078A37C097D017BFF7AE479D5122C93EF92
:103436003395E04F700302CF9178A37C097D017B21
:10344600FF7AE479E3122C93EF3395E04F70030291
:10345600BE2878A37C097D017BFF7AE479EB122CE8
:1034660093EF3395E04F7003029B5B78A37C097D55
:10347600017BFF7AE479F3122C93EF3395E04F70DA
:103486000302A49778A37C097D017BFF7AE479FC8B
:10349600122C93EF3395E04F700302A53778A37C87
:1034A600097D017BFF7AE57905122C93EF3395E0D0
:1034B6004F700302D60B78A37C097D017BFF7AE56A
:1034C600790E122C93EF3395E04F700302D8D07823
:1034D600A37C097D017BFF7AE57914122C93EF33E7
:1034E60095E04F700302B9AC78A37C097D017BFFA0
:1034F6007AE5791C122C93EF3395E04F700302BEE8
:103506009778A37C097D017BFF7AE57924122C93B9
:10351600EF3395E04F700302D92B78A37C097D0128
:103526007BFF7AE5792F122C93EF3395E04F7003EA
:1035360002A0C678A37C097D017BFF7AE5793B1260
:103546002C93EF3395E04F700302D12378A37C09C7
:103556007D017BFF7AE5794A122C93EF3395E04F94
:10356600700302D4E878A37C097D017BFF7AE579B4
:1035760055122C93EF3395E04F700302A98D78A373
:103586007C097D017BFF7AE5795D122C93EF3395FB
:10359600E04F700302B25378A37C097D017BFF7A6A
:1035A600E57965122C93EF3395E04F70030281762F
:1035B6007BFF7AE579681243C322901B47E0FCA3A0
:1035C600E0FDA3E0FEA3E02401FFE43EFEE43DFDB2
:1035D600E43CFC901B47122A5C901BA6122A68004A
:1035E600000010E4901BA2F0A3F0900987E070069B
:1035F6009009B374FFF0E4901BA2F0A3F090098742
:10360600E0FF901BA2E0FCA3E0FDC39FEC9400400A
:1036160003023951901B6775F013ED122A99EC7568
:10362600F013A42583F583E0FEA3E024B3F58274AA
:10363600093EAF82F5228F23901B5E75F013ED12C3
:103646002A99EC75F013A42583F583E0FCA3E0FD2D
:10365600A3E0FEA3E0F52F8E2E8D2D8C2C7F007E11
:10366600367D6E7C0112D00B901BA2E0FEA3E0FF1C
:10367600901B6475F013122A99EE75F013A4258336
:10368600F583E0FDD394017480948050030238E002
:103696007C00901B6975F013EF122A99EE75F013F2
:1036A600A42583F583E0FEA3E0FF1227A8901BA4C0
:1036B600ECF0A3EDF04C7036901BA2E0FEA3E0FF09
:1036C600901B6B75F013122A99EE75F013A42583DF
:1036D600F583E07D0070027D01901B6B75F013EFA2
:1036E600122A99EE75F013A42583F583EDF0901B4D
:1036F600A2E0FEA3E0FF901B6975F013122A99EE73
:1037060075F013A42583F583E475F0011228339030
:103716001B5A75F013EF122A99EE75F013A4258340
:10372600F583E0FCA3E0FDA3E0FEA3E0FFE47BB0AD
:10373600FAF9F8C3122A0570597F407E427D0FFCC4
:10374600901BA2E0FAA3E0901B5E75F013122A9973
:10375600EA75F013A42583F583122A5C12DA2C90FD
:103766001BA2E0FEA3E0901B6B75F013122A99EEE4
:1037760075F013A42583F583E0FF12D88C12DA3096
:10378600901BA4A3E0540F04901BAAF044B0F002CF
:103796003861901BA2E0FEA3E0901B5A75F013124D
:1037A6002A99EE75F013A42583F583E0FCA3E0FDCA
:1037B600A3E0FEA3E0FFE47BC0FAF9F8C3122A05F2
:1037C6007037901BA2E0FEA3E0901B6B75F01312FE
:1037D6002A99EE75F013A42583F583E02482F582F9
:1037E600E43409F583E0FF901BA4A3E0FEEF4E044A
:1037F600901BAAF044C0F08062901BA2E0FEA3E0FA
:10380600901B5A75F013122A99EE75F013A42583AE
:10381600F583E0FCA3E0FDA3E0FEA3E0FFE47BA1CB
:103826007A16F9F8C3122A057031901BA2E0FEA39E
:10383600E0901B6B75F013122A99EE75F013A42510
:1038460083F583E02482F582E43409F583E0FF9072
:103856001BA4A3E0FEEF4E901BAAF0901BA2E0FE75
:10386600A3E0901B5A75F013122A99EE75F013A473
:103876002583F583E0FCA3E0FDA3E0FEA3E0540F5F
:10388600FFE4FBFAF9F8C3122A057019E5232401AF
:10389600FFE43522FE901BAAE0FB901BA2A3E0F5F5
:1038A6002EE4FD8017E5232401FFE43522FE901B5C
:1038B600AAE0FB901BA2A3E0F52E7D0112565878D4
:1038C600AB7C1B7D017E007F031226D5901BAAE0F0
:1038D600852382852283A3F08024E5232401FFE447
:1038E6003522FE901BA2A3E0F52E7B01E4FD1256C5
:1038F6005878AB7C1B7D017E007F031226D5901B7A
:10390600ABE0852382852283F0901BA6E0F8A3E036
:10391600F9A3E0FAA3E0FB901BADE02401FF901BA6
:10392600ACE03400FEE4FCFDEB2FFFEA3EFEED3991
:10393600FDEC38FC901BA6122A5C901BA3E004F059
:103946007006901BA2E004F00236037E097FA312E4
:10395600803AE4901BAAF0FF7E0CFDFC901BA6E0CB
:10396600F8A3E0F9A3E0FAA3E0FBD3122A05400A84
:103976007E097FA37D007C108046E4FF7E08FDFC67
:10398600901BA6E0F8A3E0F9A3E0FAA3E0FBD312AC
:103996002A05400A7E097FA37D007C0C8022E4FF75
:1039A6007E04FDFC901BA6E0F8A3E0F9A3E0FAA3D1
:1039B600E0FBD3122A0540127E097FA37D007C0816
:1039C60012D41C901BAAEFF08005901BAAE4F012FB
:1039D600D921E4901BA2F0A3F0901BA2E0FEA3E085
:1039E600FFC3EE9404501F74A32FF58274093EF5AD
:1039F60083E0FF12D8FE901BA3E004F070DB901B5F
:103A0600A2E004F080D3E4FF7E04FDFC901BA6E058
:103A1600F8A3E0F9A3E0FAA3E0FBC3122A055008D5
:103A2600901BAAE0FF12D8FEE4901BA2F0A3F09030
:103A36001BA2E0FEA3E0FFC3EE9404501C74A32F68
:103A4600F58274093EF583E4F0901BA3E004F07060
:103A5600DE901BA2E004F080D6221294B18F118E64
:103A6600108D0F8C0E12C50DEF60277D09AF16AEB7
:103A760015129C117E087F007D007B017A0079007B
:103A8600122E5A7400440060097D12AF16AE15124C
:103A96009C11E4F522F52374002523F58274003584
:103AA60022F583E0FF74A22523F582741B3522F5E7
:103AB60083EFF00523E52370020522640845227092
:103AC600D67E117F947D007B017A0979A3122E5A46
:103AD60078A37C097D017B017A0079007E047F0052
:103AE6001226D5E4F52EF52F7F807E08FDFC12897F
:103AF600127E097F607D007B017A007900122E5AC2
:103B060012C50DEF60097D09AF16AE15129C119016
:103B160000B8E09000CAF09000B9E09000CBF090B9
:103B260000BAE09000CCF09000BBE09000CDF090A1
:103B360000BCE09000CEF09000BDE09000CFF09089
:103B460000BEE09000D0F0900991E0FF9000D3F025
:103B5600900992E0FE9000D4F0900993E0FD900069
:103B6600D5F0900994E0FC9000D6F0900995E0FB22
:103B76009000D7F0900996E0F99000D8F090099758
:103B8600E0FA9000D9F0E4900031F0900025EFF0D3
:103B9600A3EEF0A3EDF0A3ECF0A3EBF0A3E9F0A302
:103BA600EAF0900991E09000DCF0900992E0900034
:103BB600DDF0900993E09000DEF0900994E090002B
:103BC600DFF0900995E09000E0F0A3E9F090099706
:103BD600E09000E2F07E087F007D007B017A0979A3
:103BE600A3122E5AE4F522F52374002523F58274D8
:103BF600003522F583E0FF74A32523F58274093589
:103C060022F583EFF00523E52370020522B400D9DF
:103C1600E522B404D47E097FA37DFE7C0312D41C66
:103C2600900DA1EFF07B017A0979A37DFF7C031249
:103C3600D0EE900DA2EFF0E4FFFE12A3F6E4F52E0F
:103C4600F52F7F907E08FDFC1289127E087F007D8D
:103C5600007B017A0979A3122E5AE5112470FFE53B
:103C66001034F7FEE50F34FFFDE50E34FFFCE4FBF0
:103C76007A08F9F81228C48F278E268D258C247889
:103C86000E122A3CE4F52EF52F128912AF11AE1052
:103C9600AD0FAC0EE4F52EF52F128912AD19AC1846
:103CA600AF16AE1512AF32AD19AC18AF16AE15126F
:103CB600AFBD900979E07E008E22F52375F020A431
:103CC600FF90097BE07C002FFDEC35F0FC90097835
:103CD600E02414FFEF7F0025E0FEEF2DFFEC3E9081
:103CE6001BCAF0A3EFF090097DE075F020A4FFA3B6
:103CF600E0C3137C002FFDEC35F0FC90097CE07FDF
:103D06000033333354F8FEEF2DFFEC3E901BCCF01E
:103D1600A3EFF078AA7C1B7D017BFF7AE9797F7E91
:103D2600007F201226D5901BCCE0FEA3E0F9901B65
:103D3600B8F0EEFDA3F0901BCAE0FEA3E0901BBA1C
:103D4600F0EEFFFCA3F0901BCAA3E0FB901BBCF0B7
:103D5600A3ECF0901BC0E9F0A3EDF0A3EBF0A3EF0A
:103D6600F078A37C097D017B017A1B79AA7E007F0E
:103D7600201226D578AA7C1B7D017BFF7AE9795F24
:103D86007E007F201226D5901BCCE0FEA3E0F990A2
:103D96001BB8F0EEFDA3F0901BCAE0FEA3E0901B5B
:103DA600BAF0EEFFFCA3F0901BCAA3E0FB901BBC8D
:103DB600F0A3ECF0901BC0E9F0A3EDF0A3EBF0A3A9
:103DC600EFF078C37C097D017B017A1B79AA7E001E
:103DD6007F201226D578AA7C1B7D017BFF7AE979A4
:103DE6009F7E007F201226D5901BCCE0FEA3E0F933
:103DF600901BB8F0EEFDA3F0901BCAE0FEA3E09086
:103E06001BBAF0EEFFFCA3F0901BCAA3E0FB901BCD
:103E1600BCF0A3ECF0901BC0E9F0A3EDF0A3EBF02F
:103E2600A3EFF078E37C097D017B017A1B79AA7EFA
:103E3600007F201226D59009FFE527F0FFAE26ADBC
:103E460025AC247808122A16A3EFF0AF27AE26ADCC
:103E560025AC247810122A16A3EFF0AF27AE26ADB4
:103E660025AC247818122A16A3EFF0E4F522F523E0
:103E760074A22523F582741B3522F583E0700F7436
:103E8600A22523F582741B3522F5837420F00523C1
:103E9600E523700205226408452270D4E4F522F574
:103EA6002374A22523F582741B3522F583E0FF7463
:103EB600E32523F58274093522F583EFF00523E522
:103EC60023700205226408452270D6E4F52EF52FEC
:103ED600FF7E08FDFC12891202CC8BC3E51C9408F8
:103EE6005054901B47E0FCA3E0FDA3E0FEA3E024B2
:103EF60001FFE43EFEE43DFDE43CFC901B47122A34
:103F06005C900981E0FBE4FAF9F8901B47E0FCA31A
:103F1600E0FDA3E0FEA3E0FF12294FAC00AD01AE29
:103F260002AF03E4FBFAF9F8C3122A0570AD127268
:103F36009C1282A480A512DA437D02AF16AE15123A
:103F46009C1112C50DE4FFFE74002FF58274003E2D
:103F5600F583E0FD74A22FF582741B3EF583EDF028
:103F66000FBF00010EEF64084E70DD9000B8E090C0
:103F760000CAF09000B9E09000CBF09000BAE09053
:103F860000CCF09000BBE09000CDF09000BCE0903B
:103F960000CEF09000BDE09000CFF09000BEE09023
:103FA60000D0F0900991E0FF9000D3F0900992E0E4
:103FB600FE9000D4F0900993E0FD9000D5F09009B2
:103FC60094E0F99000D6F0900995E09000D7F09033
:103FD6000996E09000D8F0900997E09000D9F0E4B7
:103FE600900031F0900025EFF0A3EEF0A3EDF0A3E2
:103FF600E9F0900995E0FF900029F0900996E0FE1F
:1040060090002AF0900997E0FD90002BF09009911E
:10401600E09000DCF0900992E09000DDF0900993CA
:10402600E09000DEF0A3E9F0A3EFF0A3EEF0A3ED3D
:10403600F07E087F007D007B017A0979A3122E5A53
:10404600E4FEFF74002FF58274003EF583E0FD74F4
:10405600A32FF58274093EF583EDF00FBF00010E24
:10406600E4B507DFEEB404DB7E097FA37DFE7C03A7
:1040760012D41C900DA1EFF07B017A0979A37DFF84
:104086007C0312D0EE900DA2EFF0E4FFFE12A3F631
:1040960012BB7FE4F52EF52F7F907E08FDFC12897A
:1040A6001212C3297B017A0979A3127453E4F52EFF
:1040B600F52F7F407E08FDFC128912752E08752F9C
:1040C600007F417E087D007C001289127E087F00F9
:1040D6007D007B017A0979A3122E5AE5112470FF1F
:1040E600E51034F7FEE50F34FFFDE50E34FFFCE482
:1040F600FB7A08F9F81228C48F268E258D248C2386
:10410600E5112401F511E43510F510E4350FF50F2E
:10411600E4350EF50E12C38CAD19AC18AF16AE15FC
:1041260012AF32AD19AC18AF16AE1512AFBD90096D
:1041360079E075F020A4FF90097BE07C002FFDEC70
:1041460035F0FC900978E02414FFEF7F0025E0FEAF
:10415600EF2DFFEC3E901BCAF0A3EFF090097DE037
:1041660075F020A4FFA3E0C3137C002FFDEC35F00F
:10417600FC90097CE07F0033333354F8FEEF2DFFCB
:10418600EC3E901BCCF0A3EFF078AA7C1B7D017B64
:10419600FF7AE9797F7E007F201226D5901BCCE03E
:1041A600FEA3E0F9901BB8F0EEFDA3F0901BCAA3A6
:1041B600E0901BBAF0901BCAE0FF901BBBF0901B6F
:1041C600CAA3E0FE901BBCF0A3EFF0901BC0E9F081
:1041D600A3EDF0A3EEF0901BCAE0901BC3F078A30A
:1041E6007C097D017B017A1B79AA7E007F2012263D
:1041F600D578AA7C1B7D017BFF7AE9795F7E007FFB
:10420600201226D5901BCCE0FEA3E0F9901BB8F057
:10421600EEFDA3F0901BCAA3E0901BBAF0901BCA58
:10422600E0FF901BBBF0901BCAA3E0FE901BBCF006
:10423600A3EFF0901BC0E9F0A3EDF0A3EEF0901B06
:10424600CAE0901BC3F078C37C097D017B017A1B11
:1042560079AA7E007F201226D578AA7C1B7D017B59
:10426600FF7AE9799F7E007F201226D5901BCCE04D
:10427600FEA3E0F9901BB8F0EEFDA3F0901BCAA3D5
:10428600E0901BBAF0901BCAE0FF901BBBF0901B9E
:10429600CAA3E0FE901BBCF0A3EFF0901BC0E9F0B0
:1042A600A3EDF0A3EEF0901BCAE0901BC3F078E3F9
:1042B6007C097D017B017A1B79AA7E007F2012266C
:1042C600D59009FFE526F0FFAE25AD24AC2378088E
:1042D600122A16A3EFF0AF26AE25AD24AC23781034
:1042E600122A16A3EFF0AF26AE25AD24AC2378181C
:1042F600122A16A3EFF0E4FEFF74A22FF582741BB8
:104306003EF583E0700D74A22FF582741B3EF58393
:104316007420F00FBF00010EEF64084E70DBE4FE60
:10432600FF74A22FF582741B3EF583E0FD74E32F24
:10433600F58274093EF583EDF00FBF00010EEF64C0
:10434600084E70DDE4F52EF52FFF7E08FDFC128980
:104356001212D46F9009687403F022E54A2436F8E5
:10436600E6054A2278333007027836E475F0011202
:104376002AA50226FB2000EB7F2ED2008018EF54E0
:104386000F2490D43440D4FF30040BEF24BFB41A6A
:104396000050032461FFE54B6002154B054EE54EC8
:1043A6007002054D30070D7833E475F001122AA529
:1043B600EF02277402D90D7403D2078003E4C20703
:1043C600F54A8B338A348935E4F54BF54DF54EE5E0
:1043D6004B60077F2012439C80F5754CFFC201C2DB
:1043E60000C202C203C205C206C20812436AFF70B7
:1043F6000D3007057F001243ADAF4EAE4D22B425FA
:104406005FC2D5C20412436AFF24D0B40A00501A10
:1044160075F00A784B30D50508B6FF0106C6A42606
:10442600F620D5047002D20380D924CFB41A00EF47
:104436005004C2E5D20402469AD20180C6D2008058
:10444600C0D20280BCD2D580BAD20580B47F2012F9
:10445600439C2002077401B54B0040F1124361FFF3
:1044660012439C0243D5D208D2068095124361FBC3
:10447600124361FA124361F94A4B700679917A4701
:104486007BFF20022EE54B602A7E008E827583001C
:1044960012271460060EEE654C70F0C2D5EBC0E034
:1044A600EAC0E0E9C0E0EE1246FAD0E0F9D0E0FA60
:1044B600D0E0FB1226FBFF60AAEBC0E0EAC0E0E911
:1044C600C0E012439CD0E02401F9D0E03400FAD0D9
:1044D600E0FBE54C0460DCD54CD98087D20280A293
:1044E6001246DD60F7E54C700104122463A94C60A6
:1044F6000DE54C600914F54C124784EF60F3EA3081
:10450600E702F404C3995077EAF4254C0430E70136
:10451600E404F54C800D1246DD60C1EA054C254CDD
:10452600122463EA7849F630E701E4254C04D54CB9
:1045360004200501141246FAE4C0E01247847849C3
:10454600E6601320E70714F6124384802204F6D0AF
:10455600E014C0E07F00124384E54C600712437B01
:10456600154C800B30050312437BD0E00243D5D0B7
:10457600E00480C51246DD60A0E54C041224637891
:1045860049EAF6E54C20050260010424041246FAC5
:1045960074FF04C0E0124784124384E54C200502F0
:1045A600600312437BD0E0B54CE87F4512438E781A
:1045B60049E67F2B30E7047F2DF404C0E012439CCC
:1045C600D0E075F00A84C0F0124385D0E01243852E
:1045D6000243D5791080027908C206C2088008D243
:1045E600D5790A8004790AC2D5E54C047002F54CE7
:1045F600E4FAFDFEFF124361FC7B0820011312431F
:1046060061FD7B1030000A124361FE124361FF7B9D
:1046160020EC3382D592D55013C3E43000069FFFB9
:10462600E49EFEE42001039DFDE49CFCE4CBF8C27D
:1046360001EC700CCFCECDCCE824F8F870F38017DF
:10464600C3EF33FFEE33FEED33FDEC33FCEB33FB10
:10465600994002FB0FD8E9EB300105F8D0E0C448D9
:10466600B201C0E00AEC4D4E4F78207B0070C2EAE2
:10467600B54C0040BCC0E01246FCD0F0D0E02001B2
:1046860004C4C0E0C4B201C0F0124385D0F0D5F036
:10469600EB0243D5122AB544725345D95844434CCC
:1046A600443F4245DD4F45E54445E54944584345C9
:1046B600EB55451C46457A4544E64747B1504447C5
:1046C6002D444B2E446E2B444F23446C20479A2A8C
:1046D60044074800004466E54CB4FF03754C0612D7
:1046E6004361FC124361FD124361FE124361FF7890
:1046F60042022492790AA2D5200314300509B91082
:10470600020404B9080104A2D520060250010420BF
:1047160002689202B54B005034C0E07F2030031986
:104726007F30A20272067205500F124753C202C2B0
:1047360006C205C2087F30800F300503E9C0E012CB
:10474600439C300503D0E0F9D0E0B54BCC300517DB
:104756007F30B9100C12439C7F583004077F788055
:1047660003B9080312439C3002057F2D02439C7F48
:10477600202008F87F2B2006F322920280CF7F00AC
:10478600B4070050052442F8E6FF22286E756C6CCB
:104796002900D2011243613001F8C201784B30D5AD
:1047A6000108F60244072D50434958124361240379
:1047B600B405004001E49047AC9312438D743A125D
:1047C600438DD203754B040245D9E4901BA2F0A396
:1047D600F0901BA2E0FEA3E024A3F58274093EF547
:1047E60083E06010901BA3E004F070E5901BA2E04C
:1047F60004F080DD901BA3E004F07006901BA2E09D
:1048060004F0901BA2E0FEA3E024A3F974093EFA8B
:104816007B01129D70901BA6EEF0A3EFF0EE6003F5
:10482600024C0BEF14B40D004003024C0B904841B0
:1048360075F003A4C58325F0C58373024868024852
:10484600A2024AAB024ABB024AD9024AF6024B7698
:10485600024BA0024BA4024BA9024BAD024C0B0229
:104866004BB312993790097EE0FF901BA4E4F0A3A6
:10487600EFF07FD07E0712D222AD19AC18AF16AE7C
:104886001512AFBD90097EE0FF901BA4E07003A354
:10489600E06F7F317003024AF0024BA612DA4390B2
:1048A600097CE0FFE4FCFDFE7B3CFAF9F81228C423
:1048B600A804A905AA06AB0790097DE0FFE4FCFD64
:1048C600FEEB2FFFEE3AFEED39FDEC38FC901BA80F
:1048D600122A5C901BA8E0FCA3E0FDA3E0FEA3E087
:1048E600FFE47B3CFAF9F81228C4901BA8122A5C54
:1048F600901BA8E0F8A3E0F9A3E0FAA3E0FB900977
:104906007EE0FFE4FCFDFEEB2FFFEE3AFEED39FD07
:10491600EC38FC901BA8122A5C901BA8E0FCA3E0D4
:10492600FDA3E0FEA3E02408FFE43EFEE43DFDE433
:104936003CFC901BA8122A5CE47B3CFAF9F8901B1D
:10494600A8E0FCA3E0FDA3E0FEA3E0FF12294FAC24
:1049560000AD01AE02AF03901BAC122A5C901BACFB
:10496600A3A3A3E090098EF0901BA8E0FCA3E0FDB2
:10497600A3E0FEA3E0FFA3E0F8A3E0F9A3E0FAA317
:10498600E0FBC3EF9BFFEE9AFEED99FDEC98FC90E1
:104996001BA8122A5C901BA8E0FCA3E0FDA3E0FE86
:1049A600A3E0FFE47B3CFAF9F812294F901BA8120A
:1049B6002A5CE47B3CFAF9F8901BA8E0FCA3E0FD36
:1049C600A3E0FEA3E0FF12294FAC00AD01AE02AF9B
:1049D60003901BAC122A5C901BACA3A3A3E0900926
:1049E6008DF0901BA8E0FCA3E0FDA3E0FEA3E0FF92
:1049F600A3E0F8A3E0F9A3E0FAA3E0FBC3EF9BFF73
:104A0600EE9AFEED99FDEC98FC901BA8122A5C909C
:104A16001BA8E0FCA3E0FDA3E0FEA3E0FFE47B3CD3
:104A2600FAF9F812294F901BA8122A5C901BA8A32A
:104A3600A3A3E0FF90098CF0A3E0FDA3E0FB12D056
:104A46007F900978E0FFA3E0FD90097BE0FB9009E9
:104A56007AE0F52512CD1F12D6C012D7E012DA245D
:104A660012D842E47FF87E2AFDFCAB0DAA0CA90BF6
:104A7600A80AC3122A057F0050027F01E5147E00B2
:104A860070027E01EF5E70DB12D9AF12DA2812D700
:104A960034E51464017F32700512D36E800312D39D
:104AA6009AE4F5142212B83DEC4D4E4F7F33700355
:104AB600024BA6803512BBF1EF701312BC63EF7088
:104AC6000D12CB0CEF7F347003024BA6801C7F3493
:104AD600024B7112BBF1EF701312BC63EF700D1233
:104AE600CB0CEF7F357003024BA6807F7F35807B32
:104AF600E4901BA2F0A3F0901BAC122A6800000001
:104B060000E4FFFE7D0FFC901BACE0F8A3E0F9A3E8
:104B1600E0FAA3E0FBC3122A05503F901BACE0FC71
:104B2600A3E0FDA3E0FEA3E0FF129880901BA3E0A4
:104B36002FF0901BA2E03EF0901BACE0FCA3E0FD42
:104B4600A3E0FEA3E02400FFEE3401FEE43DFDE415
:104B56003CFC901BAC122A5C80A7C3901BA3E0947C
:104B66005A901BA2E094007F36400302D39A80300D
:104B7600E4901BA6F0A3F0FF12D761E4752F8075B1
:104B86002E25F52DF52CFF7E367D6E7C0112D00B81
:104B96007F3712D36E7F0102D7617F3880027F395B
:104BA60002D36E7D3080027D317F318052E4901BCE
:104BB600A2F0A3F0FF12D76112729CD3901B3EE0C5
:104BC6009488901B3DE094134008901BA2E4F0A348
:104BD60004F07F0112D76112729CC3901B3EE094D1
:104BE60088901B3DE094135008901BA2E4F0A304A8
:104BF600F0901BA2E07002A3E07D337F31700302C8
:104C0600D25412D2842212C568EF7003024CA91244
:104C1600DA4312C50DEF60097D09AF16AE15129C79
:104C260011900991E09000CAF0900992E09000CBB3
:104C3600F0900993E09000CCF0900994E09000CDBC
:104C4600F0900995E09000CEF0900996E09000CFA4
:104C5600F0900997E09000D0F07E087F007D007B01
:104C6600017A0979A3122E5A78A37C097D017B016A
:104C76007A0079007E047F001226D57E097FA37D07
:104C8600FE7C0312D41C900DA1EFF07B017A09790A
:104C9600A37DFF7C0312D0EE900DA2EFF0E4FFFEA1
:104CA60012A35512C50DEF60097D09AF16AE151298
:104CB6009C117B017A0079137D0412C4AFE47B7DDD
:104CC600FAF9F812294F900981EFF0700F7D24AFA1
:104CD60016AE15129C119009817402F07B017A00C0
:104CE60079177D0212C4AF900985EEF0A3EFF0901C
:104CF60003BDE0900987F0D3940374809480400F3D
:104D06007D24AF16AE15129C119009877403F0E44A
:104D1600F524F525900987E0FFC3E5259FE5249452
:104D2600004003024F3DE525C4F8540FC868FFE56F
:104D360024C454F048FE74BE2FF974033EFA7B0176
:104D46007D0412C4AF901B5A75F013E525122A99FB
:104D5600E52475F013A42583F583122A5CE525C4A2
:104D6600F8540FC868FFE524C454F048FE74C22FF7
:104D7600F974033EFA7B017D0412C4AF901B5E7585
:104D8600F013E525122A99E52475F013A42583F579
:104D960083122A5CE525C4F8540FC868FFE524C4CD
:104DA60054F048FE74C62FF974033EFA7B017D0267
:104DB60012C4AF901B6275F013E525122A99E524FB
:104DC60075F013A42583F583EEF0A3EFF0E525C473
:104DD600F8540FC868FFE524C454F048FE74C82F81
:104DE600F58274033EF583E0FD901B6475F013E5D0
:104DF60025122A99E52475F013A42583F583EDF091
:104E060074C92FF974033EFA7B017D0212C4AFE523
:104E1600252FFFE5243EFE901B6775F013E525124E
:104E26002A99E52475F013A42583F583EEF0A3EF04
:104E3600F0901B6B75F013E525122A99E52475F0A1
:104E460013A42583F5837401F0901B6975F013E5AF
:104E560025122A99E52475F013A42583F583E4F039
:104E6600A3F0901B5A75F013E525122A99E52475CF
:104E7600F013A42583F583E0FCA3E0FDA3E0FEA3E5
:104E8600E0FF122ADB4EA1000000B04ED200000067
:104E9600C04F14000016A100004F329000A8E0FF9A
:104EA6007E00700790098274BC800BEF64014E701F
:104EB6000A90098274BDF0A3F08071EF64024E700F
:104EC6006B90098274BCF0A304F080609000A8E0A7
:104ED600FD75F00A84FE25E025E0540C900982F069
:104EE600ED75F00A84AFF0EF25E025E0540CA3F051
:104EF6009000B1E0FF901B6C75F013E525122A991E
:104F0600E52475F013A42583F583EFF0801E900049
:104F1600A8E0FD75F00A84FEC45470900982F0ED95
:104F260075F00A84AFF0EFC45470A3F00525E525AB
:104F360070020524024D1AE4F51CF51D901B47125C
:104F46002A68000000007508097509A3E490097530
:104F5600F0A3F0900974F0F524F525900987E0FF99
:104F6600C3E5259FE52494004003025004901B5A94
:104F760075F013E525122A99E52475F013A4258307
:104F8600F583E0FCA3E0FDA3E0FEA3E0FFE47BC025
:104F9600FAF9F8C3122A05705A901B5E75F013E5EC
:104FA60025122A99E52475F013A42583F583E0FCE0
:104FB600A3E0FDA3E0FEA3E0FF752F00752E367576
:104FC6002D6E752C0112D00B12DA2C901B6C75F01D
:104FD60013E525122A99E52475F013A42583F58394
:104FE600E0FF12D88C12DA307F407E0D7D037C0004
:104FF60012D64C0525E52570020524024F61229044
:105006001BA5745FF074092409F582E434DFF58387
:10501600E493F9901BA6F07409240AF582E434DFC0
:10502600F583E493FF901BA7F0A3742EF090DF099D
:10503600E493FE644F6009EE644E6004EEB44404EB
:105046007E3180027E30901BA9EEF090DF09E4935A
:10505600B44A17A3E493B4611115827583DFA3A341
:10506600E493B46E057E3102514590DF09E493FE68
:10507600B446057E32025145EEB44D1A90DF09A3BF
:10508600E493B4611115827583DFA3A3E493B4722C
:10509600057E3302514590DF09E493B4410BA3E446
:1050A60093B470057E3402514590DF09E493FEB453
:1050B6004D16A3E493B4611015827583DFA3A3E4B0
:1050C60093B479047E358077EEB44A1990DF09A34C
:1050D600E493B4751015827583DFA3A3E493B46ECD
:1050E600047E36805A90DF09E493B44A16A3E4930B
:1050F600B4751015827583DFA3A3E493B46C047EA4
:1051060037803C90DF09E493FEB4410AA3E493B4EC
:1051160075047E388029EEB453047E39802190DFF1
:1051260009E493FEB44F047E308014EEB44E047E40
:1051360031800C90DF09E4937E3FB444027E3290C6
:105146001BAAEEF074092404F582E434DFF583E447
:1051560093FEFD3395E0FCC3ED9430EC64809480BF
:10516600400280027E30901BABEEF0E4A3F0C3ED6C
:105176009430EC64809480401074092404F582E431
:1051860034DFF583E493FE80027E30901BADEEF0B3
:1051960074092405F582E434DFF583E493901BAEAD
:1051A600F0A3742EF090DF09E493FE644F6009EEDD
:1051B600644E6004EEB444047E3180027E30901B5F
:1051C600B0EEF090DF09E493B44A17A3E493B46118
:1051D6001115827583DFA3A3E493B46E057E3102B5
:1051E60052BD90DF09E493FEB446057E320252BDFD
:1051F600EEB44D1A90DF09A3E493B46111158275DC
:1052060083DFA3A3E493B472057E330252BD90DF1D
:1052160009E493B4410BA3E493B470057E340252BF
:10522600BD90DF09E493FEB44D16A3E493B4611078
:1052360015827583DFA3A3E493B479047E35807762
:10524600EEB44A1990DF09A3E493B475101582757C
:1052560083DFA3A3E493B46E047E36805A90DF09FD
:10526600E493B44A16A3E493B4751015827583DFEC
:10527600A3A3E493B46C047E37803C90DF09E493E7
:10528600FEB4410AA3E493B475047E388029EEB4D3
:1052960053047E39802190DF09E493FEB44F047EE7
:1052A600308014EEB44E047E31800C90DF09E49316
:1052B6007E3FB444027E32901BB1EEF0A3742EF012
:1052C600A3E9F0A3EFF0E4A3F078A37C097D017BCA
:1052D600FF7AE27963FE7F081226D578AB7C097DDA
:1052E600017B017A1B79AD7E007F091226D578B441
:1052F6007C097D017BFF7AE2795B7E007F081226BE
:10530600D5E4901BA4F07E097FA37D19FC12D41C62
:10531600901BA4EFF012D921E4901BA2F0A3F09009
:105326001BA2E0FEA3E0FFC39419EE9400501F7485
:10533600A32FF58274093EF583E0FF12D8FE901B79
:10534600A3E004F070D9901BA2E004F080D1901B7A
:10535600A4E0FF02D8FEE4F522F523900987E0FFDA
:10536600C3E5239FE52294004003025652901B6733
:1053760075F013E523122A99E52275F013A4258307
:10538600F583E0FEA3E0FF74B3251DF582740935AD
:105396001CF583E5822FF582E5833EAF82F5268FE5
:1053A60027901B5E75F013E523122A99E52275F006
:1053B60013A42583F583E0FCA3E0FDA3E0FEA3E0B0
:1053C600F52F8E2E8D2D8C2C7F007E367D6E7C01EA
:1053D60012D00B901B6475F013E523122A99E5226F
:1053E60075F013A42583F583E0FFD39401748094AC
:1053F60080500302562FEFFD7C00901B6975F01359
:10540600E523122A99E52275F013A42583F583E096
:10541600FEA3E0FF1227A88D24E5247033901B6BB2
:1054260075F013E523122A99E52275F013A4258356
:10543600F583E07F0070027F01901B6B75F013E52A
:1054460023122A99E52275F013A42583F583EFF03C
:10545600901B6975F013E523122A99E52275F0135E
:10546600A42583F583E475F001122833901B5A7541
:10547600F013E523122A99E52275F013A42583F586
:1054860083E0FCA3E0FDA3E0FEA3E0FFE47BB0FA2B
:10549600F9F8C3122A05602E901B5E75F013E523FA
:1054A600122A99E52275F013A42583F583E0FCA35F
:1054B600E0FDA3E0FEA3E0FF7B407A42790F78008F
:1054C600C3122A05704612DA2C901B6B75F013E591
:1054D60023122A99E52275F013A42583F583E02487
:1054E60082F582E43409F583E0FF12D88C12DA30B3
:1054F600E4FFFE0FBF00010EBE1FF8BF40F5E52416
:10550600540F04F5254325B0E40255B9901B5A758E
:10551600F013E523122A99E52275F013A42583F5E5
:1055260083E0FCA3E0FDA3E0FEA3E0FFE47BC0FA7A
:10553600F9F8C3122A05702A901B6B75F013E52340
:10554600122A99E52275F013A42583F583E02482B7
:10555600F582E43409F583E0452404F5254325C0A6
:105566008051901B5A75F013E523122A99E522758E
:10557600F013A42583F583E0FCA3E0FDA3E0FEA3DE
:10558600E0FFE47BA17A16F9F8C3122A057024908D
:105596001B6B75F013E523122A99E52275F013A407
:1055A6002583F583E02482F582E43409F583E0451A
:1055B60024F525901B5A75F013E523122A99E52246
:1055C60075F013A42583F583E0FCA3E0FDA3E0FEBC
:1055D600A3E0540FFFE4FBFAF9F8C3122A05701290
:1055E600E5272401FFE43526FE85232EAB25E4FDC1
:1055F6008010E5272401FFE43526FE85232EAB2502
:105606007D0112565878A27C1B7D017E007F031215
:1056160026D5852782852683A3E525F0901BA2E063
:10562600852782852683F08018AD23AC22AF27AE6E
:105636002612D18B78A27C1B7D017E007F03122669
:10564600D50523E52370020522025361901BA2E0D3
:10565600FF228E2A8F2B8D2C8B2D78B07C1B7D0103
:105666007BFF7AEA79027E007F031226D5E4F52FC6
:10567600E52E75F013A4245EF582E4341BF583E071
:10568600FCA3E0FDA3E0FEA3E0FF122ADB569D008B
:1056960000258000005718E52E75F013A4245EF54A
:1056A60082E4341BF583E0F8A3E0F9A3E0FAA3E073
:1056B600FB7F807E967D987C0012294FE47BFAFA68
:1056C600F9F812294FE47B02FAF9F8D3122A0540B9
:1056D60008E47F02FEFDFC802EE52E75F013A4245F
:1056E6005EF582E4341BF583E0F8A3E0F9A3E0FA63
:1056F600A3E0FB7F807E967D987C0012294FE47B99
:10570600FAFAF9F812294FEF240AF531E43EF5309A
:105716008074E52E75F013A4245EF582E4341BF53F
:1057260083E0F8A3E0F9A3E0FAA3E0FB7F807E968E
:105736007D987C0012294FE47BFAFAF9F812294F7A
:10574600E47B02FAF9F8D3122A054008E47F02FE48
:10575600FDFC802EE52E75F013A4245EF582E4345C
:105766001BF583E0F8A3E0F9A3E0FAA3E0FB7F8052
:105776007E967D987C0012294FE47BFAFAF9F8129E
:10578600294F8E308F3112DA2CE52E75F013A424B2
:105796005AF582E4341BF583E0FCA3E0FDA3E0FEAA
:1057A600A3E4FFE4FBFAF9F8C3122A05704AE52ED2
:1057B60075F013A4245AF582E4341BF583A3A3A33E
:1057C600E0FBEB452DFFE4901BB3EFF0E52E75F003
:1057D60013A4245EF582E4341BF583E0FCA3E0FD0C
:1057E600A3E0FEA3E0FF7B407A42790F7800C31264
:1057F6002A05901BB3025893E52E75F013A4245A7C
:10580600F582E4341BF583A3A3E0FEA3E4FFE4FDE5
:10581600FC7808122A16901BB3EFF0E52E75F013EC
:10582600A4245AF582E4341BF583A3A3A3E0FFE482
:10583600901BB4EFF0E52C6031A3E52DF07E1B7FC5
:10584600B37D037C0012D41C901BB6EFF0901BB303
:10585600E0FF12D88C901BB4E0FF12D88C901BB5D9
:10586600E0FF12D88C901BB680237E1B7FB37D028F
:105876007C0012D41C901BB5EFF0901BB3E0FF1216
:10588600D88C901BB4E0FF12D88C901BB5E0FF12A9
:10589600D88C12DA30AB2BAA2AAD31AC307F647EBD
:1058A6000012C677901BB1EEF0A3EFF04E70079092
:1058B6001BB07403806DE52E75F013A4245AF5828F
:1058C600E4341BF583E0FCA3E0FDA3E0FEA3E4FFC4
:1058D600E4FBFAF9F8C3122A05702CF52FFFFED364
:1058E600901BB2E09F901BB1E09E4016E52B2FF572
:1058F60082E52A3EF583E0252FF52F0FBF00010E26
:1059060080DD532F7F8011901BB1E0FCA3E0FDAF3B
:105916002BAE2A12D41C8F2FE52F7F017001FF902A
:105926001BB0EFF07B017A1B79B022E4901BA2F04A
:10593600A3F0901BA2E475F001122849FE74A3257A
:10594600F0F58274093EF583E070E7901BA2E0FE55
:10595600A3E024A3F974093EFA7B0112915A901B25
:10596600A4122A5CE4FFFEFDFC901BA4E0F8A3E071
:10597600F9A3E0FAA3E0FBC3122A05704A12CC3F52
:105986007E097FA37D007C0412D41C8F2212D921AC
:10599600E4901BA2F0A3F0901BA2E0FEA3E0FFC3DD
:1059A600EE9404501F74A32FF58274093EF583E02C
:1059B600FF12D8FE901BA3E004F070DB901BA2E060
:1059C60004F080D3025BF0E47B02FAF9F8901BA4A2
:1059D600E0FCA3E0FDA3E0FEA3E0FF12294FEF24C5
:1059E600FFFFEE34FFFEED34FFFDEC34FFFC901BB1
:1059F600A8122A5C90096CE064017038FF7E08FDED
:105A0600FC901BA8E0F8A3E0F9A3E0FAA3E0FBD31F
:105A1600122A05401F901BA8E0FCA3E0FDA3E0FEB0
:105A2600A3E02470FFE43EFEE43DFDE43CFC901B55
:105A3600A8122A5C901BA8E0FCA3E0FDA3E0FEA34D
:105A4600E0FF12B64BEF6003025BF5901BA8E0FC8B
:105A5600A3E0FDA3E0FEA3E0FF122ADB5A780000D4
:105A660000005ABE000008005AF500000890000029
:105A76005AFBE4901BA2F0A3F0901BA2E0FEA3E069
:105A8600FF2400F58274003EF583E0FD74A32FF534
:105A96008274093EF583EDF0901BA3E004F07006D6
:105AA600901BA2E004F0901BA2E0B404CCA3E0B4E7
:105AB60000C712D340025BACE4901BA2F0A3F090A7
:105AC6001BA2E0FEA3E0FFC3EE9404501C74A32FB8
:105AD600F58274093EF583E4F0901BA3E004F070B0
:105AE600DE901BA2E004F080D612A211025BAC127B
:105AF600D2B4025BAC901BA4A3A3A3E05401FFE4C1
:105B0600FEFDFCFBFAF9F8C3122A057041901BA2B0
:105B1600F0A3F0901BA2E0FEA3E0FF2400F5827440
:105B2600003EF583E0FD74A32FF58274093EF583EC
:105B3600EDF0901BA3E004F07006901BA2E004F0C9
:105B4600901BA2E0B404CCA3E0B400C78058901B1D
:105B5600A4A3A3A3E05401FFE4FEFDFCFBFAF9F8BD
:105B6600C3122A056040E4901BA2F0A3F0901BA28A
:105B7600E0FEA3E0FF2400F58274043EF583E0FD19
:105B860074A32FF58274093EF583EDF0901BA3E014
:105B960004F07006901BA2E004F0901BA2E0B4048F
:105BA600CCA3E0B400C77E097FA37D007C0412D499
:105BB6001C8F2212D921E4901BA2F0A3F0901BA205
:105BC600E0FEA3E0FFC3EE9404501F74A32FF582FA
:105BD60074093EF583E0FF12D8FE901BA3E004F0A3
:105BE60070DB901BA2E004F080D3AF2212D8FE2215
:105BF600901CDEE0FF90097EE0FE6F7003025CCB36
:105C0600901CDEEEF0901CC4E0FCA3E0FDA3E0FED9
:105C1600A3E02401FFE43EFEE43DFDE43CFC901CD1
:105C2600C4122A5C901CC8E0FCA3E0FDA3E0FEA31E
:105C3600E02401FFE43EFEE43DFDE43CFC901CC88C
:105C4600122A5C901CCCE0FCA3E0FDA3E0FEA3E0DE
:105C56002401FFE43EFEE43DFDE43CFC901CCC1236
:105C66002A5C901CD0E0FCA3E0FDA3E0FEA3E024A8
:105C760001FFE43EFEE43DFDE43CFC901CD0122A0C
:105C86005C901CD4E0FCA3E0FDA3E0FEA3E02401AD
:105C9600FFE43EFEE43DFDE43CFC901CD4122A5C8D
:105CA600901CD8E0FCA3E0FDA3E0FEA3E02401FFE6
:105CB600E43EFEE43DFDE43CFC901CD8122A5C90D8
:105CC6001CDDE004F0D3901B38E094E8901B37E02D
:105CD6009403403AE47F107E0EFDFC901CC8E0F869
:105CE600A3E0F9A3E0FAA3E0FBD3122A05401F9034
:105CF6001CC8122A68000000007527FF7528E97580
:105D060029BF901B37E0FAA3E0FB7D05804EC390C8
:105D16001B3EE09488901B3DE094135051E47F10A5
:105D26007E0EFDFC901CD4E0F8A3E0F9A3E0FAA3F4
:105D3600E0FB122A054037901CD4122A68000000A6
:105D460000901B3FE0FAA3E0FBC39488EA9413504B
:105D5600147527FF7528E97529C37D0EAF16AE1594
:105D660012794C80097D0FAF16AE15129C11C390A7
:105D76001B38E0941E901B37E09400503EE47F10E1
:105D86007E0EFDFC901CCCE0F8A3E0F9A3E0FAA39C
:105D9600E0FB122A054024901CCC122A6800000061
:105DA600007527FF7528E97529BF901B37E0FAA310
:105DB600E0FB7D06AF16AE1512794C901B55E064DC
:105DC60003702D7F107E0EFDFC901CC4E0F8A3E04E
:105DD600F9A3E0FAA3E0FBD3122A054013901CC4F2
:105DE600122A68000000007D04AF16AE15129C1141
:105DF600901B55E06401702D7F107E0EFDFC901CFB
:105E0600D0E0F8A3E0F9A3E0FAA3E0FBD3122A0559
:105E16004013901CD0122A68000000007D07AF16C0
:105E2600AE15129C11C3901B3AE094E0901B39E02A
:105E3600942E503EE47F087E07FDFC901CD8E0F8C7
:105E4600A3E0F9A3E0FAA3E0FB122A054024901C84
:105E5600D8122A68000000007527FF7528E9752901
:105E6600C3901B39E0FAA3E0FB7D10AF16AE151206
:105E7600794CC3901B40E09488901B3FE0941350EC
:105E860026901CDCE0700804F0E4A3F0FF80159077
:105E96001CDDE0D3940274809480400BE4F0901CE7
:105EA600DCF07F0112D76122E56365627003026050
:105EB600F3AF62056274002FF582E43400F583E0E7
:105EC600F522E55E6003026075E52224F66064242F
:105ED600FD7003025FE324ED604024F5601D24F1AC
:105EE6007003025FF324FD606924CA6058246B6066
:105EF6000302605BE4F558F55980AD0559E559AEE6
:105F060058700205581424A3F58274093EF583E4FB
:105F1600F0F55CF55D755E01808E0559E559AE5864
:105F2600700205581424A3F58274093EF583E4F043
:105F3600025EAE74A32559F58274093558F583E4DB
:105F4600F0F55EFF220559E559AE58700205580274
:105F560060650559E559AE58700205581424A3F535
:105F66008274093EF583E4F0755E01755F01F55AAA
:105F7600F55BF55CF55D74A3255BF5827409355A0E
:105F8600F583E0600A055BE55B70EB055A80E70583
:105F96005BE55B7002055A74A3255BF582740935CF
:105FA6005AF583E0600A055BE55B70EB055A80E70E
:105FB600055BE55B7002055A74A3255BF5827409DF
:105FC600355AF583E0600A055BE55B70EB055A80A0
:105FD600E7055BE55B7002055A24A3806674A3257A
:105FE60059F58274093558F583E4F0FF220559E521
:105FF60059AE58700205581424A3F58274093EF56B
:1060060083E4F0755E01755F01F55AF55BF55CF5A5
:106016005D055BE55BAE5A7002055A1424A3F58252
:1060260074093EF583E070E9055BE55BAE5A7002E4
:10603600055A1424A3F58274093EF583E070E974C9
:10604600A3255BF97409355AFA7B01129D708E609F
:106056008F61025EAE0559E559AE587002055814B7
:1060660024A3F58274093EF583E522F0025EAEE5CF
:106076005F6034055DE55D7002055C0559E559AE66
:1060860058700205581424A3F58274093EF583E579
:1060960022F0C3E55D9561E55C95605003025EAE56
:1060A600E4F55EF55F8030055DE55D7002055C0533
:1060B60059E559AE58700205581424A3F58274099F
:1060C6003EF583E522F0C3E55D9401E55C9404505A
:1060D60003025EAEE4F55E74A32559F582740935B4
:1060E60058F583E522F0E4F558F559FF227F0122A1
:1060F6008E2F8F308D318A328B3312B0C78F3A8E06
:10610600398D388C377F007E407D017C00AB3AAA02
:1061160039A938A837C3122A05400302632A7E002C
:106126007F407D007B017A1C7922122E5A7E007FE9
:106136000C7D007B017A1C7916122E5A85308285D9
:106146002F83A3A3A3E0C3940A74809480500D7E8A
:106156001C7F227BFF7ADE79DA12A8FC85308285E5
:106166002F83A3A3A3E0FF7E007B017A1C7916127E
:106176007D9A12A8F212CABE853082852F83A3E0CB
:10618600C3940A74809480500D7E1C7F227BFF7A14
:10619600DE79DA12A8FC853082852F83A3E0FF7EA4
:1061A600007B017A1C7916127D9A12A8F212CABED9
:1061B600853082852F83E0FF7E007B017A1C79166D
:1061C600127D9A12A8F27E1C7F227B2012CAC4E599
:1061D600302404F582E4352FF583E0C3940A7480F5
:1061E6009480500D7E1C7F227BFF7ADE79DA12A81E
:1061F600FCE5302404F582E4352FF583E0FF7E00CC
:106206007B017A1C7916127D9A12A8F27E1C7F22D7
:106216007B3A12CAC4E5302405F582E4352FF583AE
:10622600E0C3940A74809480500D7E1C7F227BFF0D
:106236007ADE79DA12A8FCE5302405F582E4352FFA
:10624600F583E0FF7E007B017A1C7916127D9A1297
:10625600A8F27E1C7F227B3A12CAC4E5302406F5DA
:1062660082E4352FF583E0C3940A74809480500D40
:106276007E1C7F227BFF7ADE79DA12A8FCE53024C9
:1062860006F582E4352FF583E0FF7E007B017A1C5C
:106296007916127D9A12A8F2AF31126D127E007F26
:1062A6000C7D007B017A1C7916122E5AAE32AF3362
:1062B600E4FCFD7B017A1C791612693C12A8F27E79
:1062C6001C7F227B2012CAC4E53645354534600D55
:1062D6007E1C7F22AB34AA35A93612A8FC7B017A34
:1062E6001C792212D7A3C3EF943EEE940050147487
:1062F600222FF582741C3EF5837420F00FBF000137
:106306000E80E3901C60740DF0A3740AF0AF3AAEF1
:1063160039AD38AC377B017A1C792275420075435A
:106326004012BFE122E4901BA2F0A3F0901BA2E072
:10633600FEA3E024A3F58274093EF583E060109085
:106346001BA3E004F070E5901BA2E004F080DD9052
:106356001BA2E475F001122849FE74A325F0F5820C
:1063660074093EF583742BF0901BA2E0FEA3E02493
:10637600A3F58274093EAF82FE7D017C0412D41C13
:10638600901BA4EFF0901BA2E0FEA3E024A3F582ED
:1063960074093EF583E0900987F0E4901BA5F09020
:1063A6000987E0FF901BA5E0FEC39F400302652F0F
:1063B600EE75F010A424A4F9740935F0FA7B019067
:1063C6001BA2E0FEA3E029F9EA3EFA7D0412C4AF5F
:1063D600901BA5E0FB75F013A4245AF582E4341B48
:1063E600F583122A5CEB75F010A424A8F97409351C
:1063F600F0FA7B01901BA2E0FEA3E029F9EA3EFA3F
:106406007D0412C4AF901BA5E0FB75F013A4245EB7
:10641600F582E4341BF583122A5CEB75F010A42494
:10642600ACF9740935F0FA7B01901BA2E0FEA3E0FB
:1064360029F9EA3EFA7D0212C4AF901BA5E0FD756C
:10644600F013A42462F582E4341BF583EEF0A3EF87
:10645600F0901BA2E0FEA3E0FF75F010EDA42FF56F
:1064660082E5F03EF583E58224AEF582E5833409C4
:10647600F583E0FFED75F013A42464F582E4341B84
:10648600F583EFF0ED75F010A424AFF9740935F03B
:10649600FA7B01901BA2E0FEA3E029F9EA3EFA7D11
:1064A6000212C4AF901BA5E0FD7A002FFFEA3EFE64
:1064B600ED75F013A42467F582E4341BF583EEF042
:1064C600A3EFF0901BA5E0FF75F013A4246BF582F3
:1064D600E4341BF5837401F0901BA2E0FCA3E0906A
:1064E6001B6975F013122A99EC75F013A42583F530
:1064F60083E4F0A3F0EF75F013A42462F582E4348C
:106506001BF583E0FEA3E04E7016901BA5E075F028
:1065160013A42462F582E4341BF583E4F0A304F0AB
:10652600901BA5E004F00263A5E4900982F0A3F0B5
:10653600900985740FF0A374FFF002D868E4901BED
:10654600A2F0A3F0901BA2E475F001122849FE7494
:10655600A325F0F58274093EF583E070E7901BA24F
:10656600E475F001122849FE74A325F0F58274093A
:106576003EF583E070E7901BA275F001122849FEF4
:1065860074A325F0F58274093EF583E075F00AA43C
:10659600FF901BA2E475F001122849FC74A325F0B4
:1065A600F58274093CF583E02F24F0900988F09079
:1065B6001BA2E475F001122849FE74A325F0F582AA
:1065C60074093EF583E075F00AA4FF901BA2E475FA
:1065D600F001122849FC74A325F0F58274093CF5F4
:1065E60083E02F24F0900989F0901BA2E475F00156
:1065F600122849FE74A325F0F58274093EF583E05E
:1066060075F00AA4FF901BA2E475F001122849FC5C
:1066160074A325F0F58274093CF583E02F24F090ED
:10662600098AF0901BA2E475F001122849FE74A3B2
:1066360025F0F58274093EF583E075F00AA4FF9013
:106646001BA2E475F001122849FC74A325F0F5821B
:1066560074093CF583E02F24F090098BF0901BA27F
:10666600E475F001122849FE74A325F0F582740939
:106676003EF583E075F00AA4FF901BA2E475F001D5
:10668600122849FC74A325F0F58274093CF583E0D1
:106696002F24F090098CF0901BA2E475F0011228CB
:1066A60049FE74A325F0F58274093EF583E075F082
:1066B6000AA4FF901BA2E475F001122849FC74A3FA
:1066C60025F0F58274093CF583E02F24F090098DBE
:1066D600F0901BA2E475F001122849FE74A325F080
:1066E600F58274093EF583E075F00AA4FF901BA2BB
:1066F600E475F001122849FC74A325F0F5827409AB
:106706003CF583E02F24F090098EF090098CE0FF91
:10671600A3E0FDA3E0FB12D07F900988E0FFA3E091
:10672600FD90098BE0FB90098AE0F52512CD1F123A
:10673600D6C012D8EFEF6401700302D86812D87A77
:1067460022E4901BA2F0A3F0901BA2E475F00112C4
:106756002849FE74A325F0F58274093EF583E0709E
:10676600E7901BA2E475F001122849FE74A325F0F8
:10677600F58274093EF583E070E7901BA275F0017F
:10678600122849FE74A325F0F58274093EF583E0CC
:1067960075F00AA4FF901BA2E475F001122849FCCB
:1067A60074A325F0F58274093CF583E02F24F0905C
:1067B6000978F0901BA2E475F001122849FE74A333
:1067C60025F0F58274093EF583E075F00AA4FF9082
:1067D6001BA2E475F001122849FC74A325F0F5828A
:1067E60074093CF583E02F24F0900979F0901BA200
:1067F600E475F001122849FE74A325F0F5827409A8
:106806003EF583E075F00AA4FF901BA2E475F00143
:10681600122849FC74A325F0F58274093CF583E03F
:106826002F24F090097AF0901BA2E475F00112284B
:1068360049FE74A325F0F58274093EF583E075F0F0
:106846000AA4FF901BA2E475F001122849FC74A368
:1068560025F0F58274093CF583E02F24F090097B3E
:10686600F0901BA2E475F001122849FE74A325F0EE
:10687600F58274093EF583E075F00AA4FF901BA229
:10688600E475F001122849FC74A325F0F582740919
:106896003CF583E02F24F090097CF0901BA2E47570
:1068A600F001122849FE74A325F0F58274093EF51D
:1068B60083E075F00AA4FF901BA2E475F00112288C
:1068C60049FC74A325F0F58274093CF583E02F2476
:1068D600F090097DF0901BA2E475F001122849FEA4
:1068E60074A325F0F58274093EF583E075F00AA4D9
:1068F600FF901BA2E475F001122849FC74A325F051
:10690600F58274093CF583E02F24F090097EF0901F
:10691600097CE0FFA3E0FDA3E0FB12D1BE9009785D
:10692600E0FFA3E0FD90097BE0FB90097AE0F52506
:1069360012CECC02D8688F3E8E3D8D3C8C3B8B3F71
:106946008A408941901BD9740AF0E4A3F0EC3350D5
:10695600257401F0253EFFE4353DFEE4353CFDE4BB
:10696600353BFC1229E1EF2401FFE43EFEE43DFD48
:10697600E43CFCA3800BAF3EAE3DAD3CAC3B901B74
:10698600DB122A5CE4901BD7F0901BD9E0FF901B2A
:10699600D7E0C39F5065E47B0AFAF9F8901BDBE069
:1069A600FCA3E0FDA3E0FEA3E0FF12294FEB243099
:1069B600FF901BD9E024FFFDE434FFFC901BD7E0D9
:1069C600FBC3ED9BFDEC9400AB3FAA40A9418D8231
:1069D600F583EF122786901BDBE0FCA3E0FDA3E026
:1069E600FEA3E0FFE47B0AFAF9F812294F901BDBBD
:1069F600122A5C901BD7E004F0808EE4901BD7F03F
:106A0600901BD9E014FF901BD7E0FEC39F5019AB33
:106A16003FAA40A9418E82758300122714B430081C
:106A2600901BD7E004F080D8901BDAE0607EE490FB
:106A36001BD8F0901BD7E0FF901BD9E0C39FFE90B8
:106A46001BD8E0FDC39E5028ED2FF582E433F58375
:106A5600AB3FAA40A941122714FF901BD8E0F5824C
:106A6600758300A3EF122786901BD8E004F080C33D
:106A7600AB3FAA40A941742D122774901BD7E0FFA3
:106A8600901BD9E0C39FFFE49400CF2401CF3400CC
:106A9600AB3FAA40A9418F82F583E4122786901B5B
:106AA600D7E0FF901BD9E0C39F04FF22901BD7E0DD
:106AB600D3940074809480404AE4A3F0901BD7E0FE
:106AC600FF901BD9E0C39FFE901BD8E0FDC39E50EC
:106AD60027ED2FF582E433F583AB3FAA40A9411297
:106AE6002714FF901BD8E0F582758300EF122786E6
:106AF600901BD8E004F080C4AB3FAA40A941901B8C
:106B0600D88009AB3FAA40A941901BD9E0F5827510
:106B16008300E4122786901BD7E0FF901BD9E0C3C1
:106B26009FFF228E2F8F308D3112B0C78F358E3456
:106B36008D338C327F007E407D017C00AB35AA34DC
:106B4600A933A832C3122A054003026D117E007FC5
:106B5600407D007B017A1C7922122E5A7E007F0C22
:106B66007D007B017A1C7916122E5A853082852F7C
:106B760083A3A3A3E0C3940A7480948050097BFF87
:106B86007ADE79DA12A8F8853082852F83A3A3A34B
:106B9600E0FF7E007B017A1C7916127D9A12A8F21C
:106BA60012CABE853082852F83A3E0C3940A7480FF
:106BB6009480500D7E1C7F227BFF7ADE79DA12A844
:106BC600FC853082852F83A3E0FF7E007B017A1C43
:106BD6007916127D9A12A8F212CABE853082852FC6
:106BE60083E0FF7E007B017A1C7916127D9A12A83B
:106BF600F27B2012CAC0E5302404F582E4352FF575
:106C060083E0C3940A74809480500D7E1C7F227B9F
:106C1600FF7ADE79DA12A8FCE5302404F582E43541
:106C26002FF583E0FF7E007B017A1C7916127D9A90
:106C360012A8F27E1C7F227B3A12CAC4E5302405D4
:106C4600F582E4352FF583E0C3940A74809480506E
:106C56000D7E1C7F227BFF7ADE79DA12A8FCE530F6
:106C66002405F582E4352FF583E0FF7E007B017A6B
:106C76001C7916127D9A12A8F27E1C7F227B3A128C
:106C8600CAC4E5302406F582E4352FF583E0C394C3
:106C96000A74809480500D7E1C7F227BFF7ADE79F9
:106CA600DA12A8FCE5302406F582E4352FF583E0F8
:106CB600FF7E007B017A1C7916127D9A12A8F2AF2C
:106CC60031126D127B017A1C792212D7A3C3EF947D
:106CD6003EEE9400501474222FF582741C3EF58308
:106CE6007420F00FBF00010E80E3901C60740DF05D
:106CF600A3740AF0AF35AE34AD33AC327B017A1CE7
:106D0600792275420075434012BFE1227C1C7D2228
:106D16007B407A008C3B8D3C8A3D8B3EEFB426004F
:106D26004003026EE1906D32F8282873026DA402CA
:106D36006DAD026DB6026DBF026DC8026DD1026DFA
:106D4600DA026DE3026DEC026DF5026DFE026E076E
:106D5600026E10026EE1026E19026E22026E2B02A4
:106D66006E34026E3D026E46026E4F026E58026E21
:106D760061026E69026E71026E79026E81026E891F
:106D8600026E91026E99026EA1026EA9026EB102A6
:106D96006EB9026EC1026EC9026ED1026ED97BFF58
:106DA6007ADA7946026EE77BFF7ADA7962026EE773
:106DB6007BFF7ADA797F026EE77BFF7ADA799F02C8
:106DC6006EE77BFF7ADA79C1026EE77BFF7ADA79C2
:106DD600DD026EE77BFF7ADA79F9026EE77BFF7AEE
:106DE600DB7915026EE77BFF7ADB793A026EE77B89
:106DF600FF7ADB7957026EE77BFF7ADB7977026EE3
:106E0600E77BFF7ADB799E026EE77BFF7ADB79B65A
:106E1600026EE77BFF7ADB79C4026EE77BFF7ADBE3
:106E260079E3026EE77BFF7ADC7902026EE77BFF8D
:106E36007ADC7924026EE77BFF7ADC7945026EE71D
:106E46007BFF7ADC7966026EE77BFF7ADC797E026D
:106E56006EE77BFF7ADC79A7026EE77BFF7ADC7947
:106E6600C8807E7BFF7ADC79EC80767BFF7ADD79E1
:106E76000F806E7BFF7ADD793880667BFF7ADD795D
:106E86004A805E7BFF7ADD796E80567BFF7ADD79FC
:106E96008F804E7BFF7ADD79AC80467BFF7ADD7989
:106EA600D2803E7BFF7ADD79F080367BFF7ADE7911
:106EB6000C802E7BFF7ADE793280267BFF7ADE79A4
:106EC60055801E7BFF7ADE797E80167BFF7ADE791F
:106ED60093800E7BFF7ADE79A880067BFF7ADE79C7
:106EE600C8AD3EAC3DAF3CAE3B12A90022E4901BC0
:106EF600A2F0A3F0901BA2E0FEA3E024A3F5827407
:106F0600093EF583E06010901BA3E004F070E59065
:106F16001BA2E004F080DD901BA3E004F070069055
:106F26001BA2E004F0901BA2E0FEA3E024A3F582DE
:106F360074093EF583E064316003027036901BA34A
:106F4600E004F07006901BA2E004F0E47FC0FEFDB2
:106F5600FC901B5AE0F8A3E0F9A3E0FAA3E0FBC318
:106F6600122A05601AE47FC0FEFDFC901B6DE0F856
:106F7600A3E0F9A3E0FAA3E0FBC3122A05704A9046
:106F86001BA2E0FEA3E024A3F974093EFA7B0112DA
:106F96009D707C007D0A1227FDEF25E025E0540C4C
:106FA600900982F0901BA2E0FEA3E024A3F97409E5
:106FB6003EFA7B01129D707C007D0A1227FDAF050B
:106FC600EF25E025E0540C8060E47FA17E16FDFCF1
:106FD600901B5AE0F8A3E0F9A3E0FAA3E0FBC31282
:106FE6002A0560030270C9901BA2E0FEA3E024A359
:106FF600F974093EFA7B01129D707C007D0A122706
:10700600FDEFC45470900982F0901BA2E0FEA3E04D
:1070160024A3F974093EFA7B01129D707C007D0A57
:107026001227FDAF05EFC45470900983F00270C9B2
:10703600901BA2E0FEA3E024A3F58274093EF5832B
:10704600E0B43225901BA3E004F07006901BA2E08A
:1070560004F0901BA2E0FEA3E024A3F58274093E8F
:10706600F583E0900984F0805A901BA2E0FEA3E02D
:1070760024A3F58274093EF583E064337048901BBF
:10708600A3E004F07006901BA2E004F0901BA2E0BF
:10709600FEA3E024A3F58274093EF583E0FFB43035
:1070A6000790098274BC8009EFB4310A9009827492
:1070B600BDF0A3F0800DEFB4320990098274BCF0E4
:1070C600A304F012D86822E4901BA2F0A3F0901B50
:1070D600A2E475F001122849FE74A325F0F5827426
:1070E600093EF583E070E7901BA2E0FEA3E024A32F
:1070F600F974093EFA7B0112915A901B5A122A5CC6
:10710600901BA2E0FEA3E024A3F58274093EF5835A
:10711600E06010901BA3E004F070E5901BA2E00471
:10712600F080DD901BA3E004F07006901BA2E00443
:10713600F0901BA2E0FEA3E024A3F974093EFA7BBB
:107146000112915A901B5E122A5C901BA2E0FEA3CC
:10715600E024A3F58274093EF583E06010901BA33A
:10716600E004F070E5901BA2E004F080DD901BA324
:10717600E004F07006901BA2E004F0901BA2E0FE73
:10718600A3E024A3F974093EFA7B0112915A901BDD
:1071960062EEF0A3EFF0901BA2E0FEA3E024A3F5BD
:1071A6008274093EF583E06010901BA3E004F07042
:1071B600E5901BA2E004F080DD900985740FF0A332
:1071C60074FFF0901B5EE0FCA3E0FDA3E0FEA3E0ED
:1071D600F52F8E2E8D2D8C2C7F007E367D6E7C01BC
:1071E60012D00B7E097FA3E4F52EFBFD12565878CC
:1071F600A57C1B7D017E007F031226D512D9219026
:107206001BA6A3E0FF12D8FE901BA6E0FF12D8FE35
:10721600901BA474FFF0901BA6A3E0FD7FFF12D97C
:10722600F5901BA4EFF0901BA6E0FD12D9F5901B7C
:10723600A4EFF0E4901BA2F0A3F0901BA6E0FEA33F
:10724600E0FF901BA2E0FCA3E0FDC39FEC9E503E36
:1072560074A32DF58274093CF583E0FF12D8FE90E5
:107266001BA4E0FF901BA2E0FCA3E024A3F582741C
:10727600093CF583E0FD12D9F5901BA4EFF0901BB5
:10728600A3E004F070B4901BA2E004F080AC901B65
:10729600A4E0FF02D8FE12D446901B41EEF0A3EF05
:1072A600F0E4F527C3E527940374809480501912FF
:1072B600202EE52725E024D0F582E4341BF583EE65
:1072C600F0A3EFF0052780DC901BD2E0FEA3E0FFE1
:1072D600901BD1E02FFF901BD0E03EFE901BD5E027
:1072E6002FFF901BD4E03EFE7C007D031227A89062
:1072F6001B37EEF0A3EFF07F1612C2C4EF24C0FDD9
:10730600EE34F9FC1223A9E4FBFA79C0783F122186
:10731600FE1223E2901B4BEEF0A3EFF07F1712C292
:10732600C4EF24C0FDEE34F9FC1223A9E4FBFA797C
:10733600C0783F1221FE1223E2901B4DEEF0A3EF20
:10734600F07F1312C2C4EE3395E0FDFCE47B0BFA2A
:10735600F9F81228C4901B39EEF0A3EFF07F121251
:10736600C2C4EE3395E0FDFCE47B0BFAF9F8122873
:10737600C4901B3BEEF0A3EFF07F1512C2C4EE33B0
:1073860095E0FDFCE47B0BFAF9F81228C4901B3D4E
:10739600EEF0A3EFF07F1412C2C4EE3395E0FDFCCD
:1073A600E47B0BFAF9F81228C4901B3FEEF0A3EF2A
:1073B600F07F3012C2C4901BCEEEF0A3EFF0FDAC0E
:1073C60006EC1223A97B337AB3796078C412210DB7
:1073D6007BB87A1E795578401223071223E2901B58
:1073E600CEEEF0A3EFF0901BCEE0FCA3E0FD901BE9
:1073F60045ECF0A3EDF0EC1223A97B3D7A0A793730
:1074060078401221FEE4FBFA7942784412210D7B82
:10741600007AF0797F78451221FEE4FBFA79167836
:10742600451223071223E2901BCEEEF0A3EFF09055
:107436001B43EEF0A3EFF012907BEF600F12907BF0
:10744600EF60097D1FAF16AE15129C11228B278A9D
:107456002889297B017A1C790C754A00754B0A7FAD
:10746600007E487D017C0012BF06901C0CE0FFF4F4
:10747600700AA3E0F47005A3E0F46052901BD2EF0B
:10748600F0901C0DE0901BD3F0901C0EE0901BD4E6
:10749600F0901C0FE0901BD1F0901C10E0901BCFD9
:1074A600F0901C11E0901BCEF0901C14E0FE901C96
:1074B60013E0FDED8E2DF52E7E1B7FCE7534FF7508
:1074C60035DE7536DCAB2EAA2D7D231260F6E4F58B
:1074D6002CC3E52C94407480948040030275AFE57C
:1074E6002C75F00AA4FFE42FFFE5F03440FEE434E7
:1074F60001FDE433FC7B017A1C790C754A00754B5F
:107506000A12BF06901C0CE0FFF4700DA3E0F470A5
:1075160008A3E0F470030275AF901BD2EFF0901C45
:107526000DE0901BD3F0901C0EE0901BD4F0901C45
:107536000FE0901BD1F0901C10E0901BCFF0901C38
:1075460011E0901BCEF0901C14E0FE901C13E0FDA1
:10755600EEF52DEDF52EE52E452D603C901C12E046
:107566006420701912DA1FAA06A9077534FF8A3536
:1075760089367E1B7FCE901C12E0FD80127E1B7F1B
:10758600CE901C12E0FD7534FF7535DE7536DFAB27
:107596002EAA2D1260F6800C7E1B7FCE901C12E068
:1075A600FD126B29052C0274D7AB27AA28A92975C9
:1075B6004A10754B007F007E307D017C0012BF06AD
:1075C600E4F52AF52BAE2AAF2BE4FCFDFB7A10F985
:1075D600F8D3122A054027AB27AA28A929852B828A
:1075E600852A83122714F4700B852B82852A8374CF
:1075F60020122786052BE52B70CB052A80C7229003
:107606001B47E0FCA3E0FDA3E0FEA3E02401FFE4AA
:107616003EFEE43DFDE43CFC901B47122A5C901BB9
:10762600A4122A6800000010900987E070069009ED
:10763600B374FFF0E4901BA2F0A3F0900987E0FF7B
:10764600901BA2E0FCA3E0FDC39FEC940040030264
:107656007720901B6775F013ED122A99EC75F013DD
:10766600A42583F583E0FEA3E024B3F58274093EE6
:10767600AF82F5228F23901B5E75F013ED122A99C7
:10768600EC75F013A42583F583E0FCA3E0FDA3E0ED
:10769600FEA3E0F52F8E2E8D2D8C2C7F007E367D61
:1076A6006E7C0112D00B901BA2E0FCA3E0FD901BA8
:1076B6006475F013122A99EC75F013A42583F583EB
:1076C600E0D39401748094805050AF23AE2212D13F
:1076D6008B78A87C1B7D017E007F031226D5901B2C
:1076E600A4E0F8A3E0F9A3E0FAA3E0FB901BA9E06D
:1076F600FEA3E0FFE4FCFDEB2FFFEA3EFEED39FDC5
:10770600EC38FC901BA4122A5C901BA3E004F070DA
:1077160006901BA2E004F00276417E097FA3128048
:107726003AE47F3FFEFDFC901BA4E0F8A3E0F9A33A
:10773600E0FAA3E0FBD3122A057E0040047F7F8097
:10774600027F3F901BAB12D91CE4901BA2F0A3F062
:10775600901BABE0FEA3E0FF901BA2E0FCA3E0FDC4
:10776600C39FEC9E501F74A32DF58274093CF583CC
:10777600E0FF12D8FE901BA3E004F070D3901BA28A
:10778600E004F080CB7E097FA3901BABE0FCA3E076
:10779600FD12D41C12D8FE901BABE0FEA3E0FF7DC9
:1077A600007B017A0979A3022E5A7F037E0012D24A
:1077B60022C3E51C940850030278FBE51D7004E51E
:1077C6001C6408702BAF11AE10AD0FAC0EF52EF584
:1077D6002F128912EF6016AA10AB117527FF7528B4
:1077E600E97529C77D16AF16AE1512794C0278D306
:1077F600900981E0C39402748094805069AF11AE01
:1078060010AD0FAC0EE4F52EF52F128912EF6016AF
:10781600AA10AB117527FF7528E97529C77D16AF24
:1078260016AE1512794CE5112401F511E43510F563
:1078360010E4350FF50FE4350EF50EAF11AE10ADB1
:107846000FFC752608752700128BF8EF6016AA1034
:10785600AB117527FF7528E97529C77D16AF16AEDA
:107866001512794C8067AF11AE10AD0FAC0EE4F572
:107876002EF52F128912EF6016AA10AB117527FF8D
:107886007528E97529C77D16AF16AE1512794CE530
:10789600112401F511E43510F510E4350FF50FE468
:1078A600350EF50EAF11AE10AD0FFC752E08752F07
:1078B60000128912EF6016AA10AB117527FF752802
:1078C600E97529C77D16AF16AE1512794CE5112458
:1078D60001F511E43510F510E4350FF50FE4350E1A
:1078E600F50EE4F51CF51D7E117F94FD7B017A09EA
:1078F60079A3122E5A12C04DEF64037008901CE053
:10790600E004F08005E4901CE0F0901CE0E0D394E5
:107916000A74809480400C7D1EAF16AE15129C1121
:10792600123EE17FFB7E457D1E7C00AB11AA10A9AD
:107936000FA80EC3122A05400C7D0BAF16AE15120A
:107946009C11123EE1228E228F238D248A258B26BE
:10795600E52464086003027A1DC3E5269498E525AC
:10796600943A5003027A1D75242312B1CF8F2D8EBF
:107976002C8D2B8C2A7F007E507D017C00AB2DAA9E
:107986002CA92BA82AC3122A054003027ACA7E0014
:107996007F0A7D007B017A1C790C122E5AE523247E
:1079A60004F582E43522F583E0901C0CF0E52324EF
:1079B60005F582E43522F583E0901C0DF0E52324DD
:1079C60006F582E43522F583E0901C0EF0852382CD
:1079D600852283A3A3A3E0901C0FF0852382852232
:1079E60083A3E0901C10F0852382852283E0901CFF
:1079F60011F0A3E524F0E526A3F0E525A3F0E4A322
:107A0600F0AF2DAE2CAD2BAC2A7B017A1C790CF590
:107A16004275430A12BFE112B14B8F2D8E2C8D2B6E
:107A26008C2A7F007E487D017C00AB2DAA2CA92BD9
:107A3600A82AC3122A054003027ACA7E007F0A7D5D
:107A4600007B017A1C790C122E5AE5232404F58258
:107A5600E43522F583E0901C0CF0E5232405F5823D
:107A6600E43522F583E0901C0DF0E5232406F5822B
:107A7600E43522F583E0901C0EF08523828522836F
:107A8600A3A3A3E0901C0FF0852382852283A3E0A5
:107A9600901C10F0852382852283E0901C11F0A3B0
:107AA600E524F0E526A3F0E525A3F0E4A3F0AF2D49
:107AB600AE2CAD2BAC2A7B017A1C790CF5427543B2
:107AC6000A12BFE122E4901BA2F0A3F0901BA2E4ED
:107AD60075F001122849FE74A325F0F58274093E5B
:107AE600F583E070E7901BA2E0FEA3E024A3F974FF
:107AF600093EA801FC7D017BFF7ADE79E1122C9319
:107B0600EF3395E04F70061293E4027BEE901BA2D2
:107B1600E0FEA3E024A3F974093EA801FC7D017BE5
:107B2600FF7ADE79E8122C93EF3395E04F70061258
:107B3600C87D027BEE901BA2E0FEA3E024A3F974AD
:107B4600093EA801FC7D017BFF7ADE79EE122C93BB
:107B5600EF3395E04F700612C829027BEE901BA208
:107B6600E0FEA3E024A3F974093EA801FC7D017B95
:107B7600FF7ADE79F4122C93EF3395E04F70719013
:107B86001BA2E475F001122849FE74A325F0F582C4
:107B960074093EF583E070E7901BA2E0FEA3E024A3
:107BA600A3F974093EFA7B01129D70901BA4EEF0B6
:107BB600A3EFF0901BA2E475F001122849FE74A30E
:107BC60025F0F58274093EF583E070E7901BA2E08C
:107BD600FEA3E024A3F58274093EAF82FE901BA4A7
:107BE600E0FCA3E0FD12AEA7901BA6EEF0A3EFF01B
:107BF600901BA6E07002A3E0603F12D921E4901B1F
:107C0600A2F0A3F0901BA6E0FEA3E0FF901BA2E06B
:107C1600FCA3E0FDC39FEC9E502274002DF58274F8
:107C2600003CF583E0FF12D8FE901BA3E004F07041
:107C3600D3901BA2E004F080CB12D87A228F408E1C
:107C46003F8D3E8C3D85A74575A710AB44AA43A939
:107C560042A841AF40AE3FAD3EAC3D12294FE47B5A
:107C660002FAF9F812294FE47BFFFAF9F8D3122A3F
:107C760005402AAB44AA43A942A841AF40AE3FAD56
:107C86003EAC3D12294FE47B02FAF9F812294F1255
:107C960029E18F8D538EF4438E08027D87AB44AA6B
:107CA60043A942A841AF40AE3FAD3EAC3D12294F7D
:107CB600E47B02FAF9F812294FE47B04FAF9F81288
:107CC600294FE47BFFFAF9F8D3122A054033AB4477
:107CD600AA43A942A841AF40AE3FAD3EAC3D1229F2
:107CE6004FE47B02FAF9F812294FE47B04FAF9F81B
:107CF60012294F1229E18F8D538EF4438E01027D96
:107D060087AB44AA43A942A841AF40AE3FAD3EACC3
:107D16003D12294FE47B02FAF9F812294FE47B0C55
:107D2600FAF9F812294FE47BFFFAF9F8D3122A057B
:107D3600AB44AA43A942A841AF40AE3FAD3EAC3DDD
:107D4600401F12294FE47B02FAF9F812294FE47B0F
:107D56000CFAF9F812294F1229E18F8D538EF4800F
:107D66002012294FE47B02FAF9F812294FE47B30FE
:107D7600FAF9F812294F1229E18F8D538EF4438EAA
:107D860002858D8B53890F438920D28ED29DD29C3A
:107D96008545A7228E3B8F3C8B3D8A3E893F7C00E2
:107DA6007D0A1227FD900004ED122786AE3BAF3CFC
:107DB6007C007D0A1227FD8E3B8F3C7C007D0A12DB
:107DC60027FDAB3DAA3EA93F900003ED122786AEE4
:107DD6003BAF3C7C007D0A1227FD8E3B8F3C7C002E
:107DE6007D0A1227FDAB3DAA3EA93F900002ED1287
:107DF6002786AE3BAF3C7C007D0A1227FD8E3B8F6B
:107E06003C7C007D0A1227FDAB3DAA3EA93F9000AF
:107E160001ED122786AE3BAF3C7C007D0A1227FDA2
:107E26008E3B8F3C7C007D0A1227FDAB3DAA3EA906
:107E36003FED122774E4901BD7F0901BD7E0FFC3E9
:107E4600940574809480501DAB3DAA3EA93F8F8255
:107E5600758300122714FF3395E04F7008901BD7E7
:107E6600E004F080D5901BD7E06405701BAB3DAAFB
:107E76003EA93F7430122774AB3DAA3EA93F90003D
:107E860001E41227867F0122E4901BD8F0901BD7CD
:107E9600E0FFC374059FFEA3E0FDC39E5029ED2FAE
:107EA600F582E433F583AB3DAA3EA93F122714249D
:107EB60030FF901BD8E0F582758300EF122786907D
:107EC6001BD8E004F080C6901BD7E0FFFDC3740505
:107ED6009DFDE49400AB3DAA3EA93F8D82F583E467
:107EE600122786C374059FFF2212D9A412D58412C5
:107EF600DA3712D46F12D8E012202612D3C67F01C9
:107F060012200612D71C12CA6EC297E490096AF0B4
:107F160090096CF09009687403F09009677409F091
:107F26001284E990096F122A5C90096AE0C39406EC
:107F36007480948050147525017526097527647B15
:107F4600017A1B79371296FF80DF12729C12D8EFE6
:107F560090096BEFF064017012900966E0640260AC
:107F66000512206E800812C0B9800312C123900941
:107F760068E014700302802514601A24FD607624DC
:107F8600FE700302802E147003028034240570DE16
:107F960012B7C180D912ABDF128DCAEF4E60277FB0
:107FA6000112200612DA437527FF7528E97529FFA5
:107FB600901B53E0FAA3E0FB7D08AF16AE151279CD
:107FC6004CE4FF122006901B9CE0640170A0F07F39
:107FD6000112200612DA437527FF7528E97529FF75
:107FE6007B2A7A2B7D08AF16AE1512794CE4FF1268
:107FF6002006027F74129579128DCAEF4E70030225
:108006007F747527FF7528E97529FF901B53E0FAE1
:10801600A3E0FB7D08AF16AE1512794C027F7412F1
:10802600B745128DCA027F7412BDB8027F7412D48E
:1080360098027F748E278F28901B47A3A3A3E08501
:108046002882852783F0901B47E0FCA3E0FDA3E090
:10805600FEA3E0FF7808122A16852882852783A3C7
:10806600EFF0901B4BE0FEA3E0852882852783A3D3
:10807600A3F0EEFF852882852783A3A3A3EFF090C4
:108086001B4DE0FEA3E0FDE5282404F582E4352738
:10809600F583EDF0EEFFE5282405F582E43527F5B6
:1080A60083EFF0901B51E0FEA3E0FF12B3D6901BC6
:1080B6004FEEF0A3EFF0E4A3F0A3F0901B4FE0FE29
:1080C600A3E0FDE5282406F582E43527F583EDF0E7
:1080D600EEFFE5282407F582E43527F583EFF090D7
:1080E6001B37E0FEA3E0FDE5282408F582E43527EA
:1080F600F583EDF0EEFFE5282409F582E43527F552
:1081060083EFF0901B39E0FEA3E0FDE528240AF595
:1081160082E43527F583EDF0EEFFE528240BF582A2
:10812600E43527F583EFF0901B43E0FEA3E0FDE581
:1081360028240CF582E43527F583EDF0EEFFE528DB
:10814600240DF582E43527F583EFF0901B3BE0FE26
:10815600A3E0FDE528240EF582E43527F583EDF04E
:10816600EEFFE528240FF582E43527F583EFF022AC
:10817600901B5A122A6800001AA1901B5E122A68E8
:108186000016E360901B62E4F0A304F0A3F0E49011
:108196001B67F0A3F0900985740FF0A374FFF0A39A
:1081A6007401F07E117F947D00FB7A0979A3122E6B
:1081B6005A901B5EE0FCA3E0FDA3E0FEA3E0F52FD2
:1081C6008E2E8D2D8C2C7F007E367D6E7C0112D0FE
:1081D6000B7E097FA3E4F52EFBFD12565878A57C8D
:1081E6001B7D017E007F031226D5901BA5E070063D
:1081F6009009CC7490F012D9219009CCE0FF12D8E6
:10820600FE7F009009CDEFF012D8FE9009A6E0FFA0
:108216009009CEF012D8FE9009A5E0FF9009CFF0A4
:1082260012D8FE7F009009D0EFF012D8FE7F0090A2
:1082360009D1EFF012D8FE7F059009D2EFF012D8DF
:10824600FE7F009009D3EFF012D8FE7E097FCC7D29
:10825600087C0012D41C12D8FE901BA2E4F0A304E2
:10826600F0901BA2E0FEA3E0FFC39429EE94005019
:108276001F74A32FF58274093EF583E0FF12D8FE22
:10828600901BA3E004F07006901BA2E004F080D1DE
:108296007E097FA37D287C0012D41C02D8FE901B89
:1082A60047E0FCA3E0FDA3E0FEA3E0FFC0079009C2
:1082B60081E0FBE4FAF9F8D00712294F901B471228
:1082C6002A5C74A3251DF5827409351CAF82FE1243
:1082D600803A901B47E0F8A3E0F9A3E0FAA3E0FB9D
:1082E600900981E0FFE4FCFDFE1228C4901B4712B2
:1082F6002A5C900986E024EEFF900985E034FFFEB3
:1083060074A3251DF5827409351CF583E5822FF5C6
:1083160082E5833EAF82FE12C25E900986E024F6B5
:10832600FF900985E034FFFE74A3251DF5827409CC
:10833600351CF583E5822FF582E5833EAF82FE127A
:10834600C3EF900985E0FEA3E0FF7491251DF58239
:108356007409351CF583E5822FF582E5833EAF82ED
:10836600FE7D107C0012D41C900985E0FCA3E0FD84
:10837600251DFBE51C3CFA74A12BF58274093AF520
:1083860083EFF074A3251DF5827409351CAF82FEB8
:10839600ED24FFFDEC34FFFC12D41C900985E0FCB3
:1083A600A3E0FD251DFBE51C3CFA74A22BF58274A7
:1083B600093AF583EFF0ED251DF51DEC351CF51C8E
:1083C60022129937E4901BA2F0A3F0901BA2E47549
:1083D600F001122849FE74A325F0F58274093EF5D2
:1083E60083E070E7901BA4F0901BA4E0C39408748C
:1083F600809480505F901BA2E475F001122849FE1C
:1084060074A325F0F58274093EF583E0FF12D68940
:10841600901BA5EFF0E0C454F0F0901BA2E475F0B9
:1084260001122849FE74A325F0F58274093EF583EE
:10843600E0FF12D689901BA5E02FF0E0FF901BA469
:10844600E02493F582E4341BF583EFF0901BA4E05F
:1084560004F0809412BB7FEF600B12D9217BFF7A68
:10846600E079BA807512C5C3EF600B12D9217BFF84
:108476007AE079CD806412B3577E047F007D007B5D
:10848600017A0D79A3122E5A78A37C097D017B010E
:108496007A0079007E047F001226D57E097FA37DAF
:1084A600FE7C0312D41C900DA1EFF07B017A0979B2
:1084B600A37DFF7C0312D0EE900DA2EFF0E4F5262B
:1084C600F5277F907E08FDFC128CE1EF700302D841
:1084D6006812D9217BFF7AE079DB1243C3E4FF12ED
:1084E600D8FE22E4F525F524F523F5227F3812D9A6
:1084F60058901BA2EFF07F3912D958901BA3EFF0CA
:108506007F3A12D958901BA4EFF07F3B12D95890AE
:108516001BA5EFF07F3C12D958901BA6EFF07F3DCC
:1085260012D958901BA7EFF07F3E12D958901BA87E
:10853600EFF07F3F12D958901BA9EFF07E1B7FA268
:108546007D037C0012D41C901BA5E0B50731901B5F
:10855600A3E0FFE4FCFDFE7808122A29A804A90579
:10856600AA06AB07901BA2E0FFEB4FFFEAFEE9FD70
:10857600E8FCC004C005C006C007901BA480417E6D
:108586001B7FA67D037C0012D41C901BA9E0B507B7
:1085960054901BA7E0FFE4FCFDFE7808122A29A8E8
:1085A60004A905AA06AB07901BA6E0FFEB4FFFEA5E
:1085B600FEE9FDE8FCC004C005C006C007901BA884
:1085C600E0FFE4FCFDFE7810122A29D003D002D089
:1085D60001D000EF4BF525EE4AF524ED49F523ECE5
:1085E60048F5228009E4F525F524F523F522AF2583
:1085F600AE24AD23AC222212C50DEF60097D09AF72
:1086060016AE15129C117E117F947D007B017A09AE
:1086160079A3122E5A78A37C097D017B017A007911
:10862600007E097F601226D5E4F52EF52F7F807E29
:1086360008FDFC1289127E117F947D007B017A0968
:1086460079A3122E5A78A37C097D017B017A0079E1
:10865600007E097F601226D5E4F52EF52F7F907EE9
:1086660008FDFC12891212DA3A8F298E288D278C82
:1086760026E47F517E08FDFCAB29AA28A927A82657
:10868600C3122A0550037F0422E5292470FFE5283A
:1086960034F7FEE52734FFFDE52634FFFCE4FB7ADC
:1086A60008F9F81228C48F258E248D238C227E117A
:1086B6007F947D007B017A0979A3122E5A900A3F96
:1086C600E525F0FFAE24AD23AC227808122A16A3C6
:1086D600EFF0AF25AE24AD23AC227810122A16A3F4
:1086E600EFF0AF25AE24AD23AC227818122A16A3DC
:1086F600EFF0E4F52EF52FFF7E08FDFC1289127FC0
:1087060000228F4B8E4A8D498C4885A74DA2AF9289
:108716000085F54E85EF5185FF52C2AFE4F5A7FF00
:108726007E80FDFCAB4BAA4AA949A848C3122A057C
:10873600500B854A4F854B5053F5CF8076E4FFFEAC
:108746007D01FCAB4BAA4AA949A848C3122A055089
:1087560020E54BF54BE54A4480F54AE549F549E500
:1087660048F548854A4F854B5053F5CF43F5108061
:10877600427F007E807D017C00AB4BAA4AA949A8B6
:1087860048C3122A055020E54BF54BE54A4480F5CF
:108796004AE549F549E548F548854A4F854B505322
:1087A600F5CF43F520800C854A4F854B5053F5CFC6
:1087B60043F530E4F5EF75FFA0FFEFC394FF748037
:1087C600948050030F80F3E5FF30E62975EF0275BC
:1087D600B7A575B7F1438F0175FFA075EF028550F8
:1087E60082854F83E54CF0E4F5EF8552FF8551EF26
:1087F600538FFE80068552FF8551EF854EF5854DD8
:10880600A7A20092AF7F01228F298E288D278C2662
:1088160085A72AA2AF920085F52B85EF2E85FF2F1F
:10882600C2AFE4F5A7FF7E80FDFCAB29AA28A927E5
:10883600A826C3122A05500B85282C85292D53F509
:10884600CF8076E4FFFE7D01FCAB29AA28A927A8E4
:1088560026C3122A055020E529F529E5284480F586
:1088660028E527F527E526F52685282C85292D5385
:10887600F5CF43F51080427F007E807D017C00AB02
:1088860029AA28A927A826C3122A055020E529F5D2
:1088960029E5284480F528E527F527E526F52685E8
:1088A600282C85292D53F5CF43F520800C85282CBF
:1088B60085292D53F5CF43F530E4F5EF75FFA0FF7D
:1088C600EFC394FF7480948050030F80F3E5FF306C
:1088D600E62775EF0275B7A575B7F1438F0375FFE8
:1088E600A075EF02852D82852C83E4F0F5EF852FA8
:1088F600FF852EEF538FFC8006852FFF852EEF8593
:108906002BF5852AA7A20092AF7F01227536FF7547
:1089160037E575387A8F3C8E3B8D3A8C397B017AF8
:108926001C79B51243BD8F32753A607539E37538D7
:10893600167537007F007E367D6E7C0112D045E4C9
:10894600F530F53174632531F58274E73530F583FA
:10895600E493FF12D88C0531E53170020530C394DB
:108966000AE530940040DDE4F530F531C3E5319594
:1089760032E5309400501B74B52531F582741C35F0
:1089860030F583E0FF12D88C0531E53170DE053015
:1089960080DAE4FF12D88C852E30852F31E4252F1E
:1089A600FFE52E3408FEC3E5319FE5309E501B746B
:1089B600A32531F58274093530F583E0FF12D88C92
:1089C6000531E53170D7053080D37F647E007D00A8
:1089D6007C0012BA97EF702EC3900961E094029062
:1089E6000960E09400401C78007C007D017BFF7AE2
:1089F600E579817E007F02122E36EF3395E04F70C7
:108A060002FF227F01227F0122E4901BA2F0A3F045
:108A1600901BA2E475F001122849FE74A325F0F517
:108A26008274093EF583E070E7901BA2E0FEA3E0A6
:108A360024A3F974093EFA7B0112915A901BA412E1
:108A46002A5C901BA2E475F001122849FE74A32546
:108A5600F0F58274093EF583E070E7901BA2E0FE14
:108A6600A3E024A3F974093EFA7B01129D70901BC2
:108A7600A8EEF0A3EFF0901BA2E475F001122849CE
:108A8600FE74A325F0F58274093EF583E070E77E57
:108A9600097F60FD7B017A007900122E5AE4901B53
:108AA600AAF0A3F0901BA4E0FCA3E0FDA3E0FEA3C4
:108AB600E0FF901BA2E0F526A3E0F527901BA8E0B7
:108AC600F528A3E0F529129238EF703812D92190D3
:108AD6001BAAE0FEA3E02400F58274003EF583E0C5
:108AE600601D901BAAE475F001122849FE7400254A
:108AF600F0F58274003EF583E0FF12D8FE80D0E4E4
:108B0600FF12D8FE228B238A248925AB26AA27A901
:108B1600281226FBFFAB23AA24A9251226FBFE6FEB
:108B2600600AEEC39F7F0150027FFF22AB26AA2771
:108B3600A928900001122714FFAB23AA24A9259087
:108B46000001122714FE6F600AEEC39F7F015002D8
:108B56007FFF22AB26AA27A928900003122714FF1D
:108B6600AB23AA24A925900003122714FE6F600ADE
:108B7600EEC39F7F0150027FFF22AB26AA27A928BA
:108B8600900004122714FFAB23AA24A92590000401
:108B9600122714FE6F600AEEC39F7F0150027FFF0B
:108BA60022AB26AA27A928900005122714FFAB237B
:108BB600AA24A925900005122714FE6F600AEEC3A9
:108BC6009F7F0150027FFF22AB26AA27A92890008B
:108BD60006122714FFAB23AA24A925900006122704
:108BE60014FE6F600AEEC39F7F0150027FFF227F53
:108BF60000227536FF7537E575387A8F3C8E3B8DCA
:108C06003A8C397B017A1C79B51243BD8F2A753AA5
:108C1600607539E37538167537007F007E367D6ED0
:108C26007C0112D045E4F528F529746D2529F582D5
:108C360074E73528F583E493FF12D88C0529E529D6
:108C460070020528C3940BE528940040DDE4F5285E
:108C5600F529C3E529952AE5289400501B74B52506
:108C660029F582741C3528F583E0FF12D88C052976
:108C7600E52970DE052880DAE4FF12D88C852628DF
:108C8600852729E42527FFE5263408FEC3E5299F25
:108C9600E5289E501B74A32529F58274093528F50D
:108CA60083E0FF12D88C0529E52970D7052880D3E3
:108CB6007F967E007D007C0012BA97EF701A7800CE
:108CC6007C007D017BFF7AE57981122C93EF339549
:108CD600E04F7F017004FF227F01227536FF753752
:108CE600E575387A8F3C8E3B8D3A8C397B017A1C40
:108CF60079B51243BD8F2A753A607539E375381612
:108D06007537007F007E367D6E7C0112D045E4F516
:108D160028F52974632529F58274E73528F583E457
:108D260093FF12D88C0529E52970020528C3940AF9
:108D3600E528940040DDE4F528F529C3E529952AC0
:108D4600E5289400501B74B52529F582741C352836
:108D5600F583E0FF12D88C0529E52970DE05288009
:108D6600DAE4FF12D88C852628852729E42527FFF3
:108D7600E5263408FEC3E5299FE5289E501B74A30B
:108D86002529F58274093528F583E0FF12D88C056C
:108D960029E52970D7052880D37FB87E0B7D007C16
:108DA6000012BA97EF701A78007C007D017BFF7A7B
:108DB600E57981122C93EF3395E04F7F017004FF24
:108DC600227F01227F1812D0B7901BA4EEF0A3EFEA
:108DD600F07F1912D0B7901BA6EEF0A3EFF0901B10
:108DE600A4E0FCA3E02400FDEC34FAFC901BA8F000
:108DF600A3EDF0E42FFFEE34FAA3F0A3EFF0C3ECFB
:108E0600648094805015901BA8E0FEA3E0FFC3E4A5
:108E16009FFFE49E901BA8F0A3EFF0901BAAE0FE34
:108E2600A3E0FFC3EE64809480500DC3E49FFFE48B
:108E36009E901BAAF0A3EFF0901BAAE0FEA3E0FF12
:108E4600901BA8E0FCA3E0FDD39FEE6480F8EC64E1
:108E560080984006AE04AF058000901BA2EEF0A3FA
:108E6600EFF0C3901B52E09F901B51E09E500F9075
:108E76001BA2E0FFA3E0901B51CFF0A3EFF0901BE5
:108E8600A2E0FEA3E0FFC394BFEE94014019D3EF26
:108E960094D7EE9403501012CF0E901B53EEF0A30E
:108EA600EFF07E007F0122E4FEFF22E4901BA2F099
:108EB600A3F0901BA2E475F001122849FE74A325C5
:108EC600F0F58274093EF583E070E7901BA2E0FEA0
:108ED600A3E024A3F974093EFA7B0112915A901B70
:108EE600A4122A5C901BA2E475F001122849FE74B4
:108EF600A325F0F58274093EF583E070E7901BA286
:108F0600E0FEA3E024A3F974093EFA7B01129D70EA
:108F1600901BA8EEF0A3EFF0901BA2E475F00112EF
:108F26002849FE74A325F0F58274093EF583E070A6
:108F3600E77E097F60FD7B017A007900122E5AE4F4
:108F4600901BAAF0A3F0901BA4E0FCA3E0FDA3E015
:108F5600FEA3E0FF901BA2E0F52EA3E0F52F1289F9
:108F660012EF700B12D9217BFF7ADF796380091229
:108F7600D9217BFF7ADF7983901BA4E0FCA3E0FD77
:108F8600A3E0FEA3E0F5398E388D378C361243C345
:108F960022901CE2E004F07006901CE1E004F0D39D
:108FA600901CE2E094E0901CE1E0940150030290F2
:108FB6007A90096FE0FCA3E0FDA3E0FEA3E02401A4
:108FC600FFE43EFEE43DFDE43CFC90096F122A5CA2
:108FD600E4901CE1F0A3F090096FE0FCA3E0FDA390
:108FE600E0FEA3E0FF901BA2EFF090096FA3A3A3FE
:108FF600E07808122A16901BA3EFF090096FE0FCA8
:10900600A3E0FDA3E0FEA3E0FF7810122A16E49089
:109016001BA4EFF07E1B7FA27D037C0012D41C9064
:109026001BA5EFF0901BA2E0FD7F3812D965901BBF
:10903600A3E0FD7F3912D965901BA4E0FD7F3A12AB
:10904600D965901BA5E0FD7F3B12D965901BA2E078
:10905600FD7F3C12D965901BA3E0FD7F3D12D965CB
:10906600901BA4E0FD7F3E12D965901BA5E0FD7F15
:109076003F12D965227E1B7FD67C1B7DF112AF3253
:109086007E1B7FD67C1B7DF112AFBD7E1B7FDF7CF6
:109096001B7DFA12AF327E1B7FDF7C1B7DFA12AF7F
:1090A600BD7E1B7FE87C1C7D0312AF327E1B7FE8F2
:1090B6007C1C7D0312AFBD7E1B7FF17C1B7DFA12EB
:1090C600AA26EF700C7FF17C1C7D0312AA26EF60A6
:1090D6002178917C097D017B017A1B79F17E007FE5
:1090E600091226D578787C097D017B017A1B79D611
:1090F600802D7E1B7FFA7C1C7D0312AA26EF60283A
:1091060078917C097D017B017A1B79FA7E007F09C3
:109116001226D578787C097D017B017A1B79DF7E62
:10912600007F091226D5802978917C097D017B0173
:109136007A1C79037E007F091226D578787C097D12
:10914600017B017A1B79E87E007F091226D57F0113
:10915600227F00228B238A248925AB23AA24A925D2
:109166001226FBFF12D855500D74012525F525E46E
:109176003524F52480E4D200AB23AA24A92512269F
:10918600FBFF642B6004EFB42D1BAB230525E525FF
:10919600AA247002052414F91226FB642D6003D359
:1091A6008001C39200E4F529F528F527F526AB23BF
:1091B600AA24A9251226FBFF12D949505CE47F0A8E
:1091C600FEFDFCAB29AA28A927A8261228C4C8ECAC
:1091D600C8EDC0E0EEC0E0EFC0E0AB23AA24A925AD
:1091E6001226FBFF3395E0FEEF24D0FFEE34FFFEA0
:1091F600E4FCFDD0E0FBD0E0FAD0E0F9EB2FF52956
:10920600EA3EF528ED39F527EC38F52674012525D3
:10921600F525E43524F524809530000AAF29AE28DB
:10922600AD27AC26800BAF29AE28AD27AC26122978
:10923600E1228F258E248D238C227536FF7537E526
:1092460075387A8F3C8E3B8D3A8C397B017A1C7946
:10925600B51243BD8F2C753A607539E375381675AE
:1092660037007F007E367D6E7C0112D045E4F52AFC
:10927600F52B74BE252BF58274E6352AF583E49327
:10928600FF12D88C052BE52B7002052AC3940DE539
:109296002A940040DDAF2512D88CAF25AE24AD232D
:1092A600AC227808122A1612D88CAF25AE24AD232C
:1092B600AC227810122A1612D88CAF25AE24AD2314
:1092C600AC227818122A1612D88C85262A85272BC6
:1092D600E5292527FFE5283526FEC3E52B9FE52A48
:1092E6009E501B74A3252BF5827409352AF583E05D
:1092F600FF12D88C052BE52B7002052A80D27F64DD
:109306007E007D007C0002BA9712AB4D9009641274
:10931600D91C7F6412D8FEE4FF12D8FE7F6412D8EF
:10932600FEE4FF12D8FE7F6412D8FEE4FF12D8FED8
:10933600E4901BA2F0A3F0E4FF12D8FE901BA3E07A
:1093460004F07006901BA2E004F0C3901BA3E09407
:109356000B901BA2E0940040DEE4FF12D8FE7F12C1
:1093660012D8FE7F7A12D8FEE4FF12D8FEE4901BD4
:10937600A2F0A3F0901BA2E0FEA3E0FFC39407EEC9
:1093860094005020745B2FF58274E23EF583E493DB
:10939600FF12D8FE901BA3E004F070D8901BA2E049
:1093A60004F080D0E4901BA2F0A3F0E4FF12D8FEF4
:1093B600901BA3E004F07006901BA2E004F0C3909B
:1093C6001BA3E09410901BA2E0940040DE90096479
:1093D600A3E0FF12D8FE900964E0FF02D8FE78A849
:1093E6007C1B7D017BFF7AE679657E007F0812266D
:1093F600D5E4901BB0F0901BB0E0C3940274809447
:109406008040030294AD7E097F607D007B017A0077
:109416007900122E5A901BB0E025E025E024A8F52D
:1094260082E4341BF583E0FCA3E0FDA3E0FEA3E0A9
:10943600F53A8E398D388C377F007E367D6E7C010D
:1094460012D045E4F522F523745D2523F58274E6F2
:109456003522F583E493FF12D88C0523E5237002A9
:109466000522C39408E522940040DDE4FF12D88C5F
:109476007F327E007D007C0012BA97EF7020F522C5
:10948600F5230523E523AE2270020522142400F5F8
:109496008274003EF583E070E9AE22AF2322901B72
:1094A600B0E004F00293FCE4FEFF22753A607539E1
:1094B600E37538167537007F007E367D6E7C0112A7
:1094C600D045E4F52AF52B74D4252BF58274E535C1
:1094D6002AF583E493FF12D88C052BE52B70020541
:1094E6002AC3940FE52A940040DD7F987E3A7D00DA
:1094F6007C0012BA97EF706C900002E0FFE4FCFD6E
:10950600FE7810122A29E4FFFEE4FCA804A905AAA5
:1095160006AB07900001E0FE900000E02400FFEC9F
:109526003EFEE4FDEB2FFFEA3EFEED39FDEC38FC96
:10953600C004C005C006C007900003E0FFE4FCFDC0
:10954600FE7818122A29E4FFFEFDD003D002D001CE
:10955600D000EF2BF52FEE3AF52EED39F52DE83C40
:10956600F52C8006E4FFFEFDFC22AF2FAE2EAD2DBE
:10957600AC2C22E517700302963BE4F517128F9781
:10958600901CDFE004F0E0D3941E748094804002C7
:10959600E4F0901CDFE0C31390E9CC9324FF92978C
:1095A600901B47E0FCA3E0FDA3E0FEA3E02401FF3F
:1095B600E43EFEE43DFDE43CFC901B47122A5C9031
:1095C6000981E0FBE4FAF9F8901B47E0FCA3E0FD13
:1095D600A3E0FEA3E0FF12294FAC00AD01AE02AF3F
:1095E60003E4FBFAF9F8C3122A05701412729C12EE
:1095F600535C901B55EFF01282A41277B0125BF603
:109606007525017526097527647B017A1B79371242
:1096160096FF90096AE0D39406748094804016E41D
:10962600F0900966E06402600C7D1DAF16AE15125F
:109636009C11123EE122E4901BA2F0A3F0901BA223
:10964600E475F001122849FE74A325F0F582740929
:109656003EF583E070E7901BA2E0FEA3E024A3F9A9
:1096660074093EFA7B0112915A901BA4122A5CE4FB
:109676007B02FAF9F8901BA4E0FCA3E0FDA3E0FE50
:10968600A3E0FF12294FEF24FFFFEE34FFFEED3477
:10969600FFFDEC34FFFC901BA8122A5C901BA8E08F
:1096A600FCA3E0FDA3E0FEA3E02470FFE43EFEE49D
:1096B6003DFDE43CFC901BA8122A5C901BA2E475BD
:1096C600F001122849FE74A325F0F58274093EF5CF
:1096D60083E070E7901BA8E0FCA3E0FDA3E0FEA3F7
:1096E600E0FF901BA2E0F52EA3E0F52F128912EF02
:1096F600700302D86812D87A228B228A238924AB77
:1097060025AA26A92790000412271464057008903C
:109716001CE37404F0801590000A122714600D9063
:10972600000AE4122786901CE3E004F0901CE3E0B4
:10973600C394047480948050030297C0E4F0AB2273
:10974600AA23A92412C979AB22AA23A9249000022C
:1097560012285FFFAEF090000412285FFDACF0D334
:109766009FEC9E4011D3ED9470EC94177F0140025C
:109776007F038F28801DAB22AA23A9249000041200
:10978600285FFFAEF090000212285FD39FE5F09E9F
:10979600752802AB25AA26A9279000021227146570
:1097A60028600F900002E528122786900006E40242
:1097B60027869000067401122741228F538E528D00
:1097C600518C5085A754A2AF920085F555C2AFE4DF
:1097D600F5A7FF7E80FDFCAB53AA52A951A850C342
:1097E600122A05500B85525685535753F5CF80766E
:1097F600E4FFFE7D01FCAB53AA52A951A850C31247
:109806002A055020E553F553E5524480F552E551BB
:10981600F551E550F55085525685535753F5CF43CC
:10982600F51080427F007E807D017C00AB53AA52FA
:10983600A951A850C3122A055020E553F553E55205
:109846004480F552E551F551E550F550855256855F
:10985600535753F5CF43F520800C85525685535701
:1098660053F5CF43F530855782855683E493FF85BC
:1098760055F58554A7A20092AF227536FF7537E5D8
:1098860075387A8F3C8E3B8D3A8C397B017A1C7900
:10989600B51243BD8F24753A607539E37538167570
:1098A60037007F007E367D6E7C0112D045E4F522BE
:1098B600F52374632523F58274E73522F583E49353
:1098C600FF12D88C0523E52370020522C3940AE50E
:1098D60022940040DDE4F522F523C3E5239524E533
:1098E600229400501B74B52523F582741C3522F58D
:1098F60083E0FF12D88C0523E52370DE052280DA8B
:10990600E4FF12D88C7F647E007D007C0012BA973B
:10991600EF701978007C007D017BFF7AE579811272
:109926002C93EF3395E04F7003FEFF227E007F01FC
:10993600227D0A7FAC12A855901B9DE0F526900962
:1099460095E526F0FF12D7BD90097CEFF0E48F2550
:10995600F524F523F522AE24AD23AC227810122A85
:10996600298F258E248D238C227D097FAC12A85544
:10997600901B9DE0F526900996E526F0FF12D7BDCF
:1099860090097DEFF0AF2612D7BDEF7F00FE33952D
:10999600E0FDFCEF2525F525E5243EF524E5233DF0
:1099A600F523E5223CF5227D087FAC12A855901BD5
:1099B6009DE0F526900997E526F0FF12D7BD9009A0
:1099C6007EEFF0AF2612D7BDE4FCFDFEE5252FF5B0
:1099D60025EE3524F524ED3523F523EC3522F52245
:1099E600AF25AE24AD23FC229000B8E0FF12D7BD10
:1099F600900988EFF09000B9E0FF12D7BD90098971
:109A0600EFF09000BAE0FF12D7BD90098AEFF09010
:109A160000BBE0FF12D7BD90098BEFF09000BCE0D1
:109A2600FF12D7BD90098CEFF09000BDE0FF12D772
:109A3600BD90098DEFF09000BEE0FF12D7BD9009F2
:109A46008EEFF09000C1E0FF12D7BD90099AEFF0BB
:109A56009000C2E0FF12D7BD90099BEFF09000C3C3
:109A6600E0FF12D7BD90099CEFF09000C4E0FF1212
:109A7600D7BD90099DEFF09000C5E0FF12D7BD90CD
:109A8600099EEFF09000C6E0FF12D7BD90099FEF48
:109A9600F09000C7E0FF12D7BD9009A0EFF0227545
:109AA60036FF7537E575387A8F3C8E3B8D3A8C39A3
:109AB6007B017A1C79B51243BD8F24753A607539DE
:109AC600E37538167537007F007E367D6E7C011291
:109AD600D045E4F522F523743D2523F58274E63559
:109AE60022F583E493FF12D88C0523E52370020543
:109AF60022C39411E522940040DDE4F522F523C348
:109B0600E5239524E5229400501B74B52523F582A0
:109B1600741C3522F583E0FF12D88C0523E52370EB
:109B2600DE052280DAE4FF12D88C7F647E007D0099
:109B36007C0012BA97EF701A78007C007D017BFFDB
:109B46007AE579A2122C93EF3395E04F7F017004EA
:109B5600FF227F0122E4901BA2F0A3F0901BA2E457
:109B660075F001122849FE74A325F0F58274093EAA
:109B7600F583E070E7901BA2E0FEA3E024A3F9744E
:109B8600093EFA7B0112915A901BA4122A5C7E09A7
:109B96007F607D007B017A007900122E5A901BA40B
:109BA600E0FCA3E0FDA3E0FEA3E0FF12B64BEF70DE
:109BB6004D901BA2F0A3F0901BA2E0FEA3E0FFC312
:109BC600EE9408504574002FF58274003EF583E04C
:109BD600FF12D93A501812D921901BA2E0FEA3E039
:109BE6002400F58274003EF583E0FF12D8FE901B38
:109BF600A3E004F070C1901BA2E004F080B912D972
:109C0600217BFF7AE0798D1243C3228E2A8F2B8D1A
:109C16002C12B14B8F308E2F8D2E8C2D7F007E48CF
:109C26007D017C00AB30AA2FA92EA82DC3122A05D0
:109C36004003029CC07E007F0A7D007B017A1C796E
:109C46000C122E5AE52B2404F582E4352AF583E01E
:109C5600901C0CF0E52B2405F582E4352AF583E00B
:109C6600901C0DF0E52B2406F582E4352AF583E0F9
:109C7600901C0EF0852B82852A83A3A3A3E0901C5B
:109C86000FF0852B82852A83A3E0901C10F0852B8C
:109C960082852A83E0901C11F0A3E52CF0E4A3F062
:109CA600A3F0A3F0AF30AE2FAD2EAC2D7B017A1C06
:109CB600790CF54275430A12BFE122E4901BA2F02B
:109CC600A3F0901BA2E475F001122849FE74A325A7
:109CD600F0F58274093EF583E070E7901BA2E0FE82
:109CE600A3E024A3F974093EFA7B0112915A901B52
:109CF600A4122A5C901BA4E0FCA3E0FDA3E0FEA353
:109D0600E0FF12B6C8EF705512D9217BFF7AE179D0
:109D160076901BA4E0FCA3E0FDA3E0FEA3E0F539EA
:109D26008E388D378C361243C3E4901BA2F0A3F015
:109D3600901BA2E0FEA3E0FFC3EE9408502B740034
:109D46002FF58274003EF583E0FF12D8FE901BA328
:109D5600E004F070DB901BA2E004F080D312D9215E
:109D66007BFF7AE179881243C3228B238A248925D3
:109D7600AB23AA24A9251226FBFF12D855500D7431
:109D8600012525F525E43524F52480E4D200AB230E
:109D9600AA24A9251226FBFF642B6004EFB42D1B11
:109DA600AB230525E525AA247002052414F91226FD
:109DB600FB642D6003D38001C39200E4F526F527EA
:109DC600AB23AA24A9251226FBFF12D9495036AB8C
:109DD60023AA24A9251226FBFF3395E0FEEF24D003
:109DE600FBEE34FFFAAE26AF277C007D0A122E86E4
:109DF600EF2BF527EE3AF52674012525F525E435F2
:109E060024F52480BB300006AE26AF278009C3E4C4
:109E16009527FFE49526FE22E4901BA2F0A3F0907E
:109E26001BA2E475F001122849FE74A325F0F58201
:109E360074093EF583E070E7901BA2E0FEA3E024E0
:109E4600A3F974093EFA7B0112915A901BA4122AB7
:109E56005C7E097F607D007B017A007900122E5AB4
:109E6600E4901BA2F0A3F0A3E0FCA3E0FDA3E0FEB8
:109E7600A3E0FF12B551EF703F12D921E4901BA267
:109E8600F0A3F0900960E0FEA3E0FF901BA2E0FCC7
:109E9600A3E0FDC39FEC9E502B74002DF582740049
:109EA6003CF583E0FF12D8FE901BA3E004F070D3CC
:109EB600901BA2E004F080CB12D9217BFF7ADF79D8
:109EC600DA1243C3221285FDEF600C12D9217BFF03
:109ED6007AE1793B029F6F12CCD5EF600C12D92143
:109EE6007BFF7AE1794F029F6F78007C007D017BD2
:109EF600FF7AE17970122C93EF3395E04F60617E23
:109F0600117F947D007B017A0979A3122E5A78A3DA
:109F16007C097D017B017A0079007E097F6012262B
:109F2600D5E4901BA2F0A3F012D921901BA2E475F0
:109F3600F001122849FE74A325F0F58274093EF556
:109F460083E0602D901BA2E0FEA3E024A3F58274BB
:109F5600093EF583E0FF12D8FEE4FF12D8FE80CB5F
:109F660012D9217BFF7AE179731243C3E4FF12D839
:109F7600FE228E228F23E4FD7FAC12A855901B9DF6
:109F8600E0901BA6F044F7F0FB7A00E4FD7FAC12EC
:109F9600BA238007901BA6E030E7117D037FAC1241
:109FA600A855901B9DE0901BA6F080E8AB23AA2243
:109FB6007D287FAC12BA238007901BA6E030E714F9
:109FC60012C7D47D037FAC12A855901B9DE0901B51
:109FD600A6F080E5E5227A00FB7D297FAC12BA2344
:109FE6008007901BA6E030E71412C7D47D037FAC30
:109FF60012A855901B9DE0901BA6F080E5E4FD7F1E
:10A00600AC12A855901B9DE0901BA6F04408F0FBEF
:10A016007A00E4FD7FAC02BA2390096F122A680029
:10A0260000000090096FE0FCA3E0FDA3E0FEA3E0C2
:10A03600FF901BA2EFF090096FA3A3A3E07808128C
:10A046002A16901BA3EFF090096FE0FCA3E0FDA396
:10A05600E0FEA3E0FF7810122A16E4901BA4EFF0AE
:10A066007E1B7FA27D037C0012D41C901BA5EFF003
:10A07600901BA2E0FD7F3812D965901BA3E0FD7FFF
:10A086003912D965901BA4E0FD7F3A12D965901B61
:10A09600A5E0FD7F3B12D965901BA2E0FD7F3C1237
:10A0A600D965901BA3E0FD7F3D12D965901BA4E006
:10A0B600FD7F3E12D965901BA5E0FD7F3F02D96565
:10A0C600129937E4901BA2F0A3F012BB7FEF600C4D
:10A0D60012D9217BFF7AE079BA02A16912D9217BD4
:10A0E600FF7AE179C11243C312C5C3EF60087BFF53
:10A0F6007AE079CD806D7BFF7AE179D71243C3127E
:10A10600B3577E047F007D007B017A0D79A3122E62
:10A116005A78A37C097D017B017A0079007E047F51
:10A12600001226D57E097FA37DFE7C0312D41C90E7
:10A136000DA1EFF07B017A0979A37DFF7C0312D094
:10A14600EE900DA2EFF0E4F526F5277F907E08FD50
:10A15600FC128CE1EF7BFF70067AE179E880047AE5
:10A16600E279011243C3228B228A2389248F288E07
:10A17600278D268C2585A7297531007530C2752F48
:10A1860001752E007F007E367D6E7C0112CFCF7565
:10A19600A710C298901BA6122A6800000000AF28DC
:10A1A600AE27AD26AC25901BA6E0F8A3E0F9A3E008
:10A1B600FAA3E0FBC3122A05503B901BA6A3A3E01B
:10A1C600FEA3E0AB22AA23A924F5828E83122714CC
:10A1D600FF12D88C901BA6E0FCA3E0FDA3E0FEA333
:10A1E600E02401FFE43EFEE43DFDE43CFC901BA6BA
:10A1F600122A5C80A9C299C2988529A7901BA6E05D
:10A20600FCA3E0FDA3E0FEA3E0FF22900020E064B3
:10A21600547052A3E06441704CA3E064537046A3AB
:10A22600E0B44B41E4901BACF0A3F0901BACE0FE15
:10A23600A3E0FF2420F58274003EF583E0FD74A3BD
:10A246002FF58274093EF583EDF0901BADE004F026
:10A256007006901BACE004F0901BACE0B404CCA3F9
:10A26600E0B400C72290096CE064017040901BAC1A
:10A27600F0A3F0901BACE0FEA3E0FF245FF5827430
:10A28600E93EF583E493FD74A32FF58274093EF548
:10A2960083EDF0901BADE004F07006901BACE0047B
:10A2A600F0901BACE07004A3E0642070C6228E22FE
:10A2B6008F23753A607539E37538167537007F0058
:10A2C6007E367D6E7C0112D045E4F524F52574C5F5
:10A2D6002525F58274E73524F583E493FF12D88C9F
:10A2E6000525E52570020524C3940CE52494004059
:10A2F600DD852224852325E42523FFE5223404FE7B
:10A30600C3E5259FE5249E501B74A32525F582747D
:10A31600093524F583E0FF12D88C0525E52570D78D
:10A32600052480D37FB07E047D007C0012BA97EFAF
:10A33600701A78007C007D017BFF7AE57981122C0A
:10A3460093EF3395E04F7F017004FF227F01228E49
:10A35600268F27753A607539E37538167537007F8D
:10A36600007E367D6E7C0112D045E4F528F5297411
:10A37600E12529F58274E73528F583E493FF12D8A1
:10A386008C0529E52970020528C39413E528940055
:10A3960040DD852628852729E42527FFE526340480
:10A3A600FEC3E5299FE5289E501B74A32529F58247
:10A3B60074093528F583E0FF12D88C0529E5297044
:10A3C600D7052880D37FB07E047D007C0012BA9723
:10A3D600EF701A78007C007D017BFF7AE5798112A7
:10A3E6002C93EF3395E04F7F017004FF227F01220B
:10A3F6008E288F29753A607539E3753816753700DA
:10A406007F007E367D6E7C0112D045E4F52AF52B61
:10A4160074F4252BF58274E7352AF583E493FF124D
:10A42600D88C052BE52B7002052AC3940BE52A94DC
:10A436000040DD85282A85292BE42529FFE52834D7
:10A4460004FEC3E52B9FE52A9E501B74A3252BF51E
:10A45600827409352AF583E0FF12D88C052BE52B8B
:10A4660070D7052A80D37FB07E047D007C0012BAA7
:10A4760097EF701A78007C007D017BFF7AE5798181
:10A48600122C93EF3395E04F7F017004FF227F017A
:10A4960022E4901BA2F0A3F0901BA2E475F0011237
:10A4A6002849FE74A325F0F58274093EF583E07011
:10A4B600E7901BA2E0FEA3E024A3F974093EFA7B11
:10A4C6000112915A901BA4122A5C7E097F607D00BE
:10A4D6007B017A007900122E5A901BA4E0FCA3E0BF
:10A4E600FDA3E0FEA3E0FF12B64BEF703712D921B1
:10A4F600E4901BA2F0A3F0901BA2E0FEA3E0FFC332
:10A50600EE9404502B74002FF58274003EF583E020
:10A51600FF12D8FE901BA3E004F070DB901BA2E0B4
:10A5260004F080D312D9217BFF7AE0798D1243C3E0
:10A5360022E4901BA2F0A3F0901BA2E475F0011296
:10A546002849FE74A325F0F58274093EF583E07070
:10A55600E7901BA2E0FEA3E024A3F974093EFA7B70
:10A566000112915A901BA4122A5C7E097F607D001D
:10A576007B017A007900122E5A901BA4E0FCA3E01E
:10A58600FDA3E0FEA3E0FF12B64BEF703712D92110
:10A59600E4901BA2F0A3F0901BA2E0FEA3E0FFC391
:10A5A600EE9404502B74002FF58274043EF583E07C
:10A5B600FF12D8FE901BA3E004F070DB901BA2E014
:10A5C60004F080D312D9217BFF7AE0798D1243C340
:10A5D60022E4901BA2F0A3F0901BA2E475F00112F6
:10A5E6002849FE74A325F0F58274093EF583E070D0
:10A5F600E77B017A0979A3901BA2E0FEA3E0FFE4C2
:10A60600FCFD12A16D7B017A0979A37F947E117DF1
:10A61600007C0012DA407E00901BA2EEF0A3EFF061
:10A62600603D12D921E4901BA4F0A3F0901BA2E098
:10A63600FEA3E0FFA3E0FCA3E0FDC39FEC9E502237
:10A6460074A32DF58274093CF583E0FF12D8FE90C1
:10A656001BA5E004F070D5901BA4E004F080CD1299
:10A66600D87A7E117F947D007B017A0979A3022E28
:10A676005AE4901BA2F0A3F0901BA2E475F001121D
:10A686002849FE74A325F0F58274093EF583E0702F
:10A69600E77B017A0979A3901BA2E0FEA3E0FFE421
:10A6A600FCFD12A16D7B017A0979A37F947E117D51
:10A6B600007C0012DA407E00901BA2EEF0A3EFF0C1
:10A6C600603D12D921E4901BA4F0A3F0901BA2E0F8
:10A6D600FEA3E0FFA3E0FCA3E0FDC39FEC9E502297
:10A6E60074A32DF58274093CF583E0FF12D8FE9021
:10A6F6001BA5E004F070D5901BA4E004F080CD12F9
:10A70600D87A7E117F947D007B017A0979A3022E87
:10A716005A12D921E4901BA2F0A3F0901BA2E0FEEE
:10A72600A3E0FFC3EE9404501F74A32FF582740DAB
:10A736003EF583E0FF12D8FE901BA3E004F070DB29
:10A74600901BA2E004F080D3E4FF7E08FDFC901B82
:10A75600A5E0F8A3E0F9A3E0FAA3E0FBC3122A05FB
:10A76600501CE4FF7E04FDFC901BA5E0F8A3A3A308
:10A77600E0122A054008901BA4E0FF12D8FEE490E0
:10A786001BA2F0A3F0901BA2E0FEA3E0FFC3EE9491
:10A7960004501C74A32FF582740D3EF583E4F090EB
:10A7A6001BA3E004F070DE901BA2E004F080D6222A
:10A7B60012D921E4901BA2F0A3F0901BA2E0FEA305
:10A7C600E0FFC3EE9404501F74A32FF58274113E6C
:10A7D600F583E0FF12D8FE901BA3E004F070DB9037
:10A7E6001BA2E004F080D3E4FF7E0CFDFC901BA4CA
:10A7F600E0F8A3E0F9A3E0FAA3E0FBC3122A0550B0
:10A806001CE4FF7E08FDFC901BA4E0F8A3A3A3E0D4
:10A81600122A054008901BA8E0FF12D8FEE4901B00
:10A82600A2F0A3F0901BA2E0FEA3E0FFC3EE940407
:10A83600501C74A32FF58274113EF583E4F0901B2F
:10A84600A3E004F070DE901BA2E004F080D6228F15
:10A856002C8D2D85A72E75A710E52C64AC703B12A8
:10A86600D82FE4FDAF2C12CE49EF7010AF2D12D5C4
:10A8760037EF700512D7D380067F01227F0122129F
:10A88600D82F7D01AF2C12CE49EF700B12D5109048
:10A896001B9D12D7CC80037F0122E52C6480704675
:10A8A60012D82FE4FDAF2C12CE49EF7010AF2D1247
:10A8B600D537EF700512D7CE80067F01227F0122A1
:10A8C60012D82F7D01AF2C12CE49EF701612D5107B
:10A8D600901B9DEFF0E4FF12D5D112D510A312D72D
:10A8E600CC80037F0122852EA77F00227B017A1C64
:10A8F60079167E1C7F227D407C008E3F8F408C41E6
:10A906008D428B438A448945AA06A9077B0112D743
:10A91600A38E468F47E4F548F549C3E5479542E5DA
:10A926004695415061AB43AA44A94585498285486D
:10A9360083122714FF3395E04F603DE5472401FF5E
:10A94600E43546FEC3EF9542EE9541502B0549E5A9
:10A9560049AE487002054814F5828E83122714FF0B
:10A966000547E547AC4670020546142540F582E5E5
:10A976003F3CF583EFF080ADE5402547F582E53FA6
:10A986003546F583E4F022E4901BA2F0A3F0901B79
:10A99600A2E475F001122849FE74A325F0F582742D
:10A9A600093EF583E070E7901BA2E0FEA3E024A336
:10A9B600F974093EFA7B0112915A901BA4122A5C83
:10A9C600901BA4E0FCA3E0FDA3E0FEA3E0FF12B50C
:10A9D600CEEF703F12D921E4901BA2F0A3F09009AC
:10A9E60060E0FEA3E0FF901BA2E0FCA3E0FDC39F96
:10A9F600EC9E502B74002DF58274003CF583E0FF2D
:10AA060012D8FE901BA3E004F070D3901BA2E004C2
:10AA1600F080CB12D9217BFF7AE0792E1243C32234
:10AA26008D828C83E0FB8F828E83E06B600302AAAB
:10AA3600B88D828C83A3E0FB8F828E83A3E06B703C
:10AA4600718D828C83A3A3E0FB8F828E83A3A3E008
:10AA56006B705F8D828C83A3A3A3E0FB8F828E83B2
:10AA6600A3A3A3E06B704BED2404F582E43CF583CD
:10AA7600E0FBEF2404F582E43EF583E06B7033EDF2
:10AA86002405F582E43CF583E0FBEF2405F582E43A
:10AA96003EF583E0B5031BED2406F582E43CF58321
:10AAA600E0FDEF2406F582E43EF583E0B505037F7D
:10AAB60001227F002212DA0C787FE4F6D8FD758138
:10AAC6006D12D70002AB0802D9FDE493A3F8E49314
:10AAD600A34003F68001F208DFF48029E493A3F88B
:10AAE6005407240CC8C333C4540F4420C8834004FD
:10AAF600F456800146F6DFE4800B010204081020BC
:10AB0600408090C61EE47E019360BCA3FF543F3094
:10AB1600E509541FFEE493A360010ECF54C025E05F
:10AB260060A840B8E493A3FAE493A3F8E493A3C817
:10AB3600C582C8CAC583CAF0A3C8C582C8CAC583A8
:10AB4600CADFE9DEE780BEE4FD7FAC12A855901BA4
:10AB56009DE0901BA8F044F7F0FB7A00E4FD7FAC83
:10AB660012BA238007901BA8E030E7117D037FAC63
:10AB760012A855901B9DE0901BA8F080E87D287FC9
:10AB8600AC12A855901B9DE0901BA8F07D297FACC8
:10AB960012A855901B9DE0FF901BA4E4F0A3EFF0D4
:10ABA600E0FE901BA8E07C002400FFEC3E901BA674
:10ABB600F0A3EFF0E4FD7FAC12A855901B9DE0904A
:10ABC6001BA8F04408F0FB7A00E4FD7FAC12BA2320
:10ABD600901BA6E0FEA3E0FF22E517700302AC6F10
:10ABE600E4F517901CE5E004F0E0D3941E7480941D
:10ABF600804002E4F0901CE5E0FFC31390E9EC937B
:10AC060024FF9297E514640170057F1312BB0B7540
:10AC160025017526097527647B017A1B79371296FB
:10AC2600FF90096AE0D3940674809480403BE4F078
:10AC3600900966E06402603112D734900966E064D8
:10AC460001700F12D46F9009687407F09009677449
:10AC560009F0900966E06403700F12D46F900968DA
:10AC66007401F09009677409F022E4901BA2F0A326
:10AC7600F0901BA2E475F001122849FE74A325F09A
:10AC8600F58274093EF583E070E7901BA2E0FEA30F
:10AC9600E024A3F974093EFA7B0112915A901BA491
:10ACA600122A5C7E097F607D007B017A00790012A2
:10ACB6002E5A901BA4E0FCA3E0FDA3E0FEA3E0FF58
:10ACC60012B64B12D921E4901BA2F0A3F0901BA25E
:10ACD600E0FEA3E0FFC3EE9408501F74002FF58238
:10ACE60074003EF583E0FF12D8FE901BA3E004F04B
:10ACF60070DB901BA2E004F080D322E4901BA2F04C
:10AD0600A3F0901BA2E475F001122849FE74A32556
:10AD1600F0F58274093EF583E070E7901BA2E0FE31
:10AD2600A3E024A3F974093EFA7B01129D70901BDF
:10AD3600A4EEF0A3EFF012C1F7EF703F12D921E4B1
:10AD4600901BA2F0A3F0900960E0FEA3E0FF901B29
:10AD5600A2E0FCA3E0FDC39FEC9E502B74002DF5F2
:10AD66008274003CF583E0FF12D8FE901BA3E0043A
:10AD7600F070D3901BA2E004F080CB12D9217BFFA8
:10AD86007AE079081243C322E4901BA2F0A3F09064
:10AD96001BA2E475F001122849FE74A325F0F58282
:10ADA60074093EF583E070E7901BA2E0FEA3E02461
:10ADB600A3F974093EFA7B01129D70901BA4EEF074
:10ADC600A3EFF07B017A0979A312745312D921E417
:10ADD600901BA2F0A3F0901BA2E0FCA3E0FDC3EC45
:10ADE60094045030901BA5E07F0025E025E0FEEF9F
:10ADF6002DFFEC3EFE74A32FF58274093EF583E029
:10AE0600FF12D8FE901BA3E004F070CA901BA2E0CC
:10AE160004F080C222E4901BA2F0A3F0901BA2E4EF
:10AE260075F001122849FE74A325F0F58274093ED7
:10AE3600F583E070E7901BA2E475F001122849FE45
:10AE460074A325F0F58274093EF583E070E7901B44
:10AE5600A2E475F001122849FE74A325F0F5827468
:10AE6600093EF583E070E7901BA2E475F001122815
:10AE760049FE74A325F0F58274093EF583E070E778
:10AE8600901BA2E0FEA3E024A3F974093EFA7B011D
:10AE9600129D70901BA4EEF0A3EFF0129F7802D8DB
:10AEA600688E228F238C248D257E097F607D007B12
:10AEB600017A007900122E5A753AE0753993753881
:10AEC600047537007F007E367D6E7C0112D045E426
:10AED600F526F527C3E5279525E5269524501BE598
:10AEE600232527F582E5223526F583E0FF12D88C47
:10AEF6000527E52770DE052680DA7F327E007D0095
:10AF06007C0012BA97EF7020F526F5270527E5276E
:10AF1600AE2670020526142400F58274003EF583E1
:10AF2600E070E9AE26AF2722E4FEFF228E288F29A5
:10AF36008C2A8D2B7D0E7FAC12A85512D7B8852989
:10AF460082852883EFF0901B9DE0852B82852A83DE
:10AF5600F07D0D7FAC12A85512D7B88529828528B9
:10AF660083A3EFF0901B9DE0852B82852A83A3F0B7
:10AF76007D0B7FAC12A85512D7B885298285288308
:10AF8600A3A3A3EFF0901B9DE0852B82852A83A3C4
:10AF9600A3A3F07D0C7FAC12A85512D7B8852982E1
:10AFA600852883A3A3EFF0901B9DE0852B82852A3D
:10AFB60083A3A3F07F00228E288F298C2A8D2B7DD8
:10AFC6000A7FAC12A85512D7B8E5292404F582E405
:10AFD6003528F583EFF0901B9DE0FFE52B2404F563
:10AFE60082E4352AF583EFF07D097FAC12A855126D
:10AFF600D7B8E5292405F582E43528F583EFF090E6
:10B006001B9DE0FFE52B2405F582E4352AF583EF49
:10B01600F07D087FAC12A85512D7B8E5292406F5AD
:10B0260082E43528F583EFF0901B9DE0FFE52B24A5
:10B0360006F582E4352AF583EFF07F00221299EEB9
:10B0460012DA4312DA3A8F118E108D0F8C0E12C05F
:10B056004D8F22EF64027050FFFEFDFCAB11AA106B
:10B06600A90FA80EC3122A05700A12D46F90096898
:10B0760074038021900966E0640160217F0112D784
:10B086006112DA437D03AF16AE15129C11124C0CF9
:10B096009009687405F09009677409F0227D22AF63
:10B0A60016AE15129C118006E52264037003023E5B
:10B0B600E19009687403F09009677409F012D46F7F
:10B0C60022754200754140754001753F00753E008E
:10B0D600753D30753C01753B007F007E407D017CEF
:10B0E60000AB3EAA3DA93CA83BC3122A05504DAF72
:10B0F6003EAE3DAD3CAC3B7B017A1B79D7754A0031
:10B10600754B0312BF06901BD7E0F47018A3E0F44A
:10B116007013A3E0F4700E853E42853D41853C40A8
:10B12600853B3F8017E53E2440F53EE4353DF53D41
:10B13600E4353CF53CE4353BF53B809DAF42AE4102
:10B14600AD40AC3F22753800753740753601753510
:10B15600007534007533407532017531007F007E0D
:10B16600487D017C00AB34AA33A932A831C3122A28
:10B1760005504DAF34AE33AD32AC317B017A1B791D
:10B18600D6754A00754B0312BF06901BD6E0F470C5
:10B1960018A3E0F47013A3E0F4700E8534388533F9
:10B1A600378532368531358017E534240AF534E49F
:10B1B6003533F533E43532F532E43531F531809DFA
:10B1C600AF38AE37AD36AC352275350075344075BF
:10B1D6003301753200753100753048752F01752EB3
:10B1E600007F007E507D017C00AB31AA30A92FA8DC
:10B1F6002EC3122A05504DAF31AE30AD2FAC2E7B8B
:10B20600017A1B79A2754A00754B0312BF06901B83
:10B21600A2E0F47018A3E0F47013A3E0F4700E85B6
:10B226003135853034852F33852E328017E531242C
:10B236000AF531E43530F530E4352FF52FE4352EB7
:10B24600F52E809DAF35AE34AD33AC322212DA43E3
:10B256007536FF7537E275383B900978E075390029
:10B26600F53AA3E0753B00F53C90097BE0753D009F
:10B27600F53EA3E0753F00F540A3E0754100F542B9
:10B28600A3E0754300F5447B017A0979A31243BD17
:10B29600901BA212D91CE4901BA4F0A3F0901BA251
:10B2A600E0FEA3E0FFA3E0FCA3E0FDC39FEC9E50FD
:10B2B6001F74A32DF58274093CF583E0FF12D8FEB6
:10B2C600901BA5E004F070D5901BA4E004F080CD9F
:10B2D600227E097F607D007B017A007900122E5A5A
:10B2E600753A607539E37538167537007F007E3616
:10B2F6007D6E7C0112D045E4F522F523744E25239C
:10B30600F58274E63522F583E493FF12D88C052383
:10B31600E52370020522C3940FE522940040DD7FE9
:10B32600647E007D007C0012BA97EF7020F522F54E
:10B33600230523E523AE2270020522142400F5829C
:10B3460074003EF583E070E9AE22AF2322E4FEFFEF
:10B35600229000317401F0901B93E0900025F0904C
:10B366001B94E0900026F0901B95E0900027F0904B
:10B376001B96E0900028F0901B97E0900029F09033
:10B386001B98E090002AF0901B99E090002BF0901B
:10B396001B9AE090002CF0900991E09000DCF09070
:10B3A6000992E09000DDF0900993E09000DEF090C5
:10B3B6000994E09000DFF0900995E09000E0F090AD
:10B3C6000996E09000E1F0900997E09000E2F02203
:10B3D600E48F2C8E2BF52AF529900968E06401701C
:10B3E6002CAD2AAC297B37FAF9F81228C48F2C8E9B
:10B3F6002B8D2A8C29E47BE87A03F9F81228C48F6E
:10B406002C8E2B8D2A8C29E4FB7A0C8030AF2CAE47
:10B416002BAD2AAC29E47B37FAF9F81228C48F2C15
:10B426008E2B8D2A8C29E47BE87A03F9F81228C43E
:10B436008F2C8E2B8D2A8C29E47B997A09F9F812A8
:10B44600294F8F2C8E2B8D2A8C29AE2BAF2C22E4E4
:10B45600901BA2F0A3F012CB59EF704412D921E44D
:10B46600901BA2F0A3F0900960E0FEA3E0FF901B02
:10B47600A2E0FCA3E0FDC39FEC9E501F74002DF5D7
:10B486008274003CF583E0FF12D8FE901BA3E00413
:10B49600F070D3901BA2E004F080CBE4FF02D8FE4C
:10B4A60012D921E4901BA2F0A3F0E4FF12D8FE907B
:10B4B6001BA3E004F07006901BA2E004F0C3901BEF
:10B4C600A3E09410901BA2E0940040DE22E4901BBF
:10B4D600A2F0A3F012CBA6EF704412D921E4901B80
:10B4E600A2F0A3F0900960E0FEA3E0FF901BA2E0AB
:10B4F600FCA3E0FDC39FEC9E501F74002DF58274E3
:10B50600003CF583E0FF12D8FE901BA3E004F07028
:10B51600D3901BA2E004F080CBE4FF02D8FE12D940
:10B5260021E4901BA2F0A3F0E4FF12D8FE901BA327
:10B53600E004F07006901BA2E004F0C3901BA3E0A9
:10B546009410901BA2E0940040DE227536FF7537FA
:10B55600E575387A8F3C8E3B8D3A8C397B017A1CA7
:10B5660079B51243BD8F23753A607539E375381680
:10B576007537007F007E367D6E7C0112D045E4F57E
:10B5860022C3E522940C74809480500EE52290E646
:10B59600CB93FF12D88C052280E7E4F522E522C37F
:10B5A6009523501474B52522F582E4341CF583E006
:10B5B600FF12D88C052280E5E4FF12D88C7FC87E66
:10B5C600007D007C0002BA977536FF7537E5753841
:10B5D6007A8F3C8E3B8D3A8C397B017A1C79B51279
:10B5E60043BD8F23753A607539E375381675370094
:10B5F6007F007E367D6E7C0112D045E4F522C3E5E0
:10B6060022941074809480500EE52290E70F93FFE9
:10B6160012D88C052280E7E4F522E522C395235053
:10B626001474B52522F582E4341CF583E0FF12D8A4
:10B636008C052280E5E4FF12D88C7F807EEE7DFFAC
:10B646007CFF02BA977536FF7537E575387A8F3CF9
:10B656008E3B8D3A8C397B017A1C79B51243BD8FAE
:10B6660024753A607539E37538167537007F007EA4
:10B67600367D6E7C0112D045E4F523C3E52394099B
:10B6860074809480500EE52390E72693FF12D88CA1
:10B69600052380E7E4F523E523C39524501474B508
:10B6A6002523F582E4341CF583E0FF12D88C0523AC
:10B6B60080E5E4FF12D88C7FC87E007D007C000206
:10B6C600BA977536FF7537E575387A8F3C8E3B8DA0
:10B6D6003A8C397B017A1C79B51243BD8F23753AB2
:10B6E600607539E37538167537007F007E367D6ED6
:10B6F6007C0112D045E4F522C3E5229410748094AF
:10B7060080500EE52290E62D93FF12D88C052280FC
:10B71600E7E4F522E522C39523501474B52522F5F6
:10B7260082E4341CF583E0FF12D88C052280E5E420
:10B73600FF12D88C7FC87E007D007C0002BA9790ED
:10B746000967E0640160337401F012D1F012D9A4E4
:10B756001220267FB07E717D0B7C0012C7277F01E9
:10B766001220967F011220067F0112D76112AB4D7F
:10B77600900964EEF0A3EFF0D297E5176006E4F5C2
:10B7860017128F97125EAEEF700C12D9CF122E9849
:10B7960012D9D912729C7525017526097527647B05
:10B7A600017A1B79371296FF90096AE0D3940274E6
:10B7B6008094804005E4F012CF5022900967E0643F
:10B7C6000360037403F0E517606CE4F517901CE45E
:10B7D600E004F0E0D3941E748094804002E4F0907C
:10B7E6001CE4E0FFC31390E9DC9324FF92977525D0
:10B7F600017526097527647B017A1B79371296FF36
:10B8060090096AE0D39406748094804029E4F0900D
:10B816000966E06402601FA37409F0900966E0649B
:10B826000170069009687407F0900966E064037079
:10B836000590096804F0227F3812D958901B93EFBF
:10B84600F07F3912D958901B94EFF07F3A12D958ED
:10B85600901B95EFF07F3B12D958901B96EFF07F27
:10B866003C12D958901B97EFF07F3D12D958901B88
:10B8760098EFF07F3E12D958901B99EFF07F3F1258
:10B88600D958901B9AEFF07E1B7F937D047C0012A3
:10B89600D41C8F227E1B7F977D047C0012D41CE56E
:10B8A6002270028003EF7003FF8003E47F01FEFD38
:10B8B600FC228B228A2389248F288E278D268C258D
:10B8C600E4F529F52A12D66BE47F04FEFDFCAB28CD
:10B8D600AA27A926A8251228C4AB69AA68A967A819
:10B8E60066C3122A055006E565456460DBE47F08F9
:10B8F600FEFDFCAB69AA68A967A866C3122A0540C3
:10B90600EC53E7F7900960E564F0A3E565F0AE68EF
:10B91600AF69A3EEF0A3EFF0D3900961E094009035
:10B926000960E094007F0140027F0022E4901BA2A0
:10B93600F0A3F0901BA2E475F001122849FE74A34F
:10B9460025F0F58274093EF583E070E7901BA2E0CE
:10B95600FEA3E024A3F974093EFA7B0112915A90E2
:10B966001BA4122A5C901BA4E0FCA3E0FDA3E0FE4E
:10B97600A3E0FF129AA5EF702012D9217BFF7AE18E
:10B986007912901BA4E0FCA3E0FDA3E0FEA3E0F582
:10B99600398E388D378C36800912D9217BFF7AE1B2
:10B9A600792E1243C3227E097F607D007B017A00D7
:10B9B6007900122E5A12C50DEF7055901BA2F0A3F6
:10B9C600F0901BA2E0FEA3E0FFC3EE94085039748A
:10B9D600002FF58274003EF583E0FF12D93A501825
:10B9E60012D921901BA2E0FEA3E02400F582740088
:10B9F6003EF583E0FF12D8FE901BA3E004F070C171
:10BA0600901BA2E004F080B97BFF7ADF79458009BC
:10BA160012D9217BFF7AE079681243C3228F268DE3
:10BA2600278A288B2985A72A75A710E52664AC7076
:10BA36002412CE42EF701BAF2712D537EF7010AF2E
:10BA46002912D537EF700512D7D380097F01227FDF
:10BA560001227F0122E5266480703012CE42EF700B
:10BA660027AF2712D537EF701CE528FF12D537EF21
:10BA76007010AF2912D537EF700512D7D3800C7F1F
:10BA860001227F01227F01227F0122852AA77F00D2
:10BA9600228F368E358D348C33E4F537F53812D651
:10BAA6006BE47F04FEFDFCAB36AA35A934A833123D
:10BAB60028C4AB69AA68A967A866C3122A055006F6
:10BAC600E565456460DBE47F08FEFDFCAB69AA68BA
:10BAD600A967A866C3122A0540EC53E7F7900960E8
:10BAE600E564F0A3E565F0AE68AF69A3EEF0A3EFF9
:10BAF600F0D3900961E09400900960E094007F0122
:10BB060040027F00228F22E4F51412D1F012202683
:10BB160012D9A47F011220067F0112D76112D734F1
:10BB260012C50DEF7002803C7F2C7E0112D22212CC
:10BB3600C50DEF7002802D7F2C7E0112D22212C518
:10BB46000DEF7002801E7D12AF16AE15129C117B92
:10BB5600017A00790012D5A7EF700E7D1CAF16AEE4
:10BB660015129C11AF2202D31212D46F9009687479
:10BB760003F09009677409F022753A607539E37528
:10BB860038167537007F007E367D6E7C0112D045F3
:10BB9600E4F527C3E527940C74809480500EE527BE
:10BBA60090E60E93FF12D88C052780E77F887E13D8
:10BBB6007D007C0012BA97EF702EC3900961E09465
:10BBC60002900960E09400401C78007C007D017BB7
:10BBD600FF7AE579817E007F02122E36EF3395E0FB
:10BBE6004F7002FF227F01227F0122753A6075396C
:10BBF600E37538167537007F007E367D6E7C011240
:10BC0600D045E4F522C3E522940374809480500E57
:10BC1600E52290E6E293FF12D88C052280E77F0AA0
:10BC26007E007D007C0012BA97EF702EC3900961EA
:10BC3600E09402900960E09400401C78007C007D4E
:10BC4600017BFF7AE579817E007F02122E36EF3383
:10BC560095E04F7002FF227F01227F0122753A6034
:10BC66007539E37538167537007F007E367D6E7C34
:10BC76000112D045E4F522C3E5229409748094802C
:10BC8600500EE52290E5A593FF12D88C052280E799
:10BC96007F0A7E007D007C0012BA97EF702EC3905B
:10BCA6000961E09402900960E09400401C78007CF1
:10BCB600007D017BFF7AE579817E007F02122E36B8
:10BCC600EF3395E04F7002FF227F01227F01229021
:10BCD6000991E09009AFF0900992E09009B0F090D8
:10BCE6000993E09009B1F0900994E09009B2F090C0
:10BCF6000995E09009B3F0900996E09009B4F090A8
:10BD06000997E09009B5F012D921E4901BA2F0A39F
:10BD1600F0901BA2E0FEA3E0FFC39413EE94005044
:10BD26001F74A32FF58274093EF583E0FF12D8FE37
:10BD3600901BA3E004F070D9901BA2E004F080D120
:10BD46002212D921E4901BA2F0A3F0901BA2E0FEE0
:10BD5600A3E0FFC3EE9404501F74A32FF58274155D
:10BD66003EF583E0FF12D8FE901BA3E004F070DBE3
:10BD7600901BA2E004F080D3901BA4E0FF12D8FE33
:10BD8600E4901BA2F0A3F0901BA2E0FEA3E0FFC389
:10BD9600EE9404501C74A32FF58274153EF583E4CB
:10BDA600F0901BA3E004F070DE901BA2E004F0808C
:10BDB600D622E4901BA2F0A3F012D9A41220267F6B
:10BDC600011220067FE87E0312D222C29712C451C6
:10BDD600EF7002800E12C451EF7002800612C45139
:10BDE600EF700D7F0112D74B12D98CC2AF75A70F1A
:10BDF600E4901BA2F0A3F0901BA2E0FEA3E0FFE4F8
:10BE0600FCFD7B407A9CF9F8D31229EF4010901B79
:10BE1600A3E004F070E1901BA2E004F080D9B29791
:10BE260080CEE4901BA2F0A3F012CB0CEF705590DD
:10BE36001BA2F0A3F0901BA2E0FEA3E0FFC3EE94CA
:10BE460004503974002FF58274003EF583E0FF122A
:10BE5600D93A501812D921901BA2E0FEA3E0240083
:10BE6600F58274003EF583E0FF12D8FE901BA3E036
:10BE760004F070C1901BA2E004F080B97BFF7ADF6A
:10BE86007945800912D9217BFF7ADF79481243C3AD
:10BE9600227E097F607D007B017A007900122E5A8E
:10BEA60012CA1DEF704D901BA2F0A3F0901BA2E0EA
:10BEB600FEA3E0FFC3EE9408504574002FF582748C
:10BEC600003EF583E0FF12D93A501812D921901B93
:10BED600A2E0FEA3E02400F58274003EF583E0FFB5
:10BEE60012D8FE901BA3E004F070C1901BA2E004E0
:10BEF600F080B912D9217BFF7AE079681243C32218
:10BF06008F468E458D448C438B478A4889498F4F8F
:10BF16008E4E8D4D8C4CE54B2546FFE54A3545FE4C
:10BF2600E43544FDE43543FCAB4FAA4EA94DA84C7D
:10BF3600C3122A055037AF4FAE4EAD4DAC4C1297DB
:10BF4600C1AB47AA48A949EF12277474012549F5E0
:10BF560049E43548F548E54F2401F54FE4354EF5FB
:10BF66004EE4354DF54DE4354CF54C80A9228E2234
:10BF76008F23753A607539E37538167537007F007B
:10BF86007E367D6E7C0112D045E4F524C3E524940B
:10BF96001174809480500EE52490E77893FF12D8B0
:10BFA6008C052480E7AF2312D88CE522FF12D88CAB
:10BFB6007F007E537D077C0012BA97EF701A7800D7
:10BFC6007C007D017BFF7AE57981122C93EF339516
:10BFD600E04F7F017004FF227F01228F3E8E3D8D50
:10BFE6003C8C3B8B3F8A4089418F478E468D458CE2
:10BFF60044E543253EFFE542353DFEE4353CFDE4A0
:10C00600353BFCAB47AA46A945A844C3122A0550AE
:10C0160035AF47AE46AD45AC44AB3F0541E541AA19
:10C02600407002054014F91226FBF54C128708E50C
:10C03600472401F547E43546F546E43545F545E43C
:10C046003544F54480AB2275260175270975287895
:10C056007B017A097988128B0BEF3395E0C36480F4
:10C0660094807F0050027F01AD0775260175270970
:10C076007528787B017A09799A128B0BEF3395E054
:10C08600C3648094807F0050027F01EDFB7A0070CC
:10C0960006EF70037F0122EB64014A7006EF70031E
:10C0A6007F0222ED64017008EF640170037F0322B2
:10C0B6007F002212C50DEF7002801EE4FF122006DB
:10C0C6007FE87E0312D2227F011220067FE87E03DC
:10C0D60012D22212C50DEF70061299EEE4800D7F82
:10C0E6002C7E0112D22212D158EF7018FDAF16AE77
:10C0F60015129C1112D46F9009687402F0900967AA
:10C106007409F0229009687403F07D18AF16AE1515
:10C11600129C119009677409F012D46F227D19AF31
:10C1260016AE15129C1112D777EF603912C50DEFB6
:10C13600700280157F2C7E0112D22212C50DEF707F
:10C1460002800612D158EF700302B0437D18AF1675
:10C15600AE15129C1112D46F9009687403F0900901
:10C16600677409F0227D1BAF16AE15129C1190095B
:10C17600687403F07D18AF16AE15129C119009670E
:10C186007409F012D46F227FFE7EFF7D007C0012C0
:10C1960097C1EF901BA2F0A3E4F07FFF7EFFFDFCAA
:10C1A6001297C1901BA3E02FF0901BA2E03400F081
:10C1B600A3E004F07006901BA2E004F07FFE7EFF71
:10C1C6007D007C0012880E901BA2E0F54C7FFE7E5F
:10C1D600FF7D007C00128708901BA2A3E0F54C7F30
:10C1E600FF7EFF7D007C00128708E4F5A775EF103F
:10C1F600228E228F237536FF7537E575387E8522A8
:10C206003985233A7B017A1C79B51243BD8F257592
:10C216003A607539E37538167537007F007E367DCE
:10C226006E7C0112D045E4F524C3E524940B74809A
:10C236009480500EE52490E6D793FF12D88C0524FF
:10C2460080E7AF2312D88CE522FF12D88C7FC87EF8
:10C25600007D007C0002BA97900991E08F828E8360
:10C26600F0900992E08F828E83A3F0900993E08F7D
:10C27600828E83A3A3F0900994E08F828E83A3A37A
:10C28600A3F0900995E0FDEF2404F582E43EF583E2
:10C29600EDF0900996E0FDEF2405F582E43EF58386
:10C2A600EDF0900997E0FDEF2406F582E43EF58374
:10C2B600EDF0EF2407F582E43EF583E4F02285A74E
:10C2C6002CE4F5A78FBBD2ECFF20ED0DEFC39464F1
:10C2D6007480948050030F80F0C2EDC3EF946474B1
:10C2E6008094804006AC2DAD2E8030AFBDAEBEE44E
:10C2F6008F328E31F530F52F7F307E11FDFCAB325B
:10C30600AA31A930A82F1228C4E47BFF7A0FF9F8C6
:10C3160012294FAC06AD078C2D8D2E852CA7AF05A7
:10C32600AE0422753A607539E37538167537007FA5
:10C33600007E367D6E7C0112D045E4F527C3E527E5
:10C34600941274809480500EE52790E78993FF122B
:10C35600D88C052780E7E4FF12D88C7F887E137D72
:10C36600007C0012BA97EF701A78007C007D017B82
:10C37600FF7AE57981122C93EF3395E04F7F0170B8
:10C3860004FF227F0122E4B51D14E51CB4080FAF9B
:10C3960011AE10AD0FAC0EE4F52EF52F8032AF11B5
:10C3A600AE10AD0FAC0EE4F52EF52F128912E51185
:10C3B6002401F511E43510F510E4350FF50FE435D9
:10C3C6000EF50EAF11AE10AD0FFC752E08752F00D1
:10C3D600128912E5112401F511E43510F510E43542
:10C3E6000FF50FE4350EF50E22AB07AA06901B4794
:10C3F600A3A3A3E08B828A83F0901B47E0FCA3E013
:10C40600FDA3E0FEA3E0FF7808122A168B828A833A
:10C41600A3EFF0901B47E0FCA3E0FDA3E0FEA3E042
:10C42600FF7810122A168B828A83A3A3EFF0901B43
:10C4360047E0FCA3E0FDA3E0FEA3E0FF7818122A84
:10C44600168B828A83A3A3A3EFF022753A6075390F
:10C45600E37538167537007F007E367D6E7C0112D7
:10C46600D045E4F522C3E522940B74809480500EE7
:10C47600E52290E79B93FF12D88C052280E77F6424
:10C486007E007D007C0012BA97EF701A78007C005F
:10C496007D017BFF7AE57981122C93EF3395E04F8E
:10C4A6007F017004FF227F01228D26E5266402703B
:10C4B6001A1226FB901BA7F0900001122714901B5E
:10C4C600A6F0E0FEA3E0FFE4FCFD22E5266404708E
:10C4D600271226FB901BA9F0900001122714901B2F
:10C4E600A8F0900002122714901BA7F090000312E8
:10C4F6002714901BA6F08003901BA6E0FCA3E0FD8A
:10C50600A3E0FEA3E0FF22753A607539E37538169D
:10C516007537007F007E367D6E7C0112D045E4F5CE
:10C526002AF52B74A6252BF58274E7352AF583E4C4
:10C5360093FF12D88C052BE52B7002052AC3940CA9
:10C54600E52A940040DD7F887E137D007C0012BAC8
:10C5560097EF700B7E007F007DFF7C0302D41C7F6B
:10C566000122753A607539E37538167537007F0014
:10C576007E367D6E7C0112D045E4F526F52774B231
:10C586002527F58274E73526F583E493FF12D88CC8
:10C596000527E52770020526C39413E52694004077
:10C5A600DD7F887E137D007C0012BA97EF700B7ECC
:10C5B600007F007DFF7C0302D41C7F0122753A6058
:10C5C6007539E37538167537007F007E367D6E7CCB
:10C5D6000112D045E4F523F52474F62524F582747A
:10C5E600E53523F583E493FF12D88C0524E5247002
:10C5F600020523C3940BE523940040DD7F887E1358
:10C606007D007C0012BA97EF700B7E007F007DFFE5
:10C616007C0302D41C7F01220163000162000258E0
:10C626000000025A0000025C0000015E00441CC4C7
:10C6360000000E10441CC800000E10441CCC000064
:10C646000E10441CD000000E10441CD400000E1026
:10C65600441CD800000708411CDC00411CDD0041D9
:10C666001CE000421CE1000002150978021809913D
:10C67600008E328F338C348D35E4F569F568F567B5
:10C68600F566AF03AE02900985E0FCA3E0FD12D685
:10C696007BAE32AF33E4FCFDAB69AA68A967A86636
:10C6A600C3122A055006E565456460E5AE34AF352C
:10C6B600E4FCFDAB69AA68A967A866C3122A05400F
:10C6C600EB53E7F7AE64AF6522E4901BA2F0A3F04C
:10C6D60012B2D7901BA4EEF0A3EFF04E603F12D932
:10C6E60021E4901BA2F0A3F0901BA4E0FEA3E0FFC0
:10C6F600901BA2E0FCA3E0FDC39FEC9E50227400B9
:10C706002DF58274003CF583E0FF12D8FE901BA342
:10C71600E004F070D3901BA2E004F080CB12D87A2C
:10C726002285A722E4F5A775981075A70F122ADBB4
:10C73600C76F00002580C7670001C200C762000BF3
:10C7460071B0C75D000F4240C7580016E360000095
:10C75600C77575ACF8800D75ACF4800875ACF080C3
:10C766000375AC9875ADFF800675AC1E75ADFB758F
:10C77600AB43D2AC8522A722C0E0C083C082C0D022
:10C7860075D000C00630983BC298C3E565956DE547
:10C7960064956C502B856B82856A830565E565AE6D
:10C7A6006470020564142582F582E5833EF583E50F
:10C7B60099F07569007568007567007566008003F5
:10C7C60053E7F7D006D0D0D082D083D0E0327F0AAC
:10C7D6007E007D007C008F278E268D258C24E4F537
:10C7E6002BF52AF529F528AF27AE26AD25AC24ABC7
:10C7F6002BAA2AA929A828C3122A055025E4FFFE38
:10C806000FBF00010EBE04F8BF38F5E52B2401F575
:10C816002BE4352AF52AE43529F529E43528F528C7
:10C8260080C5227E097F607D007B017A0079001237
:10C836002E5A753AE07539937538047537007F00BE
:10C846007E367D6E7C0112D0457F3112D88C7F32C8
:10C856007E007D007C0012BA97EF7017FFFE0FEF87
:10C86600AC0670010E142400F58274003CF583E0DA
:10C8760070EC22E4FEFF227E097F607D007B017A58
:10C88600007900122E5A753AE07539937538047599
:10C8960037007F007E367D6E7C0112D0457F3212D6
:10C8A600D88C7F327E007D007C0012BA97EF70171D
:10C8B600FFFE0FEFAC0670010E142400F582740023
:10C8C6003CF583E070EC22E4FEFF22E4901BA2F02C
:10C8D600A3F0901BA2E475F001122849FE74A3256B
:10C8E600F0F58274093EF583E070E712D921901BBA
:10C8F600A2E0FEA3E024A3F58274093EF583E0607E
:10C906001D901BA2E475F001122849FE74A325F0C0
:10C91600F58274093EF583E0FF12D8FE80D022E44A
:10C92600901BA2F0A3F0901BA2E475F00112284917
:10C93600FE74A325F0F58274093EF583E070E712D4
:10C94600D921901BA2E0FEA3E024A3F58274093E40
:10C95600F583E0601D901BA2E475F001122849FEE4
:10C9660074A325F0F58274093EF583E0FF12D8FE24
:10C9760080D0228B298A2A892BE94A4B60467F136D
:10C9860012C2C4EE3395E0FDFCE47B0BFAF9F81213
:10C9960028C4AB29AA2AA92B900002EE8FF01228F0
:10C9A600977F1212C2C4EE3395E0FDFCE47B0BFACE
:10C9B600F9F81228C4AB29AA2AA92B900004EE8FF5
:10C9C600F01228972212C50DEF703F12D921E4907C
:10C9D6001BA2F0A3F0900960E0FEA3E0FF901BA26B
:10C9E600E0FCA3E0FDC39FEC9E502B74002DF58266
:10C9F60074003CF583E0FF12D8FE901BA3E004F020
:10CA060070D3901BA2E004F080CB12D9217BFF7A71
:10CA1600DF79B31243C322753A607539E375381668
:10CA26007537007F007E367D6E7C0112D045E4F5B9
:10CA360022F52374D12523F58274E73522F583E4A4
:10CA460093FF12D88C0523E52370020522C39410A8
:10CA5600E5226480948040DBE4FF12D88C7FF47E6C
:10CA6600017D007C0002BA9785A722E4F5A775FF31
:10CA760080F582F583A3E58264FE458370F7E4F5CD
:10CA860083F582E5FF30E613AF82AE83E4FCFD7BDF
:10CA9600607AEAF9F8D31229EF4003A380E5E5FFAF
:10CAA60030E60575EF02800CE4F5EF7D25AF16AE96
:10CAB60015129C118522A7227B2E7E1C7F227D408B
:10CAC6007C008E3B8F3C8C3D8D3E8B3FAA06A90792
:10CAD6007B0112D7A3EF2401FDE43EFCC3ED953E96
:10CAE600EC953D5020E53C2FF582E53B3EF583E590
:10CAF6003FF0EF2401FFE43EFEE53C2FF582E53BE7
:10CB06003EF583E4F0227E097F607D007B017A009A
:10CB16007900122E5A753A607539E37538167537ED
:10CB2600007F007E367D6E7C0112D045E4F522C37F
:10CB3600E522940974809480500EE52290E6E593F0
:10CB4600FF12D88C052280E77F327E007D007C00B4
:10CB560002BA977E097F607D007B017A0079001218
:10CB66002E5A753A607539E37538167537007F00A9
:10CB76007E367D6E7C0112D045E4F522C3E5229413
:10CB86001174809480500EE52290E6EE93FF12D841
:10CB96008C052280E77F647E007D007C0002BA97C8
:10CBA6007E097F607D007B017A007900122E5A751E
:10CBB6003A607539E37538167537007F007E367D25
:10CBC6006E7C0112D045E4F522C3E52294107480F0
:10CBD6009480500EE52290E6FF93FF12D88C052232
:10CBE60080E77F647E007D007C0002BA97856582BF
:10CBF600856483E47F0AFEFDFCAB69AA68A967A881
:10CC060066D3122A05402FE5829402E583940040FC
:10CC16002578627C1C7D017BFF7AE979FC7E007FAA
:10CC260002122E36EF3395E04F700553E7F7FF22D9
:10CC360053E7F77F01227F01227E017FBE7D007BC5
:10CC4600017A0979A3122E5AE4900B61F0900B65D4
:10CC5600740BF0900B697404F0E4A3F0A3F0A3F056
:10CC6600A3F0A37409F0A3743DF0E4A3F07E04FFDF
:10CC7600FD7B017A0B7971122E5A900BA17455F037
:10CC8600A374AAF022753A607539E37538167537BC
:10CC9600007F007E367D6E7C0112D045E4F528F5D6
:10CCA6002974802529F58274E63528F583E493FFF7
:10CCB60012D88C0529E52970020528C3940DE528AC
:10CCC600940040DD7FE87E037D007C0002BA977504
:10CCD6003A607539E37538167537007F007E367D04
:10CCE6006E7C0112D045E4F522F52374B12523F5B7
:10CCF6008274E63522F583E493FF12D88C0523E58A
:10CD06002370020522C3940DE522940040DD7FE0E6
:10CD16007E937DFF7CFF02BA978D238B2412D81C4D
:10CD26007A00EF4480FB7D167FAC12BA23AF231244
:10CD3600D81C7A00EF4480FB7D157FAC12BA23AF76
:10CD46002412D81C7A00EF4480FB7D137FAC12BA04
:10CD560023AF2512D81C7A00EF5401FB7D147FAC5B
:10CD660002BA23E4901BA2F0A3F0901BA2E475F094
:10CD760001122849FE74A325F0F58274093EF58355
:10CD8600E070E7901BA2E0FEA3E0FF12A2B4EF70F2
:10CD96000512D868800312D87A901BA2E0FEA3E0A1
:10CDA60024A3F974093EFA7B0102D89D8E228F23B3
:10CDB600753A607539E37538167537007F007E362B
:10CDC6007D6E7C0112D045E4F524C3E524941174EC
:10CDD600809480500EE52490E77893FF12D88C0556
:10CDE6002480E7AF2312D88CE522FF12D88C12D903
:10CDF600BA7F0022E4901BA2F0A3F012CB0CEF70D6
:10CE06003712D921E4901BA2F0A3F0901BA2E0FEFA
:10CE1600A3E0FFC3EE9404502274002FF582740041
:10CE26003EF583E0FF12D8FE901BA3E004F070DB12
:10CE3600901BA2E004F080D312D87A2212D82FE4F5
:10CE4600FDAF2685A72F75A710AE07ED4206E5C8EC
:10CE560030E7FB12D82F12D9C5E4FDEDC394087450
:10CE6600809480500A12D5C9EE25E0FE0D80EC12A2
:10CE7600D6A58F30E530600312D7CE852FA7AF3009
:10CE8600227525007524307523017522007F007EEA
:10CE9600607D017C00AB25AA24A923A822C3122AFF
:10CEA600055022AF25AE24AD23AC2212880EE42510
:10CEB60025F525E5243402F524E43523F523E43568
:10CEC60022F52280C8228D238B2412D81CEFFB7AF0
:10CED600007D0E7FAC12BA23AF2312D81CEFFB7A6B
:10CEE600007D0D7FAC12BA23AF2412D81CEFFB7A5B
:10CEF600007D0B7FAC12BA23AF2512D81CEFFB7A4C
:10CF0600007D0C7FAC02BA23E48F258E24F523F531
:10CF160022AD23AC227B37FAF9F81228C48F258E6E
:10CF2600248D238C22E47BE87A03F9F81228C48F37
:10CF3600258E248D238C22E47B997A09F9F812290F
:10CF46004F8F258E248D238C2222900966E0640360
:10CF56006038C29712D8EF90096BEFF0E4A3F09017
:10CF66000966E06402701A90096BE06014E4F51437
:10CF76007D21AF16AE15129C119009687402F080DF
:10CF8600069009687403F012D46F227B017A09793E
:10CF9600A3127453E4901BA2F0A3F0901BA2E0FE30
:10CFA600A3E0FFC3EE9404501F74A32FF582740907
:10CFB6003EF583E0FF12D8FE901BA3E004F070DB81
:10CFC600901BA2E004F080D322ABA775A70FC28EF8
:10CFD60053C7FD75A710859932C298C29975A70FD8
:10CFE60075D4CF75D50F43C7028BA78531448530DD
:10CFF60043852F42852E41127C437E007F007D6053
:10D006007C0902D67B85A73075A70F53E7F7C28E3A
:10D0160053C7FD75A710859931C298C29975A70F98
:10D0260075D4CF75D50343C702852F44852E438516
:10D036002D42852C41127C4343E7088530A7228583
:10D04600A73B75A70F53E7F7C28E53C7FD75A71009
:10D0560085993CC298C29975A70F75D4CFE4F5D5CA
:10D0660043C702853A44853943853842853741129C
:10D076007C4343E708853BA7228D228B2312D81CCD
:10D086007A00EF4480FB7D127FAC12BA23AF2212E6
:10D09600D81C7A00EF4480FB7D117FAC12BA23AF17
:10D0A6002312D81C7A00EF4480FB7D107FAC02BAB5
:10D0B60023AEA7E4F5A78FBBD2ECFF20ED0DEFC39F
:10D0C60094647480948050030F80F0C2EDEFC39493
:10D0D600647480948040067C067D008004ACBEADFE
:10D0E600BD8EA7AF05AE04228B288A29892A8C2BF0
:10D0F6008D2CE4FFE52C152CAC2B7002152B4C6007
:10D1060015AB28052AE52AAA297002052914F91261
:10D1160026FB2FFF80DEEF75F0FFA4FF221294B1ED
:10D126008F258E248D238C22EC4D4E4F601712D9FD
:10D13600217BFF7AE079EA852539852438852337EE
:10D14600852236800912D9217BFF7AE079FF1243C6
:10D15600C3227D09AF16AE15129C117B017A0079A8
:10D166000012D5A7EF700F1299EE7D1CAF16AE1503
:10D17600129C117F002212DA437D12AF16AE1512F1
:10D186009C117F01228E288F29EF2401FFE43EFEA9
:10D196008D2E7B01E4FD12565878AD7C1B7D017EF9
:10D1A600007F031226D5901BADE085298285288352
:10D1B600F07B017A1B79AD228D228B2312D81CEFCE
:10D1C600FB7A007D0A7FAC12BA23AF2212D81CEF7D
:10D1D600FB7A007D097FAC12BA23AF2312D81CEF6D
:10D1E600FB7A007D087FAC02BA23AFA775A70F753F
:10D1F600F1FE75F30375F4F875A41275A59575A679
:10D206000375AE7875AF0375D4CF75E10175C74266
:10D21600E4F5B575B00775A0FC8FA7228F828E83C3
:10D2260012D7E012DA2412D842AF82AE83E4FCFDB4
:10D23600AB0DAA0CA90BA80AD3122A0540EB12D9EA
:10D24600AF12DA28E4F50DF50CF50BF50A228F225C
:10D256008D237F6F12D8FE7F6B12D8FEAF2212D8B5
:10D26600FEAF2312D8FE752404C3E52494407480CF
:10D2760094805009E4FF12D8FE052480EC228F2208
:10D286008D237F6E12D8FE7F6F12D8FEAF2212D882
:10D29600FEAF2312D8FE752404C3E524944074809F
:10D2A60094805009E4FF12D8FE052480EC227E000B
:10D2B6007F007DFF7C0312D41C901BACEFF0600B4B
:10D2C60012C5C3901BADE4F0A3EFF078A37C097DF3
:10D2D600017B017A0079007E047F000226D5C0E03A
:10D2E600C083C082C0D075D000C007309813C298E2
:10D2F600AF63056374002FF582E43400F583E59986
:10D30600F0D007D0D0D082D083D0E0328F231299CC
:10D31600EE12DA3A8F118E108D0F8C0E12DA43ADA3
:10D3260023AF16AE15129C11124C0C9009687405A9
:10D33600F07D01AF16AE15029C119009A374EBF0B7
:10D34600A37458F0A37490F0A37445F0A3744CF042
:10D35600A37449F0A37443F0A3744FF0A3744DF083
:10D36600E4A3F0A37430F0228F2212D9217F6F122A
:10D37600D8FE7F6B12D8FEAF2212D8FE752303C3E8
:10D38600E5239440748094805009E4FF12D8FE058A
:10D396002380EC228F2212D9217F6E12D8FE7F6F56
:10D3A60012D8FEAF2212D8FE752303C3E52394409C
:10D3B600748094805009E4FF12D8FE052380EC2285
:10D3C600AFA7E4F5A743BC0175BE0475BD7C75BE69
:10D3D60007F5BD75BE0875BD0153BCFE75BB30753E
:10D3E600BC3875E8C075D1178FA72212D734E490E0
:10D3F600096CF012CE877527FF7528E275296390B0
:10D406000964E0FAA3E0FB7D20AF16AE1512794C55
:10D41600E4FFFE02CDB28E328F337FFFED1DAA04EC
:10D4260070011C4A60190533E533AA3270020532D1
:10D4360014F5828A83E06FFE90E7FF93FF80DD227A
:10D446007D027F8012A855901B9DE0FEA3E024007C
:10D45600FFE43EFEEF7803CEC313CE13D8F978026D
:10D46600C333CE33CED8F9FF22AFA775A70F8FA748
:10D47600E4FF12D74BE4FF122006E4FF122096E4E5
:10D48600FF12D761E4FF12DA1312D9D912DA300289
:10D49600D998E5176006E4F517128F97125EAEEF7E
:10D4A600700C12D9CF122E9812D9D912729CE5148B
:10D4B60064017005F51412D73422E4901BA2F0A380
:10D4C600F0901BA2E475F001122849FE74A325F022
:10D4D600F58274093EF583E070E790096C04F0026A
:10D4E600D868C29712C451EF70137F0112D74B123E
:10D4F600D98C12D9217BFF7AE27917800912D921BA
:10D506007BFF7AE279271243C322AEA775A710E400
:10D51600FDFCECC39408748094805010ED25E0FD6A
:10D526005305FE12D6A5EF42050C80E68EA7AF0581
:10D5360022AE07E4FDEDC3940874809480500A126D
:10D54600D5C9EE25E0FE0D80EC12D6A58F2FE52F6E
:10D55600600312D7CEAF2F2212D9217BFF7AE27950
:10D566003790096FE0FCA3E0FDA3E0FEA3E0F539E8
:10D576008E388D378C361243C3E4FF02D8FEAFA730
:10D5860075A70F759F3075A7107592FF7593FE7579
:10D5960094FF7595FE4396104391048FA743E78049
:10D5A600228B238A248925754A04754B007F007EC9
:10D5B600507D017C0012BF06AE24AF257D007C04A1
:10D5C60002D41CEEC41313135401FFC287EF24FFC9
:10D5D6009286E5C830E7FB12D82FD287E5C830E738
:10D5E600FB02D82FC0E0C0D053917FE50D2401F592
:10D5F6000DE4350CF50CE4350BF50BE4350AF50AAC
:10D60600D0D0D0E032E4FFFE12BF74EF700B12D917
:10D61600217BFF7ADF7915800912D9217BFF7ADF1A
:10D62600792B1243C322C0E0C0D0C2CFE5692401E2
:10D63600F569E43568F568E43567F567E43566F558
:10D6460066D0D0D0E0328F298E288D278C26AF2940
:10D65600AE28AD27AC26AB0DAA0CA90BA80AD3128F
:10D666002A0540EA22F569F568F567F5667E007FCA
:10D67600007D607C098E6A8F6BE4F564F5658C6CC1
:10D686008D6D22EFFD3395E0FCD3ED9439EC64808B
:10D6960094805006C3EF9430FF22EF24C9FF22D2B4
:10D6A60086C287E5C830E7FB12D82FD287A286E468
:10D6B60033FFE5C830E7FB02D82F7B017A007D01F6
:10D6C6007FAC12BA237B017A007D027FAC12BA23AB
:10D6D60002D8E0C0E0C083C08253917F75170190E5
:10D6E600096E7401F0D082D083D0E032900968745C
:0ED6F60001F0E4FF12DA1302D8685390F32219
:07D7080043900C5390F7223F
:07D7100043900C5390FB2233
:10D7180043900C22AFA7E4F5A775CBFE75CA0B851D
:10D72800CBCD85CACCD2CAD2AD8FA722E4FBFA7D75
:10D73800017FAC12BA23E4FBFA7D027FAC12BA2354
:10D7480002DA348F277F327E0012D222E52724FFA7
:10D7580092B37F647E0002D2228F277F327E00122E
:10D76800D222E52724FF92B67FF47E0102D2227FDF
:10D77800907E087D007C0012B64B7E007F007DFF06
:10D788007C0302D41C12D8EFEF6401700D12D9216A
:10D798007F0112D8FE7FEB12D8FE22E4FFFE12268C
:10D7A800FB600C0FEF70010E09E970F20A80EF229E
:10D7B800901B9DE0FFEFC4540F75F00AA4FEEF54D0
:10D7C8000F2EFF22EFF07F0112D5D1E4FF12D5D141
:10D7D800E4F5C8D286D28722AFA7E4F5A77593F8F7
:10D7E80075922F8593958592948FA722900968E06A
:10D7F800640870087F0112DA1302D86812D87A22F6
:10D8080012D92112A01F7BFF7AE179731243C3E476
:10D81800FF02D8FEEF75F00A84C454F0FEEF75F0ED
:10D828000A84E5F04EFF22E4F5C875CBFF75CAE619
:10D8380075CDFF75CCE675C80422ABA7E4F50DF5E8
:10D848000CF50BF50AF5A74391048BA722EFC394B7
:10D85800094005EF940E4003BF2003D38001C32283
:10D8680012D9217F6F12D8FE7F6B12D8FEE4FF0217
:10D87800D8FE12D9217F6E12D8FE7F6F12D8FEE42F
:10D88800FF02D8FEAEA775A710C2998F993099FDEF
:10D89800C2998EA7227542047543007F007E507D91
:10D8A800017C0002BFE1E4FF12200612D9217BFFB0
:10D8B8007AE179940243C37F0112200612D9217BB1
:10D8C800FF7AE179AB0243C37BFF7ADE79FA124330
:10D8D800C3E4F5A775EF1022AFA775A70F75E40687
:10D8E8008FA7D296D2A8227D017FAC12A855901B93
:10D8F8009DE05401FF22AEA7E4F5A78F993099FD6A
:10D90800C2998EA722AEA7E4F5A78F993099FDC2D8
:10D91800998EA722EEF0A3EFF07F0A12D8FE7F3E81
:10D9280002D8FE123A6012D9217BFF7ADF79A3026E
:10D9380043C3EFC394204007EF947F50028001C394
:10D9480022EFC394304007EF943A50028001C3227B
:10D95800AD077FAC12A855901B9DE0FF22AE05AD28
:10D9680007EEFB7A007FAC02BA2312CBF3EF700309
:10D9780002D86812D87A2212BC63EF700302D86802
:10D9880012D87A22C2A07FC87E0012D222D2A02248
:10D9980085A72775A70F53ABBFC2AC22AFA775A742
:10D9A8000F75A1C78FA722AFA7E4F5A75391FB8FE7
:10D9B800A7227E1C7F627D3F7C0002D67BC286E563
:10D9C800C830E7FB02D82F43B5017F017E0002D2A1
:10D9D8002253B5FE7F017E0002D2229009687408A6
:10D9E800F002D8689009687401F002D868EF6D9069
:10D9F800E7FF93FF2212D1F0D297027EEF75140150
:10DA080012DA3432E4F5A753D9BF22EF24FF92A1EA
:10DA18002212D73402D8687EE27F632243E640228E
:10DA280053E6BF2243B5022253B5FD22C2A822D233
:10DA3800AF220294B102D86802B8B802907B202DB8
:10DA4800204177616974696E6720726567697374CC
:10DA5800726174696F6E2E2E2E00202D205265671C
:10DA6800697374726174696F6E206D6F646520618B
:10DA780063746976652E00202D205265676973747A
:10DA8800726174696F6E206D6F646520636F6E6379
:10DA98006C756465642E00202D20526573746F7256
:10DAA800696E6720726567697374726174696F6EF5
:10DAB800206D6F64652E2E2E00202D204E6F207253
:10DAC8006573706F6E73652066726F6D206465761E
:10DAD8006963652E00202D2053686F727420636976
:10DAE80072637569742064657465637465643A204B
:10DAF80000202D205A65726F20706F776572206341
:10DB08006F6E73756D7074696F6E3A2000202D20EA
:10DB18004572726F7220726563656976696E6720F7
:10DB2800646174612066726F6D20646576696365EF
:10DB38002E00202D20494D504143542065786365BF
:10DB48006564696E67206465746563743A200020B3
:10DB58002D20275461736B272066696C65206D69D9
:10DB68007373696E6720696E204E414E442E002003
:10DB78002D20566F6C7461676520526567756C61FE
:10DB8800746F722044726F706F7574206465746569
:10DB9800637465642E00202D20705F616464726573
:10DBA8007373206F766572666C6F773A2000202D4C
:10DBB8002048525A5F73697A653A2000202D205711
:10DBC80061726E696E672C20536D61727420737771
:10DBD80069746368206F75743A2000202D2057619E
:10DBE800726E696E672C207468652066757365208F
:10DBF80069732063726173682E00202D205761724B
:10DC08006E696E672C20556261742044726F706F64
:10DC18007574206465746563743A2000202D20575C
:10DC280061726E696E673A2052656720537461723B
:10DC38007420776974682054656D702E00202D203B
:10DC4800275461736B272066696C65206D6973734F
:10DC5800696E6720696E20466C6173682E00202DFE
:10DC68002052544320416C61726D20747269676759
:10DC7800657265642E00202D2053746172742052E1
:10DC88006567697374726174696F6E204475652085
:10DC9800746F2074696D65206D617463682E00204F
:10DCA8002D2045565420666F7220415220746F20F3
:10DCB80053657269616C206E756D6265723A2000F9
:10DCC800202D204572726F722077726974696E67B1
:10DCD80020746F20666C6173682073746F7261675B
:10DCE800652E2000202D205761746368646F6720BB
:10DCF80054696D6572205265736574207472696722
:10DD080067657265642E00202D2053797374656DE4
:10DD18002073757370656E6465642064756520741E
:10DD28006F20706F776572206973737565732E0045
:10DD3800202D20416C61726D206E6F7420736574A4
:10DD48002E00202D204177616974696E67206D6F00
:10DD5800646520286E6F2062617474657279207022
:10DD68006F7765722900202D2048656164657220EF
:10DD780048525A207375636365737366756C6C7962
:10DD880020726561642E00202D20275461736B2753
:10DD98002066696C652067657420696E20466C6131
:10DDA80073682E00202D20526567206D6F646520F2
:10DDB8006D6573736167653A206E6F204261747494
:10DDC80065727920706F77657200202D2052656723
:10DDD800206D6F6465206D6573736167653A2054C3
:10DDE800696D6520656E6400202D205254432072B1
:10DDF800656164206D616A6F726974792066617506
:10DE08006C742E00202D2053657269616C206E752C
:10DE18006D6265722026206669726D776172652071
:10DE280076657273696F6E3A2000202D2041776104
:10DE38006974696E67206D6F6465206166746572C8
:10DE4800204C494E4B2073746174652E00202D20A0
:10DE5800526567206D6F6465206D657373616765D2
:10DE68003A2055534220706F77657220636F6E6E4B
:10DE7800656374656400202D20494D50414354204A
:10DE88006F766572203135673A2000202D20546165
:10DE9800736B207061727365206572726F722E00E9
:10DEA800202D20564444204D6F6E69746F722046B1
:10DEB80061696C65642064657465637465642E00CB
:10DEC800202D20556E6B6E6F776E206576656E74AB
:10DED8002E0030006D470020006C6F616465720091
:10DEE8007265736574006572617365007772697431
:10DEF800650052657365742053797374656D0A0DF6
:10DF0800004D617920313920323032360046696C53
:10DF1800652073797374656D2063726561746564D7
:10DF28000A0D0046696C652073797374656D206EFF
:10DF38006F7420637265617465640A0D000A0D00D0
:10DF48004572726F722072656164696E67204F6EE8
:10DF580066692061727261790A0D00577269746589
:10DF68004C6F676963616C50616765204F4B2C206B
:10DF780070616765203D20256C640057726974657F
:10DF88004C6F676963616C50616765204E4F2C2048
:10DF980070616765203D20256C64005365744B6192
:10DFA80074616C6F67204F4B0A0D006E6F7420729E
:10DFB8006573706F6E73696E6720666F7220636F2A
:10DFC8006D6D616E64204E616E6447657454617353
:10DFD8006B006E6F7420726573706F6E7369672063
:10DFE800666F7220636F6D6D616E64205265616447
:10DFF800506879736963616C416464726573730016
:10E008006E6F7420526573706F6E73696E672066E9
:10E018006F7220636F6D6D616E6420457261736508
:10E02800426C6F636B006E6F7420526573706F6E15
:10E0380073696E6720666F7220636F6D6D616E64C1
:10E0480020536574446174610A0D00467265652049
:10E0580041646472657373203D20256C640A0D0069
:10E068006E6F7420726573706F6E73696E67206669
:10E078006F7220636F6D6D616E64204765745461C3
:10E08800736B0A0D006E6F7420726573706F6E7318
:10E09800696E6720666F7220636F6D6D616E6420B4
:10E0A8005465726D696E616C476574506167650A85
:10E0B8000D004E6F74206D6F7665204B6174616C36
:10E0C8006F670A0D004E6F74206765742048727A76
:10E0D8000A0D004E6F74207772697465207061674D
:10E0E8006500667265652061646472657373203DBE
:10E0F80020256C640A0D006E6F74206672656520B9
:10E10800616464726573730A0D00777269746520BF
:10E11800256C642061646472657373203D20737597
:10E128006363657373007772697465206661696CEF
:10E138006564004572726F725072657061726552E3
:10E148006573746F7265004572726F725265737091
:10E158006F6E7365526573746F726546617433329E
:10E16800636F6D6D616E64004F4B006F6B0072657D
:10E17800616420616464726573733D256C6420007A
:10E1880072656164206661696C65640052656769DF
:10E198007374726174696F6E20706F776572204F47
:10E1A800464600526567697374617274696F6E20C0
:10E1B800706F776572204F4E004D6F76654B6174B6
:10E1C800616C6F6720737563636573730A0D00472D
:10E1D800657448727A20737563636573730A0D00FA
:10E1E80057726974652048525A20426F64792073C7
:10E1F8007563636573730A0D005772697465204807
:10E20800525A20426F6479206661696C0A0D005386
:10E2180065745573624D6F6465204F4B0A0D00534A
:10E2280065745573624D6F6465204E4F0A0D002565
:10E238006C6400253032642F253032642F2530324B
:10E248006420253032643A253032643A253032640D
:10E258000A0D0041525F31353000005F332E310026
:10E2680000000030372E30322E3235004572726F82
:10E278007250726570617265526573746F72650071
:10E288006C6F61646572006669726D776172655F53
:10E298007665720074657374007263616C007763ED
:10E2A800616C0067657474696D6500636C6600670E
:10E2B800616C006368617267657265670073657495
:10E2C80074696D6500617574680073657461736D58
:10E2D8000067640067645F61300067645F613100F4
:10E2E80067645F61320067645F6133007365745F00
:10E2F800706172616D00666173745F636C656172F1
:10E3080000777269746570616765006261636B7537
:10E31800705F7461736B00636865636B0063686B3F
:10E328006F66660063686B6F6E00636F6E00636F85
:10E33800666600706F737473796E6300636C6561F1
:10E348007200436C65617200726561640072656198
:10E3580064706167650063726561746566696C65A0
:10E368000043726561746546696C65006261747426
:10E378006572795F6F6B00626174746572795F6949
:10E388006E660077726974655F7068797369636136
:10E398006C5F7061676500726561645F706879734E
:10E3A8006963616C5F706167650065726173655F61
:10E3B800626C6F636B00746573745F726571756509
:10E3C8007374006E616E645F696E6974006E616E6D
:10E3D800645F6F6E66695F72656164006572617320
:10E3E800655F656E6400577269746541646472653F
:10E3F8007373546573740052656164416464726533
:10E4080073735465737400706567697374726174AB
:10E41800696F6E5F706F7765725F646F776E007299
:10E428006567697374726174696F6E5F706F776521
:10E43800725F7570006E616E645F6C6F61646572A7
:10E44800004765744E616E64436F6D70696C655604
:10E458006572004E616E644765745461736B005257
:10E468006573746F726546617433320057726974EC
:10E47800654C6F676963616C5061676500526561DF
:10E48800644C6F676963616C5061676500476574C8
:10E498004576656E745061676500726566617400E3
:10E4A80072656661745F737461747573004765742F
:10E4B80052756E6E696E6754696D65005265736555
:10E4C8007452756E6E696E6754696D650047657440
:10E4D8004576744D657373616765004765744F6E63
:10E4E80066690047657450616765004765745061E7
:10E4F800676531004765745061676532005365741C
:10E50800466174333200526573657400476574540C
:10E5180061736B005365745461736B005365744B7E
:10E528006174616C6F6700536574506F73747379AD
:10E538006E6300476574467265654164647265730D
:10E5480073005365745573624D6F64650053657449
:10E55800446174610047657454696D6500696400BD
:10E56800556E6B6E6F776E20636F6D6D616E640AAA
:10E578000D00256C64002564004F4B002530326483
:10E588002F253032642F2530326420253032643A0A
:10E59800253032643A25303264006F6B004E616E6C
:10E5A80064496E69740041545F575F315F48414C5C
:10E5B800460041545F575F325F48414C4600457200
:10E5C8006173655461736B426F6479004765744683
:10E5D8007265654164647265737300526561645065
:10E5E800616765466F725068795061676500476575
:10E5F8007448727A426F6479004572617365487233
:10E608007A426F6479004D6F76654B6174616C6F07
:10E618006700476574467265654164647265737323
:10E628005465737400526561644164647265737300
:10E6380054657374005772697465416464726573D4
:10E64800735465737400476574436F6D70696C65C6
:10E6580044617461005F6C6F61646572000016E369
:10E6680060001E8480536574526573746F726554BC
:10E6780061736B426F6479005365744576656E7497
:10E68800426F647900536574526573746F7265489C
:10E69800525A426F647900536574526573746F728D
:10E6A800654B6174616C6F6700526573746F726556
:10E6B80046617433320057726974655068795061E5
:10E6C8006765005265616450687950616765004507
:10E6D80072617365426C6F636B00415400526561EF
:10E6E800644F6E666900537461727452656275692D
:10E6F8006C644E616E640052656275696C64507238
:10E708006F6772657373005465726D696E616C53DF
:10E71800657444617461005365744576740052658C
:10E7280061645061676500476574457674426F643B
:10E7380079466972737448616C66004765744576FA
:10E7480074426F64795365636F6E6448616C6600E8
:10E75800536574457674496E666F005772697465BF
:10E76800506167650057726974653250616765006A
:10E7780043726561746546696C6553797374656D38
:10E788000052657365744576656E744C6F674669AB
:10E798006C65005365745573624D6F646500476519
:10E7A800745461736B426F64790047657448727A78
:10E7B800426F64795769746844617465005365747D
:10E7C8005461736B426F6479005465726D696E6150
:10E7D8006C5365745461736B0053657448727A4264
:10E7E8006F64795769746844617465005365744847
:10E7F800727A426F647900005EBCE2613FDD83C2D9
:10E808009C7E20A3FD1F419DC3217FFCA2401E5F6B
:10E8180001E3BD3E6082DC237D9FC1421CFEA0E176
:10E82800BF5D0380DE3C62BEE0025CDF81633D7C4D
:10E8380022C09E1D43A1FF4618FAA427799BC584D0
:10E84800DA3866E5BB5907DB856739BAE406581933
:10E8580047A5FB7826C49A653BD987045AB8E6A72A
:10E86800F91B45C6987A24F8A6441A99C7257B3A15
:10E878006486D85B05E7B98CD2306EEDB3510F4E84
:10E8880010F2AC2F7193CD114FADF3702ECC92D303
:10E898008D6F31B2EC0E50AFF1134DCE90722C6DDE
:10E8A80033D18F0C52B0EE326C8ED0530DEFB1F0E5
:10E8B800AE4C1291CF2D73CA947628ABF517490840
:10E8C80056B4EA6937D58B5709EBB536688AD495BB
:10E8D800CB2977F4AA4816E9B7550B88D6346A2BA2
:10E8E8007597C94A14F6A8742AC896154BA9F7B69D
:10E8F800E80A54D7896B3542200049006E0066004B
:10E908006F000F007272006D006100740069006F83
:10E918000000006E000000015300790073007400CD
:10E9280065000F00726D00200056006F006C0075C6
:10E938000000006D00650053595354454D7E312049
:10E94800202016009F13918F558F55000014918F2A
:10E95800550300000000005441534B202020202084
:10E96800202020000126918F558F5500008A5E8F48
:10E97800550A00000400004556454E544C4F475474
:10E98800585420006C5C89525752570000708752C7
:10E998005706000010000041474743202020204828
:10E9A800525A2000B333918F558F550000A4788FA9
:10E9B800550B0000E06CF76D412E006D562E00706F
:10E9C800616765000000010001000100000000000F
:10E9D800000000000000010000000000000000002E
:10E9E800000000000000010001000000000000001D
:0DE9F800000000004F4B006D4700000000C4
:00000001FF
